:020000040800F2
:100000000000012055410008ED270008EF270008F7
:10001000F1270008F3270008F5270008000000007A
:10002000000000000000000000000000F7270008AA
:10003000F927000800000000FB270008FD27000842
:10004000A5410008A541000801280008A5410008B5
:10005000A5410008A54100080D2800081328000844
:10006000A5410008A54100083B280008A54100085B
:10007000192800081B2800081D2800082928000846
:100080003528000837280008A5410008A5410008C8
:1000900000000000A54100083D280008A541000817
:1000A000A5410008A5410008A5410008A541000898
:1000B000A5410008A5410008A5410008A541000888
:1000C000A5410008A5410008A5410008A541000878
:1000D000A541000845280008A5410008A5410008E1
:1000E000A54100084328000851280008A541000840
:1000F000A54100080000000000000000A541000824
:10010000A5410008A54100085D280008A541000898
:10011000A5410008A5410008A5410008A541000827
:10012000A5410008A5410008A5410008A541000817
:08013000A5410008A5410008EB
:1001380010B5054C237833B9044B13B10448AFF319
:1001480000800123237010BDBC08002000000000BF
:100158001840010808B5034B1BB103490348AFF326
:10016800008008BD00000000C008002018400108F9
:1001780014214160704714207047406A704700009E
:10018800790100087F01000883010008990100082F
:1001980010B5044604F1100000F05CFCC4F8F80047
:1001A8000148C4F87C0110BD88010008F8B5E6B024
:1001B80004460D4616461F460A4906A800F0CAFE20
:1001C80070996F9A05910492009733466E996D9ACB
:1001D800039102922A466C990191214600F060F839
:1001E80067B0F0BD94010008F8B5E6B004460D46C6
:1001F80016461F46094906A800F0ACFE6F996E9A8C
:100208000491039200976D996C9A0291019233467A
:100218002A46214600F087F867B0F0BD940100082F
:1002280038B500281CBF01680029184A23D1184B8B
:100238001C684FF6F0710C404CF24025AC421FBFD1
:100248001B6819404CF27024A14212D1114D296843
:1002580079B911490B68C3F30B03B3F58A6F1FBF54
:100268000968C1F30B0140F28343994204BF01219D
:10027800117028B905E0094B994204BF012111709A
:100288004068BDE8324001F09FBE00BFD80800209A
:1002980000ED00E0002004E00010005C000037489A
:1002A8002DE9F04104460D46216816464A681F4666
:1002B80090478046B8F5403F2ED122680A99936846
:1002C800204698478046B8F5403F25D12368089ACC
:1002D8000799D3F80CC02046E0478046B8F5403F60
:1002E8001AD12368069A39461F692046B8478046BE
:1002F800B8F5403F10D1236829465D69324620464B
:10030800A8478046B8F5403F06D123680B9A09995B
:100318009D692046A847804621680A68204690477C
:100328004046BDE8F0812DE9F04104460D462168BC
:1003380016464A681F4690478046B8F5403F2ED17A
:1003480022680A999368204698478046B8F5403F46
:1003580025D12368089A0799D3F80CC02046E047AE
:100368008046B8F5403F1AD12368069A39461F6976
:100378002046B8478046B8F5403F10D12368294643
:100388005D6932462046A8478046B8F5403F06D109
:1003980023680999DD6900222046A847804621681C
:1003A8000A68204690474046BDE8F0814FF4403047
:1003B80070470000F0B50C4685B0114600281A4673
:1003C8001CBF0568002D0B4B11D082B104B971B95F
:1003D8000D9860B10F9E0E9F0A9B0290049603979A
:1003E8000B980C9E009001962046A8470346184695
:1003F80005B0F0BD020003002DE9F04F0646D0B06D
:100408000868F56DD6F860E0726EB76EF36E00BAE4
:1004180000906C46486800BA60600DF14008886832
:1004280000BAA060C86800BAE060086900BA206134
:10043800486900BA6061886900BAA061C86900BAF1
:10044800E061086A00BA2062486A00BA6062886A95
:1004580000BAA062C86A00BAE062086B00BA2063FA
:10046800486B00BA6063886B00BAA063C86B00BAB7
:10047800E063402058F80C1C58F820CC58F838ACE9
:100488008CEA010158F840CC8AEA01018CEA01099A
:100498004FEAF979401E48F8049BEBD187EA02003D
:1004A80000EA0E00784010EBF5610098DFF824C4EC
:1004B80041186144C81882EABE032B404FEAF06134
:1004C80053405918636859186144CF194FEAB50366
:1004D80083EABE01014081EABE0111EBF765A1681C
:1004E8004D196544A91883EAB0023A404FEAF1650C
:1004F8005A405519E26855194FEAB70282EAB0071F
:1005080065440F4005EBBE0E97EAB00717EBFE6592
:1005180027697D194FEAB10782EA0701654401EAB4
:100528000E01EB18514011EBF36561694D194FEA63
:10053800BE0187EA010E65440EEA030E15EBB00012
:100548008EEA070E0EEBF065D4F818E075446544A2
:10055800AA1881EAB30505404FEAF26E4D40AE4451
:10056800E569AE44E64477444FEAB00080EAB30E4A
:100578000EEA020E8EEAB30E0EEBF765D4F820E011
:1005880075446544691880EAB2053D404FEAF16E4A
:100598004540AE44656AAE44E6440EEBB3034FEA09
:1005A800B70787EAB20E0EEA010E8EEAB20E0EEB1C
:1005B800F365D4F828E075446544281887EAB1053E
:1005C8001D404FEAF06E7D40AE44E56AAE44E64415
:1005D8000EEBB2024FEAB30383EAB10E0EEA000E45
:1005E8008EEAB10E0EEBF265D4F830E0754465443E
:1005F800EF1983EAB00515404FEAF76E5D40AE4447
:10060800656BAE44E6440EEBB1014FEAB20282EAF2
:10061800B00E0EEA070E8EEAB00E0EEBF165D4F8B6
:1006280038E075446544EB1882EAB7050D404FEA97
:10063800F36E5540AE44E56BAE44E6440EEBB000B5
:100648004FEAB10181EAB70E0EEA030E8EEAB70E41
:100658000EEBF065D4F840E07544654481EAB30ECA
:10066800AA180EEA000E4FEAF2658EEA010E7544EA
:10067800DDF844E04FEAB000754480EAB30E654403
:100688000EEA020E15EBB7078EEAB30E0EEBF7650E
:10069800DDF848E04FEAB202754480EA020E65448C
:1006A8000EEA070E69188EEA000E0EEBF165DDF80A
:1006B8004CE07544654405EBB3034FEAB70E1427C5
:1006C8000DF1500CDFF810528EEA010B82EA0B0B89
:1006D8000BEBF36A5CF804BBDA44AA44504483EA9F
:1006E800B10B4FEAF06A8EEA0B0BDA445CF804BBF4
:1006F800DA44AA44524480EAB30B4FEAF26A8BEA1E
:10070800B10BDA445CF804BBDA444FEAB000AA44FF
:1007180080EA020BD6448BEAB30B0BEBFE6A5CF85B
:1007280004BBDA444FEAB202AA4482EA0E0B0AEB8F
:10073800B10180EA0B0B0BEBF16A5CF804BBDA44FD
:100748007F1DAA44282F0AEBB3034FEABE0EBBD382
:100758003C2F61D3502F4DD204EB870CC7F15407BF
:100768005E4CA7FB04A504465D4FA8088EEA010A63
:1007780082EA0A0A5CF804BB0AEBF3655D447D195A
:100788002C1983EAB10A4FEAF4658EEA0A0A55443D
:100798005CF804AB5CF804BB55447D19AA1884EADC
:1007A800B30A4FEAF2658AEAB10A55445D444FEA52
:1007B800B4047D1984EA020AAE448AEAB30A0AEB51
:1007C800FE655CF804AB55444FEAB2027D1982EA33
:1007D8000E0A15EBB10184EA0A0A5CF804BB0AEBBD
:1007E800F1655D447D1915EBB303401E4FEABE0E5B
:1007F800BCD12046F46D1B19F365336EC9183166F8
:10080800716E71447166B36ED218B266F16E40189B
:10081800F06650B0BDE8F08F4EEA010B0EEA010A0F
:100828000BEA020B4BEA0A0A0AEBF36554F827A015
:10083800DFF8B0C0554443EAB10B654403EAB10A96
:100848000BEA0E0B28184BEA0A0A7F1C0AEBF06524
:1008580054F827A0554440EAB30B654400EAB30AAC
:100868000BEAB10BAA184BEA0A0A7F1C0AEBF265DD
:1008780054F827A055444FEAB00040EA020B6544FB
:1008880000EA020A0BEAB30BAE444BEA0A0A7F1CE1
:100898000AEBFE6554F827A055444FEAB20242EA33
:1008A8000E0B654402EA0E0A0BEA000B15EBB101C8
:1008B8004BEA0A0A7F1C0AEBF16554F827A0554455
:1008C8007F1C65443C2F05EBB3034FEABE0EA3D350
:1008D80040E700BF9979825AA1EBD96ECDCCCCCC38
:1008E800D6C162CADCBC1B8F00B581B00168074A5B
:1008F800914200D110B9064801B000BD7C2113F027
:10090800EFFA4FF4003001B000BD00BFFC09000849
:10091800030002002DE9F0410B4A92E8F85188B033
:10092800694681E8F8510268084B9A4200D118B923
:10093800074808B0BDE8F0811422083000F04FFBEA
:1009480008B0BDE8F08100BFDC090008FC09000818
:1009580003000200152904D20268044B9A4200D110
:1009680008B903487047083000F048BBFC09000884
:100978000300020010B481B013460268074CA2427B
:1009880000D118B901B010BC0548704701B000F19A
:10099800240210BC083000F035BB00BFFC09000879
:1009A8000300020010B481B013460268074CA2424B
:1009B80000D118B901B010BC054870470A4601B00B
:1009C80000F1240110BC083000F070BBFC090008DD
:1009D800030002000123456789ABCDEFFEDCBA981E
:1009E80076543210F0E1D2C300000000000000008D
:1009F80000000000F10800081D0900085D09000852
:100A08007D090008AD09000801040008790F0008F5
:100A1800C50F0008810F0008F0B5A3B004460B48C5
:100A280002900D4616461F46094B0822402104A88D
:100A380000F0D1FA28980190009733462A462146BB
:100A480002A800F01BF823B0F0BD00BFFC090008A5
:100A5800100A000810B5040008BF002408D0054893
:100A6800054B20600822402104F1080000F0B3FA89
:100A7800204610BDFC090008100A00082DE9F041C5
:100A880004460E46216817464A681D469047804628
:100A9800B8F5003F19D1226806999368204698470F
:100AA8008046B8F5003F10D123683146DE683A46E3
:100AB8002046B0478046B8F5003F06D12368079A1C
:100AC80029461D692046A847804621680A682046AD
:100AD80090474046BDE8F08110B500F033FA4FF476
:100AE800403400280EBF034C4FF4C07113F0F8F9DE
:100AF800204610BD0200030010B5044600F022FA9B
:100B080008B9054810BD0021A160D0F87C21116802
:100B180088474FF4403010BD0200030070B504460A
:100B28000D4600F00FFA064E40B1D0F87C0141683E
:100B38008847A84224BF65604FF44036304670BDF0
:100B4800020003002DE9FF4715000C4600D02CB128
:100B5800064600F0F7F95FEA000801D16448C3E0EF
:100B6800D8F8F80001684A689047B0F5003F17D1F7
:100B7800D8F87C118A68404690478146B9F1810FC0
:100B880080F09E80A94508F1FC0A17D2D8F8F80031
:100B98000368D3F80CC02A462146E047B0F5003F69
:100BA80040F08E80D8F8F8000368D3F810C06A4681
:100BB8005146E047B0F5003F76D10AE0002004E056
:100BC800215C0AF800100098401C00900098A84288
:100BD800F6D34FF0000C4749474A484B01AC009800
:100BE800844558D2D3E9007001ADC5E9007010788A
:100BF80000281ABF042086464FF0000E085854F803
:100C08000E5028443E4D05600127D0F800E087606B
:100C1800019D4F681AF80C007D408EEA050585F0A5
:100C2800040E65680F687D4085F0FC05754485F005
:100C3800A30568400AF80C000CF1010CCFE7D3E9D2
:100C4800004501A8C0E9004510782E4D002814BFC2
:100C58004FF0040E4FF0000E01A8744651F80EE054
:100C68000459A6440127CEF80050DEF80040CEF81B
:100C780008704D68019F40687D406C400D68684071
:100C880084F0040480F0FC00041984F057040AF886
:100C98000C400CF1010CCC45D1D3D8F8F800016810
:100CA8004A689047B0F5003F0AD1D8F8F8000368C1
:100CB800D3F80C804A465146C047B0F5003F01D0F2
:100CC800114811E0002006E05AF8201081F06A313E
:100CD8004AF82010401CB0EB990FF5D3B06840F0EB
:100CE8000100B0604FF4403004B0BDE8F08700BFA9
:100CF80002000300B0400108D8080020240F0008B3
:100D0800ADBE4ED70DBE75A10100030038B50C4627
:100D1800017A1546CA0702D500F014F908B908483F
:100D280032BDD0F8F80003682146DC682A46A0479F
:100D3800B0F5003F01D0034832BD4FF4403032BD1A
:100D480002000300010003002DE9F84191B00546B7
:100D58000E461746402101A813F0C2F8297AC807A1
:100D680004D5284600F0EEF8040002D1DFF8A4808C
:100D78004BE0D4F8F800DFF8A0800368D3F810C07F
:100D88006A4601A9E047B0F5003F3ED1D4F8F80023
:100D980001684A689047B0F5003F36D1D4F87C1115
:100DA8008A6820469047D4F8F830024618461B68EF
:100DB800D3F80CC004F1FC01E047B0F5003F24D1A2
:100DC800D4F87C0141688847D4F8F83002461846C0
:100DD8001B68D3F80CC001A9E047B0F5003F14D157
:100DE800D4F8F8000268696893689847B0F5003F3E
:100DF8000BD1D4F8F80003681C693A463146A0477D
:100E0800B0F5003F08BF4FF44038404612B0BDE887
:100E1800F08100BF02000300010003002DE9F84142
:100E2800A5B0074688461646402115A813F058F87D
:100E380000220492402105A813F052F8387AC1071D
:100E48005ED5384600F07EF8050059D0D5F8F80090
:100E58002D4C0368D3F810C06A4605A9E047B0F5E1
:100E6800003F3CD1D5F8F80001684A689047B0F5D2
:100E7800003F34D1D5F87C118A6828469047D5F8C8
:100E8800F830024618461B68D3F80CC005F1FC017F
:100E9800E047B0F5003F22D1D5F87C01416888478A
:100EA800D5F8F830024618461B68D3F80CC005A9D7
:100EB800E047B0F5003F12D1D5F8F800026879682C
:100EC80093689847B0F5003F09D1D5F8F800036852
:100ED8001D6904AA15A9A847B0F5003F01D020460E
:100EE8000FE00A4B0A490B4A0396029101924046C9
:100EF8001C68049B009415AA796800F0E5F900E0E5
:100F0800054826B0BDE8F08101000300B84001089B
:100F1800936E030026C703000200030004B001011A
:100F280000170145E10A0008010B0008250B00081D
:100F3800B50300084D0B0008150D0008510D0008F9
:100F4800250E00080168024A914218BF0020704728
:100F58002C0F000810B5040008BF002404D0034873
:100F68002060204609688847204610BD2C0F0008DD
:100F780020225C3012F0B2BFF0B58468A3080022CA
:100F880004F0030407E000F15C0555F8226035BA67
:100F980041F82250521C9A42F5D300220BE000F18E
:100FA8005C0502EB830755F82360D500C5F11805E9
:100FB800EE40CE55521CA242F1D3F0BD30B5C46804
:100FC80003690022E31AD5188C5C0544521C082AD0
:100FD8002C77F8D330BD0360C1600261704738B523
:100FE800044615460022626023685A68904700202C
:100FF8006061A061A5604FF4003032BD81604FF49C
:10100800003070472DE9F84304462079D4F80C8065
:10101800450748BF244845D466691D46A8F1010024
:1010280000EAD60306EBC506B6EBC50F666102D229
:10103800A669761CA6611746A66906EB5576A661D1
:101048000E46E918884225D2A8EB03094A463146DC
:10105800F81812F043FF2268136839460FE0424639
:10106800384612F03BFF23681A68394620469047F5
:1010780007E0311811F00300F1D122681368204607
:101088009847484600EB0809A9F10101A942F0D3A5
:10109800002300E000202A1A3118F81812F01EFF69
:1010A8004FF40030BDE8F283040002002DE9FC4F44
:1010B800024685B0D0681369DFF86CC1DFF86C812F
:1010C800A0EB030A506840F004005060002703A812
:1010D80002900DF10C0ED8E9003403A8544DC0E974
:1010E80000342878534D00280CBF00230423994668
:1010F8005CF803305EF80940234401261D601C6833
:101108009E60DCF80430039DDCF80090DEF8046093
:101118005D406540484C654089EA0606474C664094
:101128007519474C6540D8E9006B03AC0028C4E941
:10113800006B0EBF002404200424029E5CF800000B
:10114800345920183F4C04600126046886600398CF
:10115800029E43406340384C7068634089EA00004F
:10116800364C6040034438484340280018BF0120EB
:101178005B1E9B41042F2CBFC0B2D80F02F1140391
:1011880053F8200007F00303C3F10303DB00D84042
:101198000DF807007F1C082F9DD315460C466A6979
:1011A800AB69E868D20842EA4372401E00EA0207C7
:1011B800002302409B420AD8524508D28020E055BD
:1011C8007F1C574516D2AAEB0701E01910E08020D2
:1011D800E05500E0E355E8687F1C8742FAD32A68A7
:1011E800136828469847BAF1000F03D051462046A5
:1011F80012F076FE2A68069E059F9368694628467F
:1012080098472A68D2F8009021462846C8472B6894
:10121800DA683946284690470EB1A86830604FF41E
:10122800003007B0BDE8F08FB04001085412000844
:10123800D80800205FC5109304850012FC68017A65
:10124800C0F524FF24AF33D426AF698B04B0010165
:1012580000170145F8B501240094002300240DE08F
:10126800009D065D0F5D7E40F643761CF60F86F006
:10127800010635400095641C009DEB189442EFD39D
:101288001846F2BDF8B5002301240094002A11E0A5
:10129800009C85188F1815F8016C17F8015C6E40D2
:1012A800F643761CF60F86F0010634400094009C45
:1012B800E318521EECD11846F2BD00005D1200087A
:1012C8008D120008010000002DE9F84F1D46DDF8D9
:1012D80028900B9F0D9C4FF0FF3300930E469246CB
:1012E800D9F800B0804632465146D847834664B3A1
:1012F800D9F8043032465146404698476FEA0B0207
:10130800521C42EA0B0200996FEAD2735B1C194027
:10131800C2430091521C024300996FEAD2735B1CCE
:101328001940009186F05531484087EA000181F064
:101338005531216080F05531C943491C0843009A52
:101348006FEAD070401C82430092D9F80800012847
:1013580009D17540E943491C0D4300986FEAD572DD
:10136800521C90430AE0F11C85EA9102D243521CB8
:10137800154300986FEAD5735B1C984386F0AA362C
:10138800009086EA0B0686F0AA33F243DB430C98FA
:10139800C2F3C0725B1C42EAD3720099D243521C5A
:1013A80091430091774000998843009987F0AA37C4
:1013B8000F403843BDE8F28F034613F8012B002A8B
:1013C800FBD1181A0138704781F0004102E000BFD4
:1013D80083F0004330B54FEA41044FEA430594EAED
:1013E800050F08BF90EA020F1FBF54EA000C55EA28
:1013F800020C7FEA645C7FEA655C00F0E2804FEAF9
:101408005454D4EB5555B8BF6D420CDD2C4480EADA
:10141800020281EA030382EA000083EA010180EA0A
:10142800020281EA0303362D88BF30BD11F0004F58
:101438004FEA01314FF4801C4CEA113102D040428E
:1014480061EB410113F0004F4FEA03334CEA1333C9
:1014580002D0524263EB430394EA050F00F0A780E1
:10146800A4F10104D5F1200E0DDB02FA0EFC22FADC
:1014780005F2801841F1000103FA0EF2801843FAD0
:1014880005F359410EE0A5F120050EF1200E012AC1
:1014980003FA0EFC28BF4CF0020C43FA05F3C018FF
:1014A80051EBE37101F0004507D54FF0000EDCF178
:1014B800000C7EEB00006EEB0101B1F5801F1BD321
:1014C800B1F5001F0CD349085FEA30004FEA3C0C25
:1014D80004F101044FEA445212F5800F80F09A801B
:1014E800BCF1004F08BF5FEA500C50F1000041EB1F
:1014F800045141EA050130BD5FEA4C0C404141EB23
:101508000101013C28BFB1F5801FE9D291F0000F1D
:1015180004BF01460020B1FA81F308BF2033A3F1CC
:101528000B03B3F120020CDA0C3208DD02F1140CC3
:10153800C2F10C0201FA0CF021FA02F10CE002F1FE
:101548001402D8BFC2F1200C01FA02F120FA0CFCF7
:10155800DCBF41EA0C019040E41AA2BF01EB045140
:10156800294330BD6FEA04041F3C1CDA0C340EDC3E
:1015780004F11404C4F1200220FA04F001FA02F381
:1015880040EA030021FA04F345EA030130BDC4F13F
:101598000C04C4F1200220FA02F001FA04F340EA34
:1015A8000300294630BD21FA04F0294630BD94F0E5
:1015B800000F83F4801306BF81F480110134013DCC
:1015C8004EE77FEA645C18BF7FEA655C29D094EA3D
:1015D800050F08BF90EA020F05D054EA000C04BFBB
:1015E8001946104630BD91EA030F1EBF00210020A6
:1015F80030BD5FEA545C05D14000494128BF41F045
:10160800004130BD14F580043CBF01F5801130BDA8
:1016180001F0004545F0FE4141F470014FF0000033
:1016280030BD7FEA645C1ABF194610467FEA655CE4
:101638001CBF0B46024650EA013406BF52EA033586
:1016480091EA030F41F4002130BD00BF90F0000F74
:1016580004BF0021704730B54FF4806404F13204B0
:101668004FF000054FF0000150E700BF90F0000F69
:1016780004BF0021704730B54FF4806404F1320490
:1016880010F0004548BF40424FF000013EE700BF60
:1016980042004FEAE2014FEA31014FEA02701FBFF0
:1016A80012F07F4393F07F4F81F06051704732F022
:1016B8007F4208BF704793F07F4F04BF41F4002179
:1016C800704730B54FF4607401F0004521F00041D7
:1016D8001CE700BF50EA010208BF704730B54FF061
:1016E80000050AE050EA010208BF704730B511F062
:1016F800004502D5404261EB41014FF4806404F19A
:1017080032045FEA915C3FF4D8AE4FF003025FEA1F
:10171800DC0C18BF03325FEADC0C18BF033202EBA3
:10172800DC02C2F1200300FA03FC20FA02F001FAFD
:1017380003FE40EA0E0021FA02F11444BDE600BFA0
:101748004FF0FF3C06E000BF4FF0010C02E000BF85
:101758004FF0010C4DF804CD4FEA410C7FEA6C5C68
:101768004FEA430C18BF7FEA6C5C1BD001B050EA0B
:10177800410C0CBF52EA430C91EA030F02BF90EAF6
:10178800020F0020704710F1000F91EA030F58BFB5
:10179800994208BF90422CBFD8176FEAE37040F017
:1017A800010070474FEA410C7FEA6C5C02D150EAB5
:1017B800013C07D14FEA430C7FEA6C5CD6D152EA70
:1017C800033CD3D05DF8040B704700BF8446104635
:1017D80062468C461946634600E000BF01B5FFF734
:1017E800B7FF002848BF10F1000F01BD4DF808ED04
:1017F800FFF7F4FF0CBF012000205DF808FB00BFD5
:101808004DF808EDFFF7EAFF34BF012000205DF82E
:1018180008FB00BF4DF808EDFFF7E0FF94BF01207B
:1018280000205DF808FB00BF4DF808EDFFF7CEFF7C
:1018380094BF012000205DF808FB00BF4DF808EDBB
:10184800FFF7C4FF34BF012000205DF808FB00BF8C
:101858004FEA410212F5001215D211D56FF47873D0
:10186800B3EB625212D94FEAC12343F0004343EA73
:10187800505311F0004F23FA02F018BF404270474E
:101888004FF00000704750EA013005D111F00040D8
:1018980008BF6FF0004070474FF00000704700BF6E
:1018A80080F0004002E000BF81F0004142001FBF0D
:1018B8005FEA410392EA030F7FEA226C7FEA236C16
:1018C8006AD04FEA1262D2EB1363C1BFD21841400B
:1018D80048404140B8BF5B42192B88BF704710F0A1
:1018E800004F40F4000020F07F4018BF404211F044
:1018F800004F41F4000121F07F4118BF494292EAAC
:10190800030F3FD0A2F1010241FA03FC10EB0C00D7
:10191800C3F1200301FA03F100F0004302D5494264
:1019280060EB4000B0F5000F13D3B0F1807F06D311
:1019380040084FEA310102F10102FE2A51D2B1F109
:10194800004F40EBC25008BF20F0010040EA0300FE
:101958007047490040EB0000013A28BFB0F5000F7E
:10196800EDD2B0FA80FCACF1080CB2EB0C0200FA34
:101978000CF0AABF00EBC25052421843BCBFD04083
:101988001843704792F0000F81F4000106BF80F4FD
:1019980000000132013BB5E74FEA41037FEA226CC0
:1019A80018BF7FEA236C21D092EA030F04D092F08B
:1019B800000F08BF0846704790EA010F1CBF0020BF
:1019C800704712F07F4F04D1400028BF40F000401C
:1019D800704712F100723CBF00F50000704700F03C
:1019E800004343F0FE4040F4000070477FEA226263
:1019F80016BF08467FEA23630146420206BF5FEA34
:101A0800412390EA010F40F4800070474FF0000333
:101A180004E000BF10F0004348BF40425FEA000CFA
:101A280008BF704743F0964301464FF000001CE0A2
:101A380050EA010208BF70474FF000030AE000BFF8
:101A480050EA010208BF704711F0004302D5404236
:101A580061EB41015FEA010C02BF844601460020A8
:101A680043F0B64308BFA3F18053A3F50003BCFAC3
:101A78008CF2083AA3EBC25310DB01FA02FC634470
:101A880000FA02FCC2F12002BCF1004F20FA02F277
:101A980043EB020008BF20F00100704702F120026A
:101AA80001FA02FCC2F1200250EA4C0021FA02F2CB
:101AB80043EB020008BF20EADC7070474FEA40029F
:101AC800B2F1FE4F0FD34FF09E03B3EB12620DD964
:101AD8004FEA002343F0004310F0004F23FA02F0CE
:101AE80018BF404270474FF00000704712F1610F75
:101AF80001D1420205D110F0004008BF6FF000404C
:101B080070474FF00000704753B94AB9002908BF21
:101B180000281CBF4FF0FF314FF0FF3000F070B9C4
:101B2800ADF1080C6DE904CE00F006F8DDF804E02C
:101B3800DDE9022304B070472DE9F047089E0D4601
:101B480004460F46002B4AD18A42944665D9B2FA18
:101B580082F343B102FA03FCC3F120029F4020FA4A
:101B680002F217439C404FEA1C4E1FFA8CF5B7FB54
:101B7800FEF1220C0EFB117742EA074201FB05F049
:101B880090420AD91CEB020201F1FF3780F01B8159
:101B9800904240F2188102396244121AA4B2B2FB90
:101BA800FEF00EFB102244EA024400FB05F5A542B4
:101BB8000AD91CEB040400F1FF3280F00681A5422B
:101BC80040F203816444023840EA0140641B00216A
:101BD8001EB1DC400023C6E90043BDE8F0878B4214
:101BE80008D9002E00F0EC800021C6E9000508465F
:101BF800BDE8F087B3FA83F1002949D1AB4202D39B
:101C0800824200F2F780841A65EB0302012017462E
:101C1800002EE2D0C6E90047DFE702B9FFDEB2FADC
:101C280082F3002B40F08F808A1A4FEA1C471FFA74
:101C38008CFE0121B2FBF7F507FB1520220C42EAC6
:101C480000420EFB05F0904208D91CEB020205F198
:101C5800FF3802D2904200F2CA804546121AA4B256
:101C6800B2FBF7F007FB102244EA02440EFB00FE29
:101C7800A64508D91CEB040400F1FF3202D2A645A0
:101C880000F2BA801046A4EB0E0440EA05409FE734
:101C9800C1F120078B4022FA07FC4CEA030C05FA35
:101CA80001F420FA07F3FD40234300FA01F94FEA53
:101CB8001C401FFA8CFEB5FBF0F81C0C00FB1855F5
:101CC80044EA054408FB0EF5A54202FA01F20BD9D5
:101CD8001CEB040408F1FF3A80F08780A54240F22B
:101CE8008480A8F102086444641B9DB2B4FBF0F33D
:101CF80000FB134445EA044403FB0EFEA64508D93D
:101D08001CEB040403F1FF306BD2A64569D9023BF2
:101D1800644443EA0840A0FB0283A4EB0E049C42FF
:101D2800C6461D4655D352D056B1B9EB0E0364EBE7
:101D3800050404FA07F7CB40CC401F43C6E90074FA
:101D48000021BDE8F087C3F1200102FA03FC20FA64
:101D580001F225FA01F19D402A434FEA1C471FFA78
:101D68008CFEB1FBF7F007FB1015110C41EA054199
:101D780000FB0EF58D4204FA03F408D91CEB0101AF
:101D880000F1FF382FD28D422DD902386144491B0A
:101D980092B2B1FBF7F507FB151142EA014205FBC8
:101DA8000EF1914208D91CEB020205F1FF3816D258
:101DB800914214D9023D6244521A45EA004139E77A
:101DC8003146304609E73946E7E61046FCE6C145A4
:101DD800AAD2B8EB020E63EB0C050138A4E745461E
:101DE800EAE7034695E74046D1E7D0467CE7023D5F
:101DF800624433E708460BE76444023843E700BF10
:101E0800704700BF1348144A08B54FF00043C0E9B3
:101E180000230422002342610122C2614FF4805151
:101E280007220383C0E90233C0E90933C0E90C1271
:101E38000361837680F8203080F82C30826380F844
:101E48003C30C36404F09EFF18B1BDE8084000F0C0
:101E580025BC08BDDC080020002401400268084BAE
:101E68009A4282B00AD14FF0B0431A6E42F400721F
:101E78001A661B6E03F400730193019B02B070474E
:101E8800002401400268054B9A4201BF4FF0B0425E
:101E9800136E23F400731366704700BF00240140DB
:101EA80030B585B000240546CDE901440394FFF719
:101EB800A9FF144805F0FEFA08B100F0EFFB11483D
:101EC800039401A9CDE9015405F0BAF808B100F06E
:101ED800E5FB0C4805F018FA08B100F0DFFB4FF0FD
:101EE800FF31084805F04EF8064805F0C5FA0548E0
:101EF80005F0A2F80446034805F068FA204605B044
:101F080030BD00BFDC080020014B024A1A60704750
:101F1800DC0800200024014008B50948FFF7C0FF8D
:101F280068B1084BB3F8AA304FF6FF72934216BF58
:101F380040F6E442044B5343B3FBF0F398B208BDB8
:101F4800002000B40075FF1FD8084C0013B500230B
:101F5800ADF80630FFF7E0FF04461948FFF7A0FF89
:101F6800184BB3F8C820B3F8A8108A4204FB00F055
:101F780018D040F6E443B0FBF3F364205B1A434304
:101F8800521A93FBF2F31E331BB2ADF80630BDF8BC
:101F980006305BB21B02ADF80630BDF8060000B291
:101FA80002B010BD4FF47A7240F6FF73B0FBF3F342
:101FB8005343A3F53923A3F50C6340F6C412E0E7B5
:101FC800001000B00075FF1F4FF0B04382B09A6A4E
:101FD80022F480529A629A6C42F480529A649B6C02
:101FE80003F480530193019B002002B070474FF027
:101FF800B04382B09A6C02439A649B6C034001938D
:10200800019B02B0704708B50420FFF7F0FF0120DC
:10201800FFF7EDFF0220FFF7EAFF002211460B2031
:1020280005F0E6FA0B2005F015FB002211460C20FE
:1020380005F0DEFA0C2005F00DFB002211460D20FC
:1020480005F0D6FA0D2005F005FB002211460E20FA
:1020580005F0CEFA0E2005F0FDFA002211460F20F9
:1020680005F0C6FA0F2005F0F5FA002211461120F6
:1020780005F0BEFA112005F0EDFA002236201146CF
:1020880005F0B6FABDE80840362005F0E3BA0000CE
:1020980008B505F027FD10B16FF0040008BD064B28
:1020A8009A6942F040429A614CF2FA321A6105F09C
:1020B8002BFD0028F2D0EFE700400058F0B585B0BE
:1020C80000230C4600930646A8B3FFF7E1FF054638
:1020D80070BB05F007FD88BB1A481B4A0223019311
:1020E800D0F8E01506F1784302EA8121B3FBF1F755
:1020F80001FB1733DB0A0293D0F8E00504F17841BD
:102108000139314402EA8022B1FBF2F002FB1011DE
:10211800C3EBD1230133694601A8039305F074FD8D
:1021280020B102280CBF01256FF0010505F0ECFC79
:10213800284605B0F0BD6FF00505F9E76FF0040516
:10214800F6E700BF0070FF1F00FCFF03014B18609B
:1021580000207047400900202DE9F04F89B0B0F108
:10216800006F06460F460092C0F0C580DFF89881E0
:10217800664DD8F8E03505EA832303F10063013B97
:10218800984200F2B880002800F0B880002900F0DA
:10219800B58040EA02035B0740F0B080FFF778FFA4
:1021A8000446A0BB05F09EFC002840F0AA80D8F8A1
:1021B800E01506F1784205EA8121B2FBF1F301FB53
:1021C8001322009B03F17843013B3344B3FBF1F046
:1021D80001FB1033DB0A01334FEAD22AA3EBD222E8
:1021E800012A039388BFC6F30A050AF58038C6F1A9
:1021F800080398BF009D069388BFC5F500654FEAA0
:10220800C828B346039B9A4505D305F07DFC2046B4
:1022180009B0BDE8F08FA6F10803069A1A44954262
:1022280019D804950197CDF814B04FF00009059B13
:1022380009EB0301049B99453ED3009BAB442F4413
:102248005D1BB5F5006F28BF4FF400650AF1010A60
:1022580008F50068D6E753F8081F5A68B2F1FF3F3F
:1022680008BFB1F1FF3FD8D0294B186810B96FF0FB
:102278000504CAE7B8F1000F04D04FF400624146E4
:1022880011F0C0F9DFF88890D9F80030CBF30A00D4
:1022980039461844AAB211F0B5F94FF40061404626
:1022A800FFF70CFF08BBD9F8003001934FF4006327
:1022B800CDF814800493B8E7019B07914B4402932F
:1022C8000120D3E9002305F059FC88B90799019B3F
:1022D800D1E9000259F80310029B5B689A4208BFD3
:1022E800884205D109F10809A1E76FF001048CE7DC
:1022F8006FF0030489E74FF0FF3488E76FF00504B7
:1023080085E76FF0040482E70070FF1F00FCFF03FD
:1023180040090020B1F1006F70B511D30B4BD3F811
:10232800E0650B4B03EA862303F10063013B994206
:1023380006D840B139B192B211F064F9002070BDED
:102348004FF0FF30FBE76FF00500F8E70070FF1F64
:1023580000FCFF03B0F1006F10B40DD3084BD3F8A5
:10236800E045084B03EA842303F10063013B9842EC
:1023780002D810BCFFF7A2BE4FF0FF3010BC704768
:102388000070FF1F00FCFF034FF0B04382B0DA6C0F
:102398000243DA64DB6C03400193019B02B070478F
:1023A8002DE9F04186B01422002101A811F062FD48
:1023B80001203B4EFFF7E8FF0220FFF7E5FF04206E
:1023C800FFF7E2FF08210122304605F091FD0125C3
:1023D8004FF40417022301A94FF09040CDE90137CB
:1023E800039505F05FFC4FF4441301A94FF09040AA
:1023F8000024CDE902354FF02008019505F052FC84
:1024080001A93046CDE90187039405F04BFC01A9E9
:102418003046CDE90187039405F044FC082301A95F
:102428003046CDE90135CDE9035405F03BFC4FF4C6
:10243800007301A94FF09040CDE90135CDE903546F
:1024480005F030FC04230DEB03013046CDE90135DE
:10245800CDE9034405F026FC22462146062005F076
:10246800C7F8062005F0F6F822462146072005F0B1
:10247800BFF8072005F0EEF822462146162005F0A1
:10248800B7F8162005F0E6F822462146162005F092
:10249800AFF8162005F0DEF806B0BDE8F08100BF01
:1024A8000004004808B51248124A134BC0E900233B
:1024B80000230122C0E90232C0E90433C0E906332F
:1024C800036205F089FE08B100F0E8F80848002129
:1024D80006F002F808B100F0E1F80548002106F01E
:1024E80021F818B1BDE8084000F0D8B808BD00BF11
:1024F800040A0020005800405D3E302070B596B0B8
:1025080005461422002103A811F0B4FC382200214A
:1025180008A811F0AFFC2A68304B9A425BD180239F
:10252800089308A84FF440230E9306F057FD08B10E
:1025380000F0B4F84FF0B0444FF4C050E36C43F0EF
:102548000103E364E36C03F001030293029B12238B
:102558000026CDE903030323CDE905634FF090403E
:10256800042303A9079305F09DFBA36DDFF870C052
:1025780043F48003A365A36D1A4C03F4800301930D
:10258800019B26620D23C4E900C320468023C4E9C9
:102598000266C4E90436C4E9066605F0BBF808B16A
:1025A80000F07CF8104AEC63A562104C0E23C4E9D5
:1025B80000231021002380222046C4E90213C4E925
:1025C8000423C4E90633236205F0A4F808B100F037
:1025D80065F8AC63A56216B070BD00BF0058004036
:1025E800440002404409002058000240A409002089
:1025F80000B59BB04822002108A811F03BFC182226
:10260800002102A811F036FC05F0B2FF4FF0B042ED
:102618000120D2F8903023F01803C2F89030D2F895
:10262800003423F4C06343F40073C2F80034D2F8D2
:10263800003403F4C0630193019B2423089381238E
:102648000B930023CDE91003B02208A8CDE912238B
:1026580006F006F908B172B6FEE74F23CDE902305D
:10266800CDE90400CDE90600022102A806F092FB9C
:1026780008B172B6FEE71BB05DF804FB08B504F0BC
:102688002FFBFFF7B5FFFFF78BFEFFF7BCFCFFF74B
:1026980009FF00F094FD00F099FDFCE772B6FEE733
:1026A80000B58DB02C22002101A811F0E3FB1748DA
:1026B800174B03601F2383604FF080420023C0E95B
:1026C8000433C0E9072383614FF48073436206F043
:1026D8000BFE08B1FFF7E2FF0C4806F031FF08B126
:1026E800FFF7DCFF4FF000530022079307480892DA
:1026F8004FF4807301A9029206920B9306F054FEE0
:1027080008B1FFF7CBFF0DB05DF804FB580A0020B5
:102718000028004010B5044690B03822002102A8D5
:1027280011F0A8FB2268194B9A422CD14FF4803340
:10273800029302A84FF480730F9306F04FFC08B180
:10274800FFF7ACFF4FF0B0430220D3F8902042F4DB
:102758000042C3F890209A6D42F480629A659B6D9E
:10276800002203F4806311460193019B04F040FFAB
:10277800022004F06FFF00222A20114604F038FFDF
:102788002A2004F067FF10B010BD00BF00280040E9
:102798007047000008B504F0B9FA044B0120C3F8EB
:1027A8008800BDE8084005F03BBF00BF00040058A2
:1027B80004F0B3BA08B504F0B0FA00F033FCFFF740
:1027C800EFFDFFF720FCBDE80840FFF76BBE08B53A
:1027D80004F09CFABDE808400121002005F0D0BEB5
:1027E80070477047FEE7FEE7FEE7FEE7FEE7704743
:1027F8007047704770470000014806F0C7BE00BF29
:10280800580A0020012005F079BB022005F076BBAC
:1028180070477047014805F0F7B800BF4409002029
:10282800014805F0F1B800BFD00A00207047FFF753
:10283800F7BF7047202005F061BB7047014807F0DB
:1028480069BA00BF300B0020014806F0D1BC00BFB8
:10285800580A0020014807F0C4B800BFBC0A00208D
:102868002DE9F04389B080460020109E07908946E4
:1028780015461F46FDF7D4FCF0B9104CCDE9009081
:10288800CDE9020407AB0E480593142304933A4696
:10289800434629460068FDF78DFD2346324604F17C
:1028A800140153F8044B42F8044B8B42F9D1079BAF
:1028B800337509B0BDE8F0830120FAE7900A0020DB
:1028C800AC4001081FB50E4C00233C2202A8CDE9FC
:1028D80002336275237500F0B9F8042303AA009443
:1028E80012210848FFF7BCFF07491422204611F0BF
:1028F800B1FAB0FA80F35B09637504B010BD00BF8C
:10290800A40A0020D4400108DE0D0020054808B5BF
:102918000823036006F080FE18B1BDE80840FFF701
:10292800BDBE08BDBC0A00204FF0B04307B55A6EC3
:1029380042F001025A665B6E002203F00103019324
:1029480011463220019B04F053FE322003B05DF89B
:1029580004EB04F07FBE00000CB407B5054A05ABD4
:102968001021019311F058F903B05DF804EB02B09F
:10297800704700BFE640010830B585B0044602A89C
:102988000D4610F075FFBDF90C30064A0093102172
:10299800029B2046FFF7E0FF2046FEF70DFD28804A
:1029A80005B030BDE64001084FF0B04210B593685D
:1029B80023F40043936010F0E3FF0E4B01241C70D6
:1029C80000F0B6F810F0ACFC0B4810F0C3FC0B4B51
:1029D8004FF400421A61002010F0C2FCFFF794FA8D
:1029E80000F012F910F0B8FD21462046BDE810406D
:1029F80010F0D2BDC80A0020812900080040005804
:102A080010F0E0BD08B5FFF787FA40F6B8339842F2
:102A18000CD8B0F5E16F0BD3FE23A0F5E160584365
:102A28004FF49663B0FBF3F0C0B208BDFE20FCE79C
:102A38000020FAE77FB5684600F0CAF80198FFF76A
:102A48003DF800B207B05DF804FB0000194A38B53C
:102A5800D2F88035591C044619D104F065F90546A9
:102A680004F06EF9054404F065F92B0EE3712B0CA4
:102A7800A3712B0A6371030EE370C0F30742C0F31E
:102A880007232571C0B2A2706370207038BD190A7F
:102A9800C3718171190C1B0E41710371D2F8843511
:102AA800C370D2F88405C0F30722C0F30743000EB1
:102AB800E9E700BF0070FF1F38B5094BD3F8803530
:102AC80003600133054609D104F02EF9044604F0E9
:102AD80031F9444004F034F944402C6038BD00BF5B
:102AE8000070FF1F0121022010F040BD00210220CC
:102AF80010F03CBD00207047024B187808B100F078
:102B0800BBB87047C80A002082B00190019802B093
:102B180000F04EB94FF0B04382B0DA6C42F00202D6
:102B2800DA64DB6C03F002030193019B02B0704787
:102B38002DE9F043254C87B004F008F904F00EF9AC
:102B480004F014F90123002502934FF4805903235C
:102B580001A9204604934FF4005803950595FFF703
:102B6800D9FFFFF7D7FFFFF7D5FFFFF7D3FFCDF862
:102B7800049005F097F801A920464FF40067CDF8B6
:102B8800048005F08FF801A920464FF4004601970C
:102B980005F088F801A92046019605F083F82A4631
:102BA8004946204605F0A4F92A464146204605F044
:102BB8009FF92A463946204605F09AF92A463146B1
:102BC800204605F095F907B0BDE8F08300040048F9
:102BD80010B50446FFF7BAF9074BA36040F30F207E
:102BE800FEF718FF054B064A2360064B6060C4E9F0
:102BF8000323002010BD00BF0000484200007A44B3
:102C08000D093E00AB03050000207047014B186812
:102C1800704700BFCC0A00200320704708B5014662
:102C28004FF47A7200238002890DFEF76DFF08BD0C
:102C38004FF47A73A0FB0303800A40EA835070477D
:102C4800034B98689A689042FBD1C043704700BF15
:102C58000028004008B5FFF7F3FF014B186008BDD6
:102C6800CC0A002008B5FFF7EBFF024B1B68C01A1F
:102C780008BD00BFCC0A0020024B187808B1FFF746
:102C8800DFBF7047C90A002010B5074B074C012267
:102C9800DA654FF48071204606F070FA4FF0FF3382
:102CA8002363002010BD00BF00280040580A002000
:102CB80002460021014806F07ABC00BF580A0020ED
:102CC80002460121014806F072BC00BF580A0020E4
:102CD80010B58CB02C220021044601A811F0CAF8C6
:102CE800FFF7D2FF0C4B0D481B681C4400230893C8
:102CF80006934FF00053E443079301224FF4807387
:102D080001A902940B9306F04FFB08B1FFF7C6FC2C
:102D180000200CB010BD00BFCC0A0020580A0020CB
:102D280038B50546FFF78CFF02210446074806F030
:102D380045FCC4F309024FF47A71A2FB0121920AFF
:102D4800A30A2A8043EA805038BD00BF580A0020F1
:102D58000148002106F032BC580A00200148012130
:102D680006F02CBC580A0020F8B50F4D2E78CEB9C5
:102D78000E4C4FF0FF372763FFF792FCFFF784FFF5
:102D88004FF48071204606F0F9F92046276306F0D3
:102D9800B9FB32462046022106F009FCFFF75AFF2C
:102DA80001232B700020F8BDC90A0020580A002012
:102DB800014610B54FF47A7200238002890DFEF7A0
:102DC800A3FE0146FFF73CFF0446FFF739FF031B4C
:102DD8008B4200D310BD00BFF7E710F0D9BE00004A
:102DE80010B5064C0221204606F0E8FB0221421CE1
:102DF8002046BDE8104006F0DABB00BF580A0020A4
:102E08001648174A08B54FF4E133C0E900230023F8
:102E18000C22C0E90233C0E90523C0E90733C0E941
:102E28000933036107F057FD08B1FFF737FC0B487A
:102E3800002107F0CCFE08B1FFF730FC074800215D
:102E480007F0E5FE08B1FFF729FC044807F09FFEEC
:102E580018B1BDE80840FFF721BC08BD300B0020C1
:102E68000044004070B596B006461422002103A81D
:102E780011F000F83822002108A810F0FBFF326892
:102E8800274B9A424AD10223089308A8254B0A9354
:102E980006F0A4F808B1FFF701FC4FF0B043002595
:102EA8009A6D214C42F400329A659A6D02F4003210
:102EB8000292029ADA6C42F00102DA64DB6C03F0E7
:102EC80001030193019B0C220223CDE90323032371
:102ED800CDE9055303A907234FF09040079304F069
:102EE800E1FE124925621423C4E900131023C4E942
:102EF800023520468023C4E90435C4E9065504F0A8
:102F080009FC08B1FFF7CAFB2520F467002202215B
:102F1800A66204F06DFB252004F09CFB16B070BD82
:102F28000044004004000C00D00A00208000024049
:102F380002680C4B9A4210B5044612D14FF0B042C9
:102F48000C21936D23F4003393654FF0904004F007
:102F580055FFE06F04F052FCBDE81040252004F056
:102F680087BB10BD0044004008B50A460146024828
:102F780006F034FE002008BD300B002013B5114BBD
:102F8800114C18604FF40013009302AB13E90600CC
:102F9800204607F0A0FD2368DA69D103FCD4DA697A
:102FA8005202FCD59A68084842F480029A6007F0F9
:102FB800D8FD06490448012207F046FD002002B06A
:102FC80010BD00BFC40B0020300B0020CC0B00202C
:102FD80008B5074B1860FFF716F8FFF711FF054A09
:102FE800D2F8803043F00063C2F88030002008BD7A
:102FF800C80B00200008005808B54FF0B043084837
:103008009A6B42F400329A639A6B22F400329A6304
:10301800FFF78EFF0F2004F02BFB002008BD00BF38
:10302800300B002008B5074807F055FC08B1FFF73A
:1030380035FB054804F06EFB18B1BDE80840FFF702
:103048002DBB08BD300B0020D00A00200268044BBD
:103058009A4203D1034B00201B681847704700BFF2
:1030680000440040C80B002002680B4B9A4210B580
:1030780004460FD1094B1B682BB1D0F8902012B928
:1030880007480121984720460549BDE8104001221C
:1030980007F0DABC10BD00BF00440040C40B00209C
:1030A800CC0B002002480122102104F021BF00BFF0
:1030B8000004004802480022102104F019BF00BF94
:1030C8000004004810B50A4C23780BB9E37C6BB1B7
:1030D800FFF7F8FB0038074B18BF012040001870B5
:1030E8001B78022B02BF00232370E37410BD00BFBE
:1030F800DE0D0020D40B002038B5114C2378F3B92D
:10310800E37CE3B90F4D2B68012B07D92B68042BFF
:1031180004D80D4A0421012000F01AFA2B68042B68
:103128000DD9FFF7CFFB0038084B18BF012040002E
:1031380018701B78022B02BF00232370E37438BD7C
:10314800DE0D0020D00B002040410108D40B0020E8
:1031580008B5FFF7A7FF01F01FFABDE80840FFF721
:10316800A9BF022801D8FFF79DBF7047022801D8E0
:10317800FFF7A0BF70470000022808B51BD801223E
:1031880010210D4804F0B4FE3220FFF7BDFC0A48B8
:103198000022102104F0ACFE01221021064804F0A0
:1031A800A7FE3220FFF7B0FCBDE808400248002225
:1031B800102104F09DBE08BD00040048704708B502
:1031C800FFF7F2FBBDE8084000F060BB4FF0FF30AE
:1031D80010F05CBA7047704770470000014BD87018
:1031E800704700BF5C000020014B1874704700BF97
:1031F8005C00002020B1037813B1024810F076BCBF
:10320800704700BF140D002008B50220002110F0FF
:1032180005FABDE80840014810F068BC2C0D0020F4
:103228000021012010F0FAB910B5094C60B12060F6
:10323800084810F00DFC2168064810F091FCBDE824
:103248001040044810F052BC42F210732360EFE7BC
:10325800740000202C0D002010B5094C2060236854
:103268000BB9084B2360084810F0F2FB21680648A8
:1032780010F076FCBDE81040034810F037BC00BFE2
:103288000C000020A0860100440D002010B5044663
:1032980080B190F906306BB9094810F0D9FB094B99
:1032A800E2791A70084B1868FFF7D6FF074B1868C1
:1032B800FFF7BAFFBDE810400021022010F0AEB9B8
:1032C800C80C0020F80C00200C000020740000201E
:1032D80038B504460D4607484FF40061FFF73AF841
:1032E80030B92A4621460348BDE83840FEF734BFC6
:1032F80038BD00BF00F003080A460149FFF70AB8C5
:1033080000F0030838B50C4810F0A2FB08F0E4F808
:1033180060B90A4C0A480125257007F06FFF20782C
:10332800294607F0C1FC044810F0E0FBBDE838402E
:10333800044810F0DBBB00BF2C0D0020000000206B
:103348005C000020FC0C002008F062B930B585B0A4
:10335800FFF758FB044607F09DFD054680B10024A1
:103368003C4810F075FB3C4B3A481968A14238BFFD
:10337800214610F0F5FB374810F0B8FB05B030BD1A
:1033880001464FF4807010F049F9684600F0E6FFF6
:1033980023B203EB4303FE2203EB4313B3FBF2F325
:1033A8002E4A392111702E4950680978DBB28DF800
:1033B8000C3001705068457050682724847050683C
:1033C8000124C47050680371264B187840B11D70F1
:1033D800536861F07F0119703A23137005231CE0CC
:1033E800214B2248197811B901780029F6D000211B
:1033F80001701970536804215971BDF80030516883
:10340800180A88715168CB71BDF8083051681B0AD9
:103418000B72BDF808304B720A231549154C097810
:10342800012988BF00235370637A33B107F01EFD6A
:10343800012802D1204610F00BFB0F4B0748D97822
:10344800002207F03DFD063089D107F009FD04464A
:1034580086E700BF2C0D0020740000200400002027
:10346800C70C00205C0D0020F30D0020DD0D0020AE
:10347800D40B0020C80C00205C00002008B5104BBD
:103488000122002102201A7010F0C8F80D4810F02F
:103498002DFB0D4B1B788BB10C4B1A7872B9DB7C6A
:1034A80063B90B4B1A68042A9EBF1A6801321A6066
:1034B8000021BDE80840102010F0B0B808BD00BFDA
:1034C8005C0D0020440D0020F80C0020DE0D0020CB
:1034D800D00B0020044B1B78022B03D100210820BD
:1034E80010F09CB8704700BF0000002008B507F036
:1034F800FCFF80B907F0BAFC01280CD1BFF34F8F4D
:103508000549064BCA6802F4E0621343CB60BFF377
:103518004F8F00BFFDE708BD00ED00E00400FA058D
:103528007047704770477047022807D0202808D096
:10353800012809D10021022010F070B800210820CC
:10354800FAE7024B01221A70704700BF580E00209C
:1035580070B505460C46164607F09CFC0346002845
:1035680034D000241A4810F073FA1A4B1848196816
:10357800A14238BF214610F0F3FABDE87040144864
:1035880010F0B4BA4A68F05CD0540133DAB294420D
:10359800F8D8114B0D701B78012B88BF00244C7094
:1035A8000E4C637A33B107F061FC012802D1204642
:1035B80010F04EFA0A4B0B48D978002207F080FC2D
:1035C8000630CED107F04CFC0446CBE70549DDE7D1
:1035D8002C0D002074000020D40B0020C80C002003
:1035E8005C00002004000020044B1B7823B9044A27
:1035F80005210120FFF7ACBF704700BFD40B0020A6
:103608004541010810B5002490B03C22214601A88C
:10361800009410F02FFC2F4B2022DA7219788DF8C5
:10362800001059788DF8011099788DF80210D97822
:103638008DF8031019798DF8041059798DF8051053
:1036480099798DF80610D9798DF80710197A8DF8BF
:103658000810597A8DF80910997A8DF80A108DF8A2
:103668000B2021460DF10B0258180131007B02F89E
:10367800010F1C29F8D193F828208DF8282093F8F9
:1036880029208DF8292093F82A208DF82A2093F8EC
:103698002B208DF82B2093F82C206AB193F83F202B
:1036A80052B10DF12B0100229818013290F82C002C
:1036B80001F8010F142AF7D107484FF40061FEF70B
:1036C80049FE20B9044840226946FEF745FD10B07E
:1036D80010BD00BF7800002000F80308014940220F
:1036E8000FF090BF00F8030870B52A4D28796B7960
:1036F8004D2BC0B233D1C0EB001080000A2838BF70
:103708000A204FF47A735843234BAC791860EB794D
:103718004D2BE4B22BD1C4EB0414A40095F82C3043
:103728001E4E63BB95F83F304BBB42F21070FFF75B
:103738007BFD3068FFF790FD2B7A194A1949DBB2F7
:1037480013706B7A184ADBB213700023EA1892F8E8
:103758002C20D2B2CA540133142BF7D170BD6B7927
:10376800482B0ABF4FF461636B795843C6E7EB797E
:10377800482B0ABF4FF46163EB795C43CEE7FFF750
:1037880053FD012C38BF01244FF47A735C43346035
:10379800CFE700BF78000020740000200C00002054
:1037A800F20D0020DE0D0020D40B002010B590B0E3
:1037B80000213C2201A8009110F05CFB4022314915
:1037C80068460FF01FFF9DF800203AB99DF80100E8
:1037D800272803D19DF80210012909D0FFF712FF0D
:1037E8004FF47A70FFF790F9FFF77EFF10B010BD25
:1037F800254B1A70587099709DF80310D9709DF870
:10380800041019719DF8051059719DF806109971E9
:103818009DF80710D9719DF8081019729DF80910C4
:1038280059729DF80A1099729DF80B1001F03F012A
:10383800D972D87AD1B288421BD89DF8282083F84B
:1038480028209DF8292083F829209DF82A2083F82C
:103858002A209DF82B2083F82B200DF12B01002224
:103868009818013211F8014F80F82C40142AF7D12A
:10387800BAE701F140006844194410F8340C0873A1
:103888000132D6E700F80308780000201FB50024AD
:1038980003A92046039407F00BFE03A9012007F0B3
:1038A80007FE384B3848009422464FF4FA7110F05E
:1038B80071F8364B3648009422464FF4FA7110F0EE
:1038C80069F8344B3448009401224FF4FA7110F02F
:1038D80061F82046FEF73AFC08B1FEF7DFFE2F4BF1
:1038E800009400224FF4FA612D4810F053F82D4A45
:1038F800002101200FF04EFF2B4A002102200FF07B
:1039080049FF2A4A002104200FF044FF284A0021D9
:1039180008200FF03FFF00F09DFB2649264807F0DE
:103928007DFD264807F06AFC1B4810F0DFF8244BA1
:103938000021187807F0B8F922490094224B096849
:103948002248002210F026F8204810F0CFF8FFF7A0
:103958002DFF1F4A002110200FF01CFF1D4A0021D7
:103968004FF480700FF016FF1B4B1C4819681C4B56
:103978000094002210F00EF8184810F0B7F804B0C0
:1039880010BD00BF2D350008140D00202F3500088C
:10399800E00C002029350008C80C0020DD340008A0
:1039A800FC0C0020FDAF0008553300085133000817
:1039B8000D33000800000301100000205C00002007
:1039C8000000002074000020113200082C0D002097
:1039D80001310008593100080C000020440D002076
:1039E8008534000810B50024A2B07C22214603A823
:1039F800029410F03FFA53238DF8083040F2271351
:103A0800ADF80A3001238DF80C30ADF80440FEF70C
:103A1800F9FF00B200EB400000EB4010FE23B0FBC2
:103A2800F3F08DF80D0001A800F0A8FCA0B9582308
:103A38008DF80E30072430228021144810F01AFA2D
:103A4800224602A9114810F04EFA104A21460120D8
:103A5800FFF77EFD22B010BD430001338DF80E3014
:103A68008DF80F0000F098FD094B1A6812128DF8B6
:103A780010201A688DF811205A685B688DF8133089
:103A880012128DF812200C24D5E700BF5D0D00201E
:103A9800840E002030B50378592B91B0044640F0CD
:103AA800F281052959D84378443B162B55D8DFE8CD
:103AB80013F031015400210154002901540054002D
:103AC80054005400940054000C0154005400540055
:103AD800990154005400B0005400540054001700D9
:103AE8008578482D11D1B64A14210120FFF730FD01
:103AF80041F28830FFF708F840F6B830FFF704F8CD
:103B080011B0BDE83040FFF7F1BC532D0ED1302283
:103B18008021AC4810F0AEF9FFF764FF41F288301D
:103B2800FEF7F2FFA74A1521012086E0432D16D1A2
:103B3800002468468DF8004007F0D8FAA14A4C23C3
:103B48001370272393709DF800305470012041337F
:103B5800D07013710521FFF7FBFC11B030BD442D67
:103B6800FBD1984C592323705A236370A57000F039
:103B7800E7FB2C228021201D10F07CF90023257002
:103B8800637001252723A370E5702571FEF73AFFBE
:103B98008D49FE23B0FBF3F00B6864229BB2B3FBA4
:103BA800F2F3A3710B6800EB400000EB40109BB2EE
:103BB8006071B3FBF2F002FB1033E3714B689BB208
:103BC800B3FBF2F323724B689BB2B3FBF2F102FB37
:103BD8001133637222460A21A6E78378303BDBB2B1
:103BE800092BBAD879497A4A0B700B78DBB2537231
:103BF800744A592313704D2353700B7830339370E4
:103C080003210120FFF7A4FC11B0BDE83040FFF705
:103C1800F9BC8578482D15D16A4A562313700023BC
:103C28005370272393700323182101201371937174
:103C380007235171D070D371082111B0BDE830400D
:103C4800FFF786BC432D88D15E4C00213C2201A899
:103C5800009110F00FF96846FFF740FD24228021FB
:103C680004F10C0010F006F99DF8003063709DF81F
:103C78000130A3709DF80230E3709DF80330237182
:103C88009DF8043063719DF80530A3719DF80630E6
:103C9800E3719DF8073023729DF808302570637230
:103CA8009DF80B509DF80930A3729DF80A30E37215
:103CB8002A4603A9257304F10D0010F014F905F143
:103CC8000D012246C9B2012045E7807839280CD871
:103CD8003038C0B2FFF745FA3A4A23781370637850
:103CE8005370A378937003211EE711B0BDE83040EC
:103CF800FFF77ABC80783928F7D83038C0B2FFF798
:103D080035FAE9E780783928EFD83038C0B2FFF7BC
:103D180033FAE1E78378303BDAB2092AE5D8C0788C
:103D28003038C2B2092AE0D82179A1F14802D2B2CA
:103D38000B2ADAD8274D45FA02F2D507D5D40A223C
:103D48004D2902FB030036D13C2358434FF47A73C4
:103D58005843214B1860214B1860FFF765FA194A40
:103D68002378137063785370A3789370E378D370D3
:103D78002379137105210120FFF7EAFB144B002278
:103D88001A7027225A7001229A70DA70A278303A93
:103D980002EB8201E278303A02EB4102D2B21A71A8
:103DA80022795A710E4A1278D2B21A72074A1278D8
:103DB800D2B25A7228E74829C8D14FF46163C4E7E0
:103DC8004B4101085D0D0020840E0020D40B00201B
:103DD80078000020DEF7FFFF740000200C000020B0
:103DE800F20D00208278303AD3B2092B3FF67DAF2E
:103DF800C378303BD9B209293FF677AF0079A0F1F3
:103E08004801C9B20B293FF670AF624D45FA01F17E
:103E1800C9073FF56AAF0A214D2801FB02332DD1AE
:103E28003C2253434FF47A7253435B4A1360106841
:103E3800FFF712FA594A2378137063785370A378FE
:103E48009370E378D3702379137105210120FFF76C
:103E58007FFB534B00221A7027225A7001229A7056
:103E6800DA70A278303A02EB8201E278303A02EB5B
:103E78004102D2B29A712279DA7193E74828D1D1F6
:103E88004FF46162CDE7502B48D102297FF665AE29
:103E98004378303B012B3FF660AE8378312B7FF4BB
:103EA8005CAE0B2904D8FFF79FFB00213B4A3BE699
:103EB8003B4D0234002214F8013FA918303B01326F
:103EC800DBB20C2A0B73F6D1FFF778F9334B50228B
:103ED80027211A709970002201215A70D97003F8AD
:103EE800041FA9180132097B0C2A01F1300103F8DB
:103EF800011FF6D100232B7027236B700123AB70B1
:103F0800EB70284B1B78DBB22B72274B1B78DBB28C
:103F18006B72EA72FFF776FB1121C7E7412B7FF43A
:103F28001CAE4378432B7FF418AE16297FF415AEE8
:103F38001E4D421C002312F8011FE9540133142BB3
:103F4800F9D1FFF7BFF81A4B5B7D012B19D1144942
:103F58000023EA5CC8180133D2B2142B80F82C2055
:103F6800F7D1114B00221A701B78DBB24B72FFF7A6
:103F780049FB0A4A631E1534A34206D1074A162193
:103F8800D2E5094B02221A70F3E713F8011F02F871
:103F9800011BF1E7DEF7FFFF0C0000205D0D00209C
:103FA80078000020F20D0020D40B0020DE0D002048
:103FB800A40A002037B504460D46002939D0224806
:103FC8000FF094FD2B78A3B39CB36068237880B37B
:103FD800032B0DD0392B2ED0022B2AD16178012941
:103FE80027D00B0625D403B0BDE83040FFF752BDFB
:103FF8006378012B07D10078012802D0022800D06D
:1040080008B907F029F800240DF107008DF80740DA
:1040180007F06CF80D4A4C231370272393709DF812
:104028000730547001204133D07013710521FFF718
:104038008FFA03B030BD6378012BFAD10378044AB4
:1040480003F001031370F4E7E00C00205D0D00207D
:10405800C70C0020034B0022C3E902220122C3E956
:1040680000227047F40D002000487047F40D00202E
:104078004FF0B04382B0DA6C0243DA64DB6C034081
:104088000193019B02B070472DE9F04186B00024EE
:104098000220154D0594FFF7EBFF0420FFF7E8FF1A
:1040A800124F03944FF4807601230DEB0001CDE904
:1040B80001632846032304934FF4005803F0F2FDEC
:1040C80001A93846CDF8048003F0ECFD22464146AC
:1040D800384603F00DFF28462246314603F008FF14
:1040E800204606B0BDE8F0810004004800080048FA
:1040F800032810B50ED8012810D868B902460B4815
:104108004FF4807103F0F4FE002209484FF4005187
:1041180003F0EEFE002010BD0122F0E70022034864
:104128004FF4807103F0E4FE0122EEE7000400483A
:10413800000800480220704700207047012070479F
:1041480000280CBF0F201620704700000D48854638
:1041580002F0C4FD0C480D490D4A002302E0D45872
:10416800C4500433C4188C42F9D30A4A0A4C0023B9
:1041780001E013600432A242FBD30FF083FEFEF786
:104188007DFAFEE70000012000000020BC080020A6
:10419800784C0108BC0800205C2C0020FEE74FF09A
:1041A800B04382B0DA6C42F00102DA64DB6C03F0EF
:1041B80001030193019B02B07047000030B587B03E
:1041C800FFF7EDFF4FF4805101224FF0904003F0CC
:1041D8008FFE01224FF400614FF0904003F088FEFB
:1041E8004FF4C0551123CDE9015301A901234FF024
:1041F8009040039303F056FD08240A2500224FF44B
:1042080080514FF0904003F073FE0120FEF77CFCD4
:1042180001224FF480514FF0904003F069FE0120D5
:10422800FEF772FC013DE9D14FF400614FF0904078
:1042380003F058FE08B9013CDFD14FF400614FF09C
:10424800904003F04FFE68BBFFF7A9FF0424012349
:10425800039001A92A48CDE9014303F023FD284C26
:1042680001220421204603F043FE2120FEF74CFCE6
:1042780000220421204603F03BFE2120FEF744FCE7
:1042880001220421204603F033FE2120FEF73CFCE6
:1042980020460022042103F02BFE4FF42570FEF780
:1042A80033FCDDE7FFF77BFF4FF0B04300249A6D46
:1042B80042F480029A659B6D03F4800300934FF4E7
:1042C800C052009B1223CDE901230323CDE9034308
:1042D80004230DEB03014FF09040059303F0E2FC3B
:1042E80008480949094B8460C0E900130123C0E963
:1042F8000334C0E90744446103F06EFF07B030BDE2
:1043080000040048040E0020005800401A0910203C
:10431800FFF754BF10B1012809D0704701394A424C
:104328004A414FF090404FF4007103F0E1BD4B1E3D
:104338005A4202485A410821F7E700BF00040048E2
:1043480008B50120FEF70DFF6420FEF7DDFB00F045
:1043580023F9BDE808400120FEF708BF054B1A689D
:1043680002805A689B684381034B028101221A70BC
:10437800704700BF840E0020DD0D002010B50446F4
:1043880000F008F810F0FF001CBFEE232370AA23EA
:10439800637010BD2DE9F3470024304E304D346072
:1043A80021462046FFF7B6FF21460120FFF7B2FF5E
:1043B80021460220FFF7AEFF2A4F4FF05208A146D0
:1043C800012195F8640185F86081C5F86891FFF7C7
:1043D800A1FF0320FEF798FB00228821284602F05F
:1043E800E3FB0DF10602C021284602F02BFC80BB3E
:1043F800BDF806204EF6AA639A422AD14FEA440A2B
:104408000AF1540A5FFA8AFA5146284600F032F94E
:10441800F8B90DF10602C021284685F860A102F01E
:1044280011FCB0B9284600F0E9FA90B932680123C6
:104438001A4432603A68C5F86831A34013433B60B8
:104448000134032C05F5C875BAD1306802B0BDE84F
:10445800F0870021E0B2FFF75DFFF1E77C0E002056
:10446800BC000020780E00202DE9F74F354C83461C
:1044780004F5966A4FF00A094FF00E0848F2E8076B
:104488004FF490164FF48045D4F86821002A51D093
:10449800204600F0A7FD0DF102020DF101012046B2
:1044A80000F05AFB0DF1030201A9204600F09FFE1F
:1044B8000021204600F0E2F801220021204600F009
:1044C800A1F901221146204600F09CF9BBF1020F28
:1044D8000ED81D4B1D4A33F81B501D4B12F80B808C
:1044E80053F82B601B4A1C4B12F80B9053F82B7097
:1044F8002A460121204600F0D0F932460021204604
:1045080000F0CBF93946204600F0D2F842460021A7
:10451800204600F0CFF84A460121204600F0CAF8AC
:104528000DF102020DF10101204600F015FB0122F8
:10453800C4F87C2104F5C8745445A5D103B0BDE87E
:10454800F08F00BFBC0000206041010880410108D5
:1045580068410108834101087441010810B50B7EC8
:104568009BB9D0F87C21098912B1C0E95E1310BD4E
:10457800084BD0F878411A68C2F580734B4304FBA6
:1045880002331B12C0F87831F1E70123C0F87C31FF
:10459800EDE700BFB80000202DE9F84FDFF8BCA018
:1045A8002F4DFFF7B5FEDAF800300BB12B6813B9C1
:1045B800FFF7F0FE28602B682A4E0024A3423460DF
:1045C8007460B46044DDDFF8A080284DDFF8A0B047
:1045D8000220FFF749FF88F80040D5F86831012B21
:1045E8002CD103FA04F90A272149284600F05AFC7D
:1045F800B0B959462846FFF7B1FF9BF818307BB988
:10460800D5F8783146F82430DAF8003043EA09035F
:10461800CAF8003098F8003043F0010388F80030F9
:104628000120FEF771FA9BF818309BB1013F17F093
:10463800FF07D9D14FF47A7346F8243001200134AA
:10464800FEF762FA032C05F5C875C6D198F8003054
:10465800BDE8F88FD5F87831EEE700BF780E002076
:10466800800E0020840E0020DD0D0020BC000020FC
:104678005C0E00204A088A2102F096BA152906D84D
:10468800044BCB40DB0702D50174002070476FF064
:10469800070070470B00300010B50A460C46092188
:1046A80002F0A4FA18B9237803F00103237010BDAF
:1046B80001F06BBE01F053BD01F04DBEF7B500230C
:1046C8000C46174601210DF1070206468DF8073002
:1046D80002F08CFA0546D8B9012F9DF8073026D18B
:1046E800042C3AD8DFE804F003171A1D200043F021
:1046F8001004A3420CD022460121304602F054FA9D
:10470800054628B9716986F830413046FFF7D0FF71
:10471800284603B0F0BD43F02804EAE743F0040458
:10472800E7E743F04004E4E743F08004E1E7042CC2
:1047380013D8DFE804F00306090C0F0003F0EF04B8
:10474800D7E703F0D704D4E703F0FB04D1E703F07D
:10475800BF04CEE703F07F04CBE76FF00305D7E78C
:1047680013B500230C460DF1070201218DF807301F
:1047780002F03CFA78B99DF80730C3F300122270B2
:10478800C3F3C002A270C3F380026270C3F3801245
:10479800DB09E270237102B010BD37B50D460DF18B
:1047A8000202F821044602F04DFA70B901AA042168
:1047B800204602F067FA40B9BDF802201AB1019B01
:1047C800B3FBF2F32B602B68A36103B030BD037F0A
:1047D8000B700020704737B50D460DF106022021F9
:1047E800044602F02FFA28B9BDF8063023B9236A27
:1047F8002B60207703B030BDDB002B6023620123E0
:104808002377F7E70529F8B504460E46154635D847
:1048180062B100EB810301215A6B0023701E04284A
:1048280007D8DFE800F00E171A1D240011460123EF
:10483800F4E784F828103444E5B984F828500020B7
:1048480007E0C2F34F224421204602F0BDF90028B8
:10485800F1D0F8BD84F82A10EDE784F82B10EAE7C8
:104868005B00FE226021204602F0D5F9EFE71B012C
:10487800EF22F7E7012384F82830E0E76FF0030020
:10488800E7E7052996BF4018002390F828301370F1
:1048980094BF00206FF00300704770B543180446BA
:1048A80093F828000E46154618B904EB8106726382
:1048B80070BD05291BD8DFE801F00309121416168C
:1048C800626304EB860400206563F1E7C2F34F22BC
:1048D8004421204602F078F90028E9D1F1E7E263A3
:1048E800EFE72264EDE7C2F34F226421F1E76FF0AE
:1048F8000300DDE737B50446154605292CD8DFE85F
:1049080001F0030717191B1B436B2B60002021E0E4
:104918000DF10602442102F095F9D8B9BDF8062038
:1049280053029AB12B60A363012384F8293011E064
:10493800C36BEAE7036CE8E70DF10602642102F0B5
:1049480081F938B9BDF806305B02DEE7A36B2B604E
:1049580084F8290003B030BD6FF00300FAE737B5DB
:104968000D460DF107020121044602F03FF938B95E
:104978009DF8073084F83031DB092B7084F84C300F
:1049880003B030BD2DE9F843037C0C4601F8083B21
:104998000546FFF702FF40BB207304F110012846CB
:1049A800FFF719FF08BB04F11401284600F021FCA9
:1049B800D8B904F1240705F1270904F117080646B8
:1049C8003A46B1B22846FFF795FF70B9013619F893
:1049D800013F08F8013F062E07F10407F0D104F162
:1049E8003C012846FFF7BBFF08B1BDE8F883211D4D
:1049F8002846BDE8F84301F030BD0000F0B50022BC
:104A0800054693B0882102F0CFF84FF47A72A5F8E2
:104A180052214FF4C872A5F854214C4AC5F85821C0
:104A280000234B4A85F8F030C5F8D4202B6202A940
:104A38002846FFF7A7FF044670B9ADF8080002AE94
:104A48000FCE05F110070FC70FCE0FC70FCE0FC738
:104A580096E80F0087E80F003E4BC5F834314FF455
:104A6800FA730126A5F838314FF42063A5F83C31D4
:104A78003246802185F85061284602F095F8324682
:104A88000746FF21284602F08FF800221146074307
:104A9800284602F089F83C4364B204430DF107024A
:104AA8009121284602F0A2F864B29DF8073085F8F3
:104AB8003A31044332460021284602F075F864B2C0
:104AC80004430022FF21284602F06EF864B2044332
:104AD80000228021284602F067F864B2204340B2E1
:104AE800002488BBA1B2012228460134FFF78AFEC0
:104AF800062CF6D140BB04466885024604212846A8
:104B0800FFF780FE00BB024605212846FFF77AFE24
:104B1800D0B94FF490136B634FF4804201212846BB
:104B2800FFF7BBFE80B94FF40C13FF22C5E90F3025
:104B380085F830210121284602F036F8012385F84E
:104B4800323108B985F8154113B0F0BD856B010005
:104B5800A470090064008403012300F079BD2DE9E5
:104B6800F0428EB00C460C2304AA1421054602F02C
:104B780005F8844600286CD19DF81A309DF81B6012
:104B88009DF817209DF81810A07506EB03269DF8D0
:104B98001630206002EB03229DF81930606003EBA9
:104BA80001239BB25B029DF8121023619DF813301C
:104BB800B5F8520103EB012392B252029BB2E260B4
:104BC800A382B0F57A7F9DF8101095F83171B6B2CE
:104BD8000AD0704300F5FA704FF47A76B0FBF6F01D
:104BE8002E7F002E39D186B2002F40D0B001C0B23E
:104BF800B608E0750DF10F002681CDE90040284682
:104C080001F086FE844620BB9DF80FE084F818E08A
:104C180005F150060FCE07AF0FC796E80700E37DF2
:104C280087E80700D4E90301A28AADF83020D4E967
:104C38000149CDE90A01CDE9084907AC8DF83330BF
:104C48008DF834E00FCC50350FC597E8070086E89B
:104C5800070060460EB0BDE8F0822E8C5E43B2EBD2
:104C6800262F4FEA262C04D157B948F6E026002013
:104C7800BFE780B25043A2EB0C06B0FBF6F0B2E7F8
:104C880042F2B826B2E70000F7B517460E210DF13B
:104C980006021D460B4C064601F0D4FFBDF806304F
:104CA80004EA43433B6050B90DF106020C2130463B
:104CB80001F0C8FFBDF8063004EA43442C6003B095
:104CC800F0BD00BF0000FE1F73B590F8DA30013B5D
:104CD800022B06460C4634D801AB6A460121FFF781
:104CE800D3FF009BB3F57F0F054603D8019BB3F5AF
:104CF8007F0F23D915BB34B11349304602B0BDE844
:104D0800704001F00FBC0422FF21304601F04CFF37
:104D18002A4604467021304601F046FF2A460443DD
:104D2800FF21304601F040FF64B204432A46802147
:104D3800304601F039FF64B2044365B2284602B038
:104D480070BD0025FAE700BF5F06002037B50446AE
:104D580001228021057C01F027FF0122FF21204646
:104D680001F022FF00221146204601F01DFF94F8B1
:104D78003A219121204601F017FF01220021204607
:104D880001F012FF0022FF21204601F00DFF002252
:104D98008021204601F008FF012D29D0032D37D0AE
:104DA800002D3CD101222946204601F0FDFE0123B9
:104DB8008DF80730A0B103B030BD01460DF10702F0
:104DC800204601F013FF9DF80730DB0705F10105C8
:104DD80008D538B9B5F5FA6FEFD16FF00600EAE7F4
:104DE8000546F0E7B5F5FA6F08BF6FF00600E2E791
:104DF80018B929462046FFF767FF022200212046FE
:104E080001F0D2FE0028D6D1042384F83231D2E74B
:104E180018B901212046FFF757FF0422EEE76FF08B
:104E28000700C8E738B5057C044625B1204600F0E0
:104E380054FD28B138BDFFF789FF0028F6D0F9E7FF
:104E4800002DF7D1032384F83231F3E773B5064612
:104E5800002501220B21304601F0A6FE002204465F
:104E68000B21304601F0A0FE0DF107020443132187
:104E7800304601F0BBFE9DF8073064B204430135AB
:104E88005B0760B2EDB205D0032D08D00028E0D052
:104E980002B070BD032D08BF6FF00B00F8E76FF08C
:104EA8000B00F5E738B50023037404460D46FFF7F9
:104EB800B9FF50B929462046FFF751FE28B90146E7
:104EC8002046BDE83840FFF7C1BF38BD152970B589
:104ED800054616461C4667D10122FF2101F064FEF3
:104EE800002211460446284601F05EFE00220443D3
:104EF800FF21284601F058FE64B2044301228021B4
:104F0800284601F051FE64B2044302228521284656
:104F180001F04AFE64B204430422FF21284601F04E
:104F280043FE64B204430022CD21284601F03CFE32
:104F380064B204431122CC21284601F035FE64B244
:104F480004430722FF21284601F02EFE64B20443E1
:104F58000022BE21284601F027FE64B2044306223F
:104F6800FF21284601F020FE64B204430922CC2127
:104F7800284601F019FE64B204430022FF212846A6
:104F880001F012FE64B204430122FF21284601F019
:104F98000BFE64B2002204431146284601F004FEC9
:104FA80064B2204340B270BD042A17D80A2101F028
:104FB800FBFD0028F7D1231E18BF01231B01EF2298
:104FC8008421284601F027FE0028ECD185F8DA6014
:104FD80001462846BDE87040FFF738BF6FF00A0069
:104FE800E1E7000070B594B005464022002104A80E
:104FF8000EF040FF002301212846ADF806308DF859
:1050080003308DF80430029300F0B8FC95F81421B1
:1050180095F81311012A04D840F0AD80202940F2F8
:10502800AC8001AA02A9284600F02DFB04460028FE
:1050380040F09E8095F85031002B40F0A280D5F8C2
:105048004C11284601F06EFA0446002840F0908082
:105058002346214604222846FFF738FF0446002845
:1050680040F086800122FF21284601F09DFD0DF1C8
:10507800060206468421284601F0E4FD224606433E
:10508800FF21284601F090FD76B2064374B2002C49
:105098006ED1BDF806301B01C5F8D43004A92846E6
:1050A800FFF770FC0446002862D10DF10301284681
:1050B800FFF7F2FA044600285AD19DF8033085F824
:1050C800313104AE0FCE05F110040FC40FCE0FC45A
:1050D8000FCE0FC496E80F0084E80F000DF103020D
:1050E8000121284601F082FD0446002840D19DF8A0
:1050F800033085F83031024601462846FFF7DEFACC
:105108000446A8BB024602212846FFF7D7FA044600
:1051180070BB0323014685F832310DF1050228469C
:1051280001F019F9044618BB9DF8053085F8E830F8
:105138000DF105020121284601F00DF90446B8B920
:105148009DF8053085F8E03003AA0321284600F0D1
:1051580001FF044660B9039BC5F8E43003AA0421A3
:10516800284600F0F7FE044610B9039BC5F8DC306A
:10517800204614B070BD0C2951E7284600F010F9FC
:1051880054E701495DE700BF6C05002013B50C46E4
:105198000DF10702132101F029FD9DF8073013F0E6
:1051A800180F03F0070218BF6FF00500226002B065
:1051B80010BD13B590F8DA30042B0C460BD101A9B9
:1051C800FFF7E4FF019B042B01D1012300E000233A
:1051D800237002B010BD01AA142101F007FD0028B8
:1051E800F7D19DF80430DB07EFD42070F1E700F029
:1051F8004ABA13B50C460DF10602282101F022FD2A
:1052080078B9BDF80620C2F30B0312F4006F18BF7B
:10521800A3F580534FF0FA0214BF13FB02F3534374
:10522800236002B010BDF0B54FEAD20C4FF0FF3446
:105238001C6002F00702664600278E4200D207B1C2
:10524800F0BD845D664503BF1441E4B215463D4692
:1052580014F0010704D005EBC6051D600136ECE724
:105268000135082D4FEA5404F2D1F7E7034B8009C2
:1052780053F82000003818BF012070471808002094
:1052880010B5B1EBD20F4FEAD20402F0070381BF89
:1052980001229A40035D13438ABF03556FF0310022
:1052A800002010BD0A460623B02101F049BC0A4679
:1052B8000623B02101F062BC2DE9F04F85B080468D
:1052C800109E0E9D01968A4693461C464FF0000993
:1052D800119B994508D10023129A1660F3B16FF01B
:1052E800310005B0BDE8F08F01AB3246294658467B
:1052F800FFF799FF019F7B1C0DD00F9BF818FFF754
:10530800B5FF504507D13A462046FFF7B9FF7E1C46
:1053180009F10109DCE76FF03103DDE7214640467A
:10532800FFF7C0FF0028DCD102A94046FFF7BFFF06
:105338002544234602AAAB42D3D013F8014B12F8F6
:10534800011B8C42F7D0CAE770B5C02288B00E4660
:10535800012190F83041054601F026FCF0B901A979
:105368002846FFF79FFDC8B90122FF21284601F012
:105378001BFC98B93246B621284601F063FC68B98F
:105388000246FF21284601F00FFC38B922460121C8
:10539800284601F009FC08B985F8304108B070BD0D
:1053A800F0B50F4689B01646FF210122044601F0E8
:1053B800FBFB0246A8B94F21204601F0F5FB80B956
:1053C8002C224E21204601F0EFFB024648B9FF216E
:1053D800204601F0E9FB20B9B422B621204601F0AD
:1053E800E3FB0025C4F82451A4F82851DEB935465A
:1053F80007ABB422CDE903730623CDE90032029549
:1054080004F5927304F5957231462046FFF754FF70
:1054180030B9012384F8153184F8137184F81461C4
:1054280009B0F0BD013505F1B400FFF71FFF0028F2
:10543800DED12C2DF6D1DBE710B541F001020021B9
:10544800044601F0B1FB78B9204600F046FA58B995
:1054580001462046FFF7FAFC30B9024601462046CD
:10546800BDE8104001F0A0BB10BD2DE9F74F4FF08B
:10547800000B88461746FF21012205461E469DF867
:1054880038A09DF83C908DF807B001F08DFB5A4686
:1054980004465946284601F087FB5A460443FF2133
:1054A800284601F081FB64B2044364B2B8F1000FEE
:1054B80032D0BAF1000F06D00C9ACB21284601F061
:1054C80095FB204344B2B9F1000F07D00DF1070254
:1054D800EE21284601F08AFB204344B20122FF2135
:1054E800284601F061FB012204430021284601F00F
:1054F8005BFB64B204430022FF21284601F054FB01
:1055080064B29DF807300D9A204323F0100340B28F
:10551800137003B0BDE8F08FBAF1000F06D03A4619
:10552800CB21284601F040FB204344B2B9F1000FDB
:10553800D4D033468022EE21284601F06CFBCBE71D
:105548002DE9F04387B091460022054688468DF83C
:1055580017201E461BB390F83071012211462846C9
:1055680001F022FB044658BB40212846FFF764FFA0
:10557800044628BBB9F1010F13D10DF11703CDE98A
:105588000290CDE900830246034649462846FFF7C4
:105598006CFF40B10446204607B0BDE8F0831F46C3
:1055A800DBE788F80000002EF5D03A4601212846AE
:1055B80001F0FAFA04460028EDD185F83071EAE7DF
:1055C800002388F800302046E4E72DE9F04305463B
:1055D80087B0884691461E4623B390F83071022260
:1055E8000121284601F0E0FA044660BB014628463E
:1055F800FFF722FF044630BBB9F1010F14D10DF1BA
:105608001703CDE90209009302460346CDF804804A
:1056180049462846FFF729FF40B10446204607B00F
:10562800BDE8F0831F46DAE788F80000002EF5D0C1
:105638003A460121284601F0B7FA04460028EDD180
:1056480085F83071EAE7002388F800302046E4E75F
:10565800F8B51D46164600232A4690F830710446D0
:10566800FFF76EFF70B903462A4631462046FFF71A
:10567800ACFF38B93A460121204601F095FA08B93D
:1056880084F83071F8BD2DE9F04F002393B0CDE9CF
:105698000A12C0F82431A0F828310122FF21CDE9EF
:1056A8000E33B0F83C818DF8343005468DF835302E
:1056B80001F07AFA0446002840F0E38002464F21C0
:1056C800284601F071FA0446002840F0DA802C22BE
:1056D8004E21284601F068FA0446002840F0D1809F
:1056E8000246FF21284601F05FFA0446002840F0F0
:1056F800C880B422B621284601F056FA044600288C
:1057080040F0BF8002468021284601F04DFA044649
:10571800002840F0B68003460DF135020DA9284651
:10572800FFF796FF0446002840F0AB800323CDE93D
:105738000203B421062305F5957A05F592790EAE94
:10574800CDE90031049601464B4652462846FFF7FC
:10575800B3FD0446002840F094800DF13601284638
:105768000E9FFFF7F1FD0446002840F08A80BDF83F
:105778003630434540F2AA80C5F82401A5F828012F
:1057880007F1B400FFF772FD08B92B2F7DD9062366
:10579800B4224FF0030BCDE90032CDE9027B049629
:1057A8004B46524601212846FFF786FD002840F067
:1057B8008B800DF1360128460E9FFFF7C5FD064682
:1057C80000287CD1BDF83630434540F2828001265E
:1057D8000696BDF83630434560D2A3EB080383EA4A
:1057E800E372A2EBE3729DF81860099205F59273D3
:1057F8004FF0030B0793079B18689B881090ADF830
:1058080044303A460FAB06215046FFF70CFD0F9F78
:105818007B1C56D007F1B400FFF728FD069B984281
:105828003CD10BF101033A4648460893FFF728FD9F
:10583800002849D149462846FFF734FD002843D1BE
:105848000DF136012846FFF77FFD00283CD1BDF851
:105858003620A2EB0803002BB8BF5B42424516D99D
:10586800099A934218D910A92846FFF71BFD079AF1
:105878000799034610981060BDF844208A806BB1E0
:105888001C46204613B0BDE8F08F013778E7DDF8F5
:1058980020B009930137AEE7DDF820B00A9BC3F8C2
:1058A80000B00B9B1E70012385F815310A9B1B68FD
:1058B80085F813310B9B1B7885F81431E1E7044612
:1058C800DFE76FF03104DCE70446DAE70026B34689
:1058D8007EE70123834606937BE737B5002304461A
:1058E8008DF807304FF4FA650DF107012046FFF7F0
:1058F80060FC58B99DF80730012B07D0013D03D053
:10590800204601F0E5F9EFE76FF0060003B030BD7F
:1059180002464FF08043934202D8002013B97047E3
:105928009B08F8E7C11891424FEA50009CBFC01885
:10593800521A9B08F2E773B500228321054601F04D
:1059480033F9044688B94FF4FA660DF1070283214A
:10595800284601F04BF99DF807300343DBB20446B3
:105968001BB9013EF1D16FF00604012283212846BC
:1059780001F01AF9204340B202B070BD2DE9F04F92
:1059880090F8F06091B04FF00009072ECDE9079923
:1059980004460F4600F0A2820122802101F004F99A
:1059A80001228046FF21204601F0FEF84A4648EAD7
:1059B80000084946204601F0F7F84FFA88F848EA07
:1059C80000080622FF21204601F0EEF84FFA88F879
:1059D80048EA00080DF115028321204601F006F976
:1059E8009DF815204FFA88F848EA000842F00402AA
:1059F8008321204601F0D8F84FFA88F848EA0008D1
:105A08000722FF21204601F0CFF84FFA88F801223B
:105A1800812148EA0008204601F0C6F84FFA88F8C4
:105A280048EA0008204601F053F94FFA88F848EA96
:105A3800000801228021204601F0B6F84FFA88F8C4
:105A480048EA000517F0010B6DB200F01E82F2075C
:105A580000F11E826B229421204601F0A5F88046B1
:105A68002046FFF768FF06AA48EA0008902120466A
:105A780001F008F945EA0805069B6DB22422942135
:105A880005432046C3F3062AC3F3C03901F08CF856
:105A98006DB205432046FFF74EFF6DB2054306AAD7
:105AA8009021204601F0EEF8069B6DB21BBA252224
:105AB800942105432046099301F076F86DB2054319
:105AC8002046FFF738FF6DB2054306AA902120460D
:105AD80001F0D8F8069B6DB21A0E05431B0C6DB287
:105AE8008DF828208DF8293017F00203029300F072
:105AF800DB8016F0020840F0D7800222942120466D
:105B080001F052F801902046FFF715FF019B0DF1B7
:105B180016020343902120461D4301F067F86DB239
:105B28007B2294210543204601F03EF86DB20543DF
:105B38002046FFF700FF6DB205430DF117029021D3
:105B4800204601F053F86DB2772294210543204690
:105B580001F02AF86DB205432046FFF7ECFE6DB25E
:105B6800054306AA9021204601F08CF8069B5A0EA0
:105B78008DF82C20C3F386428DF82D20C3F3C6225E
:105B88008DF82E206DB2C3F30612DB0003F0780304
:105B9800942105438DF82F20204678228DF8153062
:105BA80001F002F86DB205432046FFF7C4FE6DB25E
:105BB800054306AA9021204601F064F8069B9DF84B
:105BC800152002EB53728DF83020C3F386528DF8FE
:105BD8003120C3F3C6328DF83220C3F306228DF884
:105BE80033206DB2C3F346029B0103F040039421B6
:105BF80005438DF83420204679228DF8153000F0C1
:105C0800D3FF6DB205432046FFF795FE6DB20543FD
:105C180006AA9021204601F035F8069B9DF815202C
:105C280002EB93628DF83520C3F3C6428DF8362017
:105C3800C3F306328DF837206DB2C3F346129B00CA
:105C480003F07C03942105438DF8382020467A22FE
:105C58008DF8153000F0A8FF6DB205432046FFF718
:105C68006AFE6DB2054306AA9021204601F00AF8A3
:105C7800069B9DF815208DF83E8002EB93728DF8F7
:105C88003920C3F3C6526DB28DF83A20C3F30642E9
:105C980005438DF83B20C3F34622C3F386036DB258
:105CA8008DF83C208DF83D3017F00403019300F087
:105CB800F180730700F1EE807B229421204600F0EA
:105CC80073FF80462046FFF736FE07AA48EA000819
:105CD8009021204600F0D6FF45EA08084FFA88F8D8
:105CE80048EA00057C229421204600F05DFF6DB251
:105CF80005432046FFF71FFE6DB2054308AA902111
:105D0800204600F0BFFF6DB2732294210543204660
:105D180000F04AFF6DB205432046FFF70CFE6DB256
:105D2800054306AA9021204600F0ACFF069B6DB201
:105D38001B0274229421054320461FFA83F800F0C1
:105D480033FF6DB205432046FFF7F5FD6DB20543FD
:105D580006AA9021204600F095FF6DB29DF81B30F1
:105D6800752294210543204643EA080800F01CFFE9
:105D78006DB205432046FFF7DEFD6DB2054306AA66
:105D88009021204600F07EFF069B6DB21B029BB25D
:105D98007622942105432046039300F005FF6DB257
:105DA80005432046FFF7C7FD6DB2054306AA9021BB
:105DB800204600F067FF6DB29DF81B20039B05434A
:105DC8006DB21343002281212046039300F0ECFEBC
:105DD80006220543FF21204600F0E6FE6DB205438A
:105DE8000DF115028321204600F000FF9DF81520D3
:105DF8006DB2054302F0FB028321204600F0D4FE79
:105E08006DB205430122FF21204600F0CDFE6DB2A0
:105E1800054301220021204600F0C6FE6DB205436D
:105E28000022FF21204600F0BFFE6DB2054300228C
:105E38008021204600F0B8FE6DB205436DB2039B89
:105E4800FDB9BBF1000F29D1029AAABB019AAAB1E8
:105E5800720713D4079AC4F81821089AC4F81C21A9
:105E68004FEA4822C4F820213BB1A3F5C8534FF4A8
:105E78007A7253431B095B421BB2E3603E4384F8CA
:105E8800F060284611B0BDE8F08FD946DA462BE617
:105E9800CA4629E64FF00008434693E7F007D3D4F3
:105EA8000998BDF8282084F813A184F81491C4F83F
:105EB8002A01A4F82E21C7E7B107C7D49DF81620F8
:105EC80084F8F1209DF8172084F8F2200BA904F13A
:105ED800F30002930DF0FAFF029BB7E74D46D0E7B7
:105EE80050B10138002330F0FF019AB203F10103E9
:105EF80003D100EB022080B270474008F3E7C3B239
:105F0800000A03FA00F0013070470000084B5A43BA
:105F18004FF47A7302F5FA724FF4FA60B2FBF0F0BC
:105F2800B2FBF3F203FB0100B0FBF2F0704700BFD5
:105F3800002F3A00064B5A434FF47A7002F5FA7272
:105F4800B2FBF0F24A4302F5FA72B2FBF0F0704786
:105F5800002F3A002DE9FF4102294FF000050746BE
:105F680016468DF80350ADF804501CD80DF1020206
:105F78002946FEF7A1FB044630B90DF1030246217C
:105F8800384600F033FE04469DF80300FFF7B7FFDC
:105F980081B29DF802203846FFF7CCFF30602046DA
:105FA80004B0BDE8F081032918D10DF10202294699
:105FB800FEF782FB0446002846D101460DF1020295
:105FC8003846FEF779FB044628B901AA512138461C
:105FD80000F038FE0446BDF80400D7E7042935D19F
:105FE80002A9FEF7BDFB9DF80B30ABB10DF1020223
:105FF80029463846FEF760FB044658B901AA5121E4
:10600800384600F01FFE0446BDF80400FFF777FF8E
:1060180085B214B1002015E01D460DF102020121E0
:106028003846FEF749FB04460028F3D10DF1060275
:106038007121384600F006FE0446BDF80600FFF759
:106048005EFF80B2401BA3E72846A7E728462C46F8
:10605800A4E7F0B5022985B0054616461ED80DF10D
:1060680005020021FEF728FB0446A0B99DF805208B
:1060780031462846FFF74AFF83B2B3F5807F9ABFBF
:1060880000F1FF32D2B2FF22A5F8D82046212846D7
:1060980000F08AFD0446204605B0F0BD03291FD153
:1060A8000DF105020021FEF707FB9DF8052031469A
:1060B80004462846FFF72AFF80B2FFF711FF024681
:1060C800ADF80600A5F8D800002CE4D151212846E7
:1060D80000F07AFD04460028DDD1C5F8E460DAE76F
:1060E800042939D102A9FEF73BFB9DF80B70B7B123
:1060F8000DF1050200212846FEF7DEFA04460028C5
:10610800C9D10DF106025121284600F09BFD044635
:10611800BDF80600FFF7F3FE87B2002CBBD10DF1E6
:10612800050201212846FEF7C7FA04460028B2D125
:106138009DF8052031462846FFF7E8FE3844FFF76A
:10614800CFFE71210246284600F03EFD0446002895
:10615800A1D1C5F8DC609EE76FF003049BE7F0B5BA
:1061680085B000238DF80330D30705460F46164641
:1061780005D439B9A2F10C03DAB2062A11D96FF0A5
:106188000300E6E0012921D1A2F10803DAB2062AC8
:10619800F5D8062B1AD8DFE803F03B1969198A19D4
:1061A8009D00062B12D8DFE803F004112D112F11E2
:1061B800310018225721284600F0F6FC0822562103
:1061C800284600F0F1FC002840F0C3807408013C28
:1061D800E4B2002F00F09180012FD0D101AA042150
:1061E8002846FFF7B7FE50B922467021284600F02E
:1061F800DBFC20B9019A04212846FFF72AFF85F81D
:10620800E06099E03022D5E74022D3E75022D1E779
:106218001022482100F0C8FC08224721284600F037
:10622800C3FC022204463221284600F0BDFC0C22A1
:1062380004433021284600F0B7FC64B2044301222D
:10624800FF21284600F0B0FC64B2044364B2302257
:106258003021284600F0A8FC00220443FF212846EC
:1062680000F0A2FC64B2204340B2ACE728224821E7
:1062780000F09AFC08224721284600F095FC0322EA
:1062880004463221284600F08FFC044364B20922F8
:106298003021284600F088FC01220443FF212846CB
:1062A80000F082FC64B2044364B22022D0E73822B2
:1062B800482100F079FC08224721284600F074FCA8
:1062C800032204463221284600F06EFC044364B2DF
:1062D8000822DDE74822114600F066FC0822472123
:1062E800284600F061FC032204463221284600F0CB
:1062F8005BFC044364B20722CAE702AA03212846CA
:10630800FFF728FEB0B903AA02212846FFF722FEAC
:1063180080B922465021284600F046FC50B9029A1E
:1063280003212846FFF795FE20B9039A0221284643
:10633800FFF78FFE85F8E86058B969692846FEF7C7
:10634800B7F930B9024601230DF103012846FFF7DA
:106358003CF905B0F0BD13B5144629B1012910D098
:106368006FF0030002B010BD0DF10702502100F0DC
:106378003DFC0028F6D19DF8073001335B002370FF
:10638800F0E70DF107027021F1E7F0B5002385B0C1
:106398004FF4FA62CDE9002344F61F63994206469A
:1063A8000F4604D86FF00305284605B0F0BD02A9D2
:1063B800FEF7D6F905460028F6D19DF809209DF884
:1063C800083013439DF80A201343A7F636341BD030
:1063D8006A4602213046FFF7BDFD00283BD19DF8F3
:1063E80008302BB1009B03F24E239C42DAD9E41A01
:1063F8009DF80A3023B3009B03F2B223B4EB430F9A
:106408004FEA4302CED9A41A9DF80B305BB101AA1A
:1064180003213046FFF79EFD019B03F52573A34238
:10642800C0D2C0B9E41A9DF80C30002BBCD0A4F23D
:10643800262204213046FFF70CFE77610546B3E7B4
:106448009DF80930002BDFD0009B03F525739C4293
:10645800A8D9E41AD8E70546A6E770B54FF4FA625A
:1064680086B00023CDE9022340F636330B600C4694
:1064780004A90646FEF774F90546002836D19DF8AA
:1064880011209DF8103013439DF81220134319D0A2
:1064980002AA02213046FFF75DFD002840D19DF891
:1064A80010302BB1029B03F24E2223681344236061
:1064B8009DF81230EBB1029B03F2B222236803EB82
:1064C800420323609DF81330EBB99DF814305BB19B
:1064D80001AA04213046FFF73DFD019B03F2262265
:1064E800236813442360D8B923687361284606B02B
:1064F80070BD9DF81130002BE4D0029B03F5257286
:1065080023681344DDE703AA03213046FFF722FD81
:10651800039B03F525722368134423600028D4D015
:106528000546E3E72DE9F743002406460D462046D5
:1065380015F80480B8F1000F00D010B103B0BDE821
:10654800F083671CB8F1FF0F15F8079029D1A71C35
:10655800EB5DB9F1030F36D8DFE809F0020B131B26
:10656800271D2C44E27802EB0323A6F834313C467D
:10657800DEE7271D2C44E27802EB0323A6F8363128
:10658800F5E7271D2C44E27802EB0323A6F83831FF
:10659800EDE7271D2C44E27802EB0323A6F83C31F3
:1065A800E5E7B8F1040F0ED802344246291901A8CC
:1065B8000DF099FC434601AA4946304604EB08070A
:1065C80000F0BEFAD3E76FF00300D0E773B50023FD
:1065D8000E4613600DF1070105461446FEF7F7F85D
:1065E80040B99DF807302BB1B38A2A6A53438033E8
:1065F8001B0A236002B070BD13B5CB681360144644
:1066080001AAFFF7E3FF18B92368019A134423602E
:1066180002B010BDF8B5B0F85451D0F8580168432D
:106628008030000A0E464543DDE90717144652B18B
:10663800B60206EB5202B2FBF4F202EB42025243FC
:1066480002F50042140C069A534301F50042120C5D
:1066580006200332B2FBF0F2C2EBC202B2F5803F71
:1066680038BF033103F500433EBFB1FBF0F1C1EB86
:10667800C10101F500414FEA134334BF090C1B491E
:1066880003FB03F338BF494303EB57030B44B3FB46
:10669800F7F39B03FE2205F120007F33B3FBF2F3EF
:1066A8005C434FF47A7704F5FA748009B4FBF7F485
:1066B8002401FFF72DF904F5FA74BC4228BF4FF402
:1066C800FA63064629BFB4FBF3F300205B19B4FB59
:1066D800F7F428BFB3FBF4F0FFF71AF9099B8642D9
:1066E80094BF1E6018600020F8BD00BF0000F0FFD6
:1066F8002DE9F04F91B0CDE90723036A0E930B699A
:1067080009930546CB680B930F460FAAFFF774FF52
:106718000EAA39462846FFF759FF58BB0F9C95F833
:10672800E0B0D5F8DC3005934FF47A7606FB04F137
:1067380001F5004104910E990A910499D5F8E430C5
:106748000693BBF1080F04F180040CBF0223032356
:1067580024F0FF0A090C95F8E820DFF8A081CDF8AD
:106768003CA00C9109D1079BC3F80080089BC5F891
:106778004081186011B0BDE8F08F06990D93284646
:10678800FFF7C4FB5A46059981462846FFF7BEFB2A
:106798000D9B5B490C9A814403FB09F94FEAC9290F
:1067A80040F2776309F5FA79240AB9FBF6F903FB95
:1067B80009F909F5FA79B9FBF6F909FB04F404F1CA
:1067C8008003099C74430C40B4FBF2F44D4A1B0A45
:1067D800944228BF1446012B38BF01230C204FF4E4
:1067E800167258435443FFF793F83B7E3A894FEAB1
:1067F800400B002B7FD14249049B0B4003F5FA71F3
:10680800414B5A4341F25C23B2FBF3F20A9B7343B8
:10681800B3F5481F28BF4FF44813A1EB4303B1FB5E
:10682800F6F1B3FBF6F31B02B3FBF1F63602C6F53D
:106838008036564306F50046360C06F5803676084F
:106848007643B60B4FF44870704304F5004300F5E7
:1068580000401B0C5B43000C00FB0030FFF758F8AE
:1068680003046422323341F28837B3FBF2F340F673
:10687800B532B3FBFBF302FB0377244B9F429CBF6B
:1068880042F21073B7FBF3F7DDE90532134403F561
:10689800FA734FF47A7B4FF4FA62B3FBFBF0B3FB65
:1068A800F2F202F5C812B2FBF0F088BF4FF470475D
:1068B800FFF72EF8000200F5FA70B0FBFBF040433A
:1068C80007FB0700FFF724F80BFB00F0079B0B9A68
:1068D800404528BF40461860089BC5F84001CDE9EF
:1068E80002934FF448730093019433465146284667
:1068F800FFF790FE3EE74FF48036A3E7AE878F029E
:106908000000FFFF666666009A9906000F279F241D
:106918002DE9F04F8BB0002711F0780FDDE914B89E
:106928000446019299468DF80E708DF80F708DF817
:1069380010708DF81170ADF812700997C1F3C30A81
:1069480000F0AF80AAF10503DBB20A2B01D86B4A2D
:10695800D75C0DF10E0200212046FDF792FF9DF84D
:106968000E500646D5B1002840F09D8009AB05AA17
:1069780059462046FFF7BCFE002840F09680099B48
:10698800ABF80A30014606AA2046FDF7B3FF069D7C
:1069980025B1059B9D422CBF0025012520B904AADD
:1069A80002212046FDF76DFF9DF8106026B30028F0
:1069B8007DD107AA02212046FDF79CFF88B9012254
:1069C800FF21204600F0F0F858B90DF11202B62167
:1069D800204600F037F920B90246FF21204600F092
:1069E800E3F8BDF81230079E5B02C4F848311EB1C7
:1069F8009E422CBF0026012628B90DF11102032161
:106A08002046FDF73EFF9DF8113093B1002873D161
:106A1800B9F1000F03D0019B1B02B3FBF9F908AAD7
:106A280003212046FDF766FF089B4B4594BF0023D2
:106A3800012320B9012F3CD1FF2288F8002098F8C3
:106A480000200AB9ABF80A200DF10F0201212046F7
:106A58000193FDF716FF08BB9DF80E20019B002A45
:106A680008BF0125BAF1040F18BF9DF80F2084F85C
:106A78002E501ABFB2FA82F25209012284F82F204E
:106A88009DF81020002A9DF8112008BF0126002A31
:106A980008BF012384F8306084F831300BB0BDE8BA
:106AA800F08F012755E700257EE735467CE700266D
:106AB800A9E70AF1FF32092A0AD8DFE802F005053A
:106AC80005090907090B070B0522B6E70422B4E7F5
:106AD800012E01D10322B0E7BAF1040F01D0012B36
:106AE80001D10222A9E7012D1BBF002388F800303D
:106AF80088F800502B46A2E70023A0E7864101084A
:106B080007B502F10A03009393B20A4690F86011A0
:106B1800D0F85C0101F0B2FB03B05DF804FB13B5DB
:106B280002F10A0390F860410093D0F85C0193B237
:106B38000A4644F0010101F037FC02B010BD000024
:106B48003F2BF8B50E46054611461C4611D80A4F8C
:106B580038461A4600F8016B0DF0C5F9621C394633
:106B68002846FFF7CDFF00280CBF00206FF0130068
:106B7800F8BD6FF00300FBE7900E002073B51546D3
:106B88008DF8071001220DF1070104461E46FFF794
:106B9800B7FF28B9324629462046FFF7C0FF08B19B
:106BA8006FF0130002B070BD08B5064B19705A702B
:106BB80019460222FFF7A4FF002814BF6FF0130044
:106BC800002008BD900E002008B5074B1970110A67
:106BD80059709A7019460322FFF792FF002814BFD4
:106BE8006FF01300002008BD900E002037B5154641
:106BF8008DF8071001220DF107010446FFF780FF09
:106C080028B9012229462046FFF789FF08B16FF00D
:106C1800130003B030BDF7B515460DF1070206465F
:106C28000F461C46FFF7E2FF50B99DF807301D409C
:106C380044EA0502394630468DF80720FFF7B4FFCD
:106C480003B0F0BD73B514468DF8071001220DF19D
:106C580007010646FFF754FF18B16FF0130002B0A2
:106C680070BD074D022229463046FFF758FF00281D
:106C7800F3D12A786B7803EB02232380EFE700BF78
:106C8800900E002073B514468DF8071001220DF1FF
:106C980007010646FFF734FF18B16FF0130002B082
:106CA80070BD0A4D042229463046FFF738FF0028F8
:106CB800F3D16B782A781B0403EB0263EA78134458
:106CC800AA7803EB02232360E9E700BF900E0020B7
:106CD80008B50220FBF718FF002008BD7047000028
:106CE80010B5032000F072FC01F0AAFD064B1860F5
:106CF8000F20FBF7FFFE044618B9FBF772FD20468C
:106D080010BD0124FBE700BF280800204FF0E02257
:106D1800136923F00203136170474FF0E0221369EF
:106D280043F0020313617047014BD3F89005704795
:106D38000070FF1F014BD3F8940570470070FF1FC8
:106D4800014BD3F8980570470070FF1F024A53683B
:106D580023F0010353607047002004E0024A53689F
:106D680023F0020353607047002004E0024A53688E
:106D780023F0040353607047002004E08068C0F3E8
:106D880080007047F7B5002301930446002800F0FF
:106D9800E980856D25B9FBF761F8E56584F85450FD
:106DA80023689A68D00040F1A1809A68D10000F168
:106DB800B480A26D42F01002A265E26D42F00102B9
:106DC800E26501251846FFF7D9FFA26D02F010020F
:106DD800024340F0C980A26D206922F4817242F01A
:106DE8000202A2659A68D2075DD4226BA67E94F847
:106DF8002CC0003A18BF01221703D4E902120A4333
:106E0800217E42EA8132617E42EAC13242EA46325A
:106E1800002842EA4C02B4BF20F000414FF40011B0
:106E28003A430A4394F82010012903D1002E76D161
:106E380042F48032616A21B1A66A01F4E0713143FB
:106E48000A43D968E66C21F4FE3121F4FF7111433D
:106E5800D96094F83C206168012A01F0404C4CEA62
:106E6800060609D1D4E910273A433243A66C3243C7
:106E780042EA0C0242F001061F693E4A3A40324398
:106E88001A6121F00042B2F1804F0CD0B1F1004FED
:106E980009D0394ED6F8082701F4701122F470127F
:106EA8000A43C6F808275A69666BA16B22F00702E5
:106EB80032435A615A6922F0700242EA01125A6159
:106EC800002835D19A6A62F00F029A625B6903F072
:106ED80007039E423CD10023E365A36D23F003031F
:106EE80043F00103A365284603B0F0BD9A6823491F
:106EF80022F0104222F0170242F080529A60204A93
:106F08001268B2FBF1F2013252000192019A002A92
:106F18003FF44BAF019A013AF7E7002552E7A16D1C
:106F280041F02001A165E16D41F00101E16581E7D2
:106F3800B0F5001FCAD19A6AE269013A92006FF06F
:106F48000F0102F01C0201FA02F2216E0A43BCE7AB
:106F5800A36D23F0120343F01003A365E36D43F020
:106F68000103E3650125BEE7A36D43F01003A365A4
:106F7800F8E700BF02FCFF1F00200140400D03009E
:106F880028080020F8B54569082D04460E460AD0A1
:106F98000368DB68D80705D5A36D43F02003A36514
:106FA8000120F8BD0425FBF7A7FD074623681A68EA
:106FB8002A4221D0A26D42F40072A265DA6812F466
:106FC800406F14D1A27E92B91A6812070FD51846DD
:106FD800FFF7D4FE28BB5A6822F00C025A60A26D53
:106FE80022F4807222F0010242F00102A265207EA2
:106FF80000BB0C221A60D4E7711CD8D0FBF77CFDCB
:10700800C01BB04201D8002ED0D123681B682B408A
:10701800CCD1A26D84F8543042F00402A26503205A
:10702800BFE7A26D42F02002A265E26D42F00102C4
:10703800E265DCE70020B4E70368186C70470000DD
:10704800F7B50023019390F85430012B044600F063
:10705800C58005680669012380F854302846FFF783
:107068008DFE002840F0B480D1E90020022826F0E7
:10707800040300F08280B3F1004FC2F3110E13D164
:10708800AB6A43EA0E03AB628B68686903EA0223C2
:1070980023F07C4323F0FF0320EA02210B43002A5C
:1070A8006B6126DB002055E0236E00F01F074FF0D0
:1070B8000F0C0CFA07FC6FEA0C0623EA0C0CBEF165
:1070C800000F11D1C2F38463BB4043EA0C0323666B
:1070D8008008E36901309842D6D8A86AC2F383636E
:1070E800BB4006403343CEE792FAA2F3B3FA83F3E8
:1070F800EAE73B493B48D1F80837824203F0E0759C
:1071080019D11B02CED4D1F8083723F0E0732B43F2
:1071180043F40003C1F80837334B1A68334BB2FB0A
:10712800F3F20C2302FB03330193019B002BB9D02C
:10713800019B013BF8E72E48824210D113F0807082
:10714800B0D1D1F8083723F0E0732B4343F08073B4
:10715800C1F80837002384F8543003B0F0BD25483F
:1071680082429FD113F480009CD1D1F8083723F0D4
:10717800E0732B4343F48003EAE7B3F1004F01BF08
:10718800AB6AC2F311018B43AB62002A8ADA154855
:1071980013498242D1F8083709D1D1F8082703F0FA
:1071A800A07322F0E0721343C1F808377AE7104859
:1071B800824204D1D1F8082703F44003F1E70D48CF
:1071C80082427FF46FAFD1F8082703F0C073E8E775
:1071D800A26D42F02002A2651846BBE70220BCE778
:1071E80000200140001000B028080020400D0300D6
:1071F800004000B8002000B4026838B504461046C4
:10720800FFF7BCFD08B9002038BD9368990707D47B
:10721800936823F0004323F0170343F010039360AF
:10722800FBF76AFC054623689B685B07EBD5FBF711
:1072380063FC401B0228F6D923689B685A07F2D5DD
:10724800A36D43F01003A365E36D43F00103E36509
:107258000120D9E773B50023026801939368DD071D
:10726800044602D5002002B070BD9168214B194236
:1072780009D0A36D43F01003A365E36D43F0010348
:10728800E3650120EFE7936823F0004323F0170339
:1072980043F001039360184BD3F8083718021CD445
:1072A800637E012BDED0FBF727FC144E05462268CF
:1072B8001368DB07D6D49368D9075FBF9368334058
:1072C80043F001039360FBF717FC401B0228EED93B
:1072D80023681B68DA07EAD4CBE7094B094A1B681D
:1072E800B3FBF2F301330193019B002BD8D0019B30
:1072F800013BF8E71700008000200140E8FFFF7F0E
:1073080028080020400D030038B504460068FFF740
:1073180035FD054620BB94F85430012B20D00123BD
:1073280084F854302046FFF795FFB0B9A36D226862
:1073380023F4706323F0010343F48073A3651C23D3
:10734800E065136084F85400936823F0004323F049
:10735800170343F00403936038BD84F85450FBE7E7
:107368000220F9E7026838B5936891680446C807AF
:1073780001D4002038BD9907FBD4936803F00503B6
:10738800012B19D1936823F0004323F0170343F02E
:107398000203936003231360FBF7AEFB05462368E3
:1073A8009B68DB07E5D5FBF7A7FB401B0228F6D94E
:1073B80023689B68DA07F2D5A36D43F01003A36531
:1073C800E36D43F00103E3650120D3E770B504469C
:1073D80000284BD0836D43F002038365FFF70CFF51
:1073E800054668B92046FFF7BDFF054608B90123E1
:1073F800A3652268936823F0104323F01703936072
:1074080023685A6822F4677222F003025A6040F235
:107418009F321A60D968164A0A40DA601A6922F05F
:1074280040421A615A6922F007025A611A6A02F048
:10743800F0221A625A6A02F0F0225A62DA6A02F0FC
:10744800F022DA629A6A0B4A00269E62D2F808375E
:1074580023F0FE73C2F808372046FAF713FDE665F5
:107468002666A66584F85460284670BD0125FBE7AA
:1074780000023E830020014010B590F85430012BE3
:10748800044615D0012380F85430FFF7B5FE58B9EB
:107498002046FFF767FF38B9A36D23F4807323F004
:1074A800010343F00103A365002384F8543010BDA1
:1074B8000220FCE7F7B50023019390F85430012B24
:1074C80004467FD0012380F85430FFF74BFF236830
:1074D8009A6812F00102054607D0A36D43F0100325
:1074E800A365002384F854302DE0A16D364F21F4B4
:1074F800817141F00201A165DE68D96826F4FF4672
:1075080026F07C0621F40041360421F00301360CF4
:10751800D96008209968394041F00041996099681C
:10752800002913DA0199013101910199B1F52E3F32
:10753800F5D3A36D23F0120343F01003A3650023D2
:1075480084F854300125284603B0F0BDD3F8B410B0
:10755800013801F07F010A44DCD199681A480140DA
:1075680041F001019960D3F8B41021F07F0141EA9C
:10757800D202C3F8B4209A68024042F002029A602C
:10758800FBF7BAFA074623689A68D20708D4DA687C
:107598003243DA60A36D23F0030343F001039FE74E
:1075A800FBF7AAFAC01B0228EDD923689B68D90704
:1075B800E9D5A36D43F01003A365E36D43F0010320
:1075C800E365BFE70225BEE7E8FFFF7F0749CA6812
:1075D80022F4E0620302120403F4E063120C134382
:1075E80043F0BF6343F40033CB60704700ED00E025
:1075F800164B30B5DC68C4F30224C4F10703251D1B
:10760800042B28BF0423062D4FF0FF358CBF033C05
:10761800002405FA03F321EA0303A54022EA050240
:10762800A340002843EA0203ACBF00F16040084AC7
:107638004FEA0313B8BF00F00F00DBB2AABF00F592
:107648006140135480F8003330BD00BF00ED00E006
:1076580014ED00E0002807DB044A4109012300F08B
:107668001F00834042F82130704700BF00E100E06E
:1076780000280CDB4309064900F01F0020330122D3
:10768800824041F82320BFF34F8FBFF36F8F7047BD
:1076980000E100E070B5D0E913456560446D14B1B0
:1076A800D0E916456560D0E9105404F01C060124A1
:1076B800B4406C60046863608368102B0BBFA260E1
:1076C800A160E160E26070BD0268416CD3B210B5A0
:1076D800083B1424B3FBF4F30B4CA24288BF0B4ABB
:1076E80021F0030199BF01F1804202F502325218DC
:1076F80007338264064AC26403F01F03012202FAB8
:1077080003F3036510BD00BF070402401C080240D4
:107718008008024038B500285ED002682F4B9A4294
:107728004FF014014CD82E4B1344B3FBF1F32D4901
:107738009B00C0E91013022380F8253013680569FF
:1077480023F4FF4323F070031360D0E9024323437B
:107758002B43456911682B4385692B43C5692B4326
:10776800056A2B430B431360FFF7AEFFB4F5804F58
:1077780004BF002343604268816C02F07F030B6002
:10778800D0E91314013A032A4C6020D8164A174945
:1077980081651A44013B9200012103F0030301FAB9
:1077A80003F300214265C3651160114A5364002345
:1077B8000122C36380F8243080F82520184638BD9C
:1077C8000C4B1344B3FBF1F30B499B00B1E70023C7
:1077D800C0E91533C365EAE70120F0E70704024072
:1077E800F8FFFDBF000002403F8200104009024040
:1077F80000090240F8FBFDBF0004024038B500282C
:1078080041D00268136823F0010313601F4B9A42AA
:107818004FF0140130D81E4B1344B3FBF1F31D494C
:107828009B00C0E91013012403F01C0304FA03F3BE
:10783800002515604B60FFF747FF836C41681D60AA
:10784800D0E913325A604A1E032A06D8124B0B4459
:107858009B0094401D60114B5C640023C363C0E926
:107868001533C0E90B33C0E90D33C36580F8253003
:1078780080F82430184638BD094B1344B3FBF1F3A4
:1078880008499B00CDE70120F5E700BF0704024047
:10789800F8FFFDBF000002403F82001000090240CF
:1078A800F8FBFDBF0004024070B590F82450012D8C
:1078B80004463BD090F825600125AE4280F824505C
:1078C8004FF000062CD1022580F825500568C663C4
:1078D8002E6826F001062E60FFF7DCFE036BBBB1B5
:1078E8002B6843F00E032B60A36C1A68D20342BFC7
:1078F8001A6842F480721A60636D1BB11A6842F408
:1079080080721A602B6843F001032B60002070BD61
:107918002B6823F004032B602B6843F00A03E2E78B
:107928008023C36380F824602846F0E70220EEE74E
:10793800034640B190F82520022A06D00422C263EB
:10794800002280F82420012070470268806C1168AA
:1079580021F00E011160016821F480710160116845
:1079680021F001011160D3E9100202F01C0101228B
:107978008A404260D3E9132151605A6D32B11168CF
:1079880021F480711160D3E9162151600122002091
:1079980083F8252083F82400704710B590F8253027
:1079A800022B03D00423C363012010BD03681A68A7
:1079B80022F00E021A601A6822F001021A60826C24
:1079C800136823F480731360D0E9101303F01C02CA
:1079D800012393404B60D0E913325A60436D33B1B1
:1079E8001A6822F480721A60D0E916325A600123AC
:1079F80080F82530836B002480F8244013B1984721
:107A08002046D2E71846D0E770B4426C046C03688D
:107A180026681D6802F01C020421914031420FD0F3
:107A280015F0040F0CD01A6892065EBF1A6822F08F
:107A380004021A60036B6160002B33D070BC1847D6
:107A480002219140314217D015F0020F14D01A6864
:107A5800940606D41A6822F00A021A60012280F8F5
:107A68002520114A93428CBF104B114B59600023BB
:107A780080F82430C36ADFE708219140314211D0F1
:107A880029070FD5196821F00E011960012303FA9F
:107A980002F26260C36380F82530002380F8243046
:107AA800436BC9E770BC7047800002400004024085
:107AB800000002400A4A536943F4802330B55361F9
:107AC800EFF3108472B60023CD58C5500433B3F5D4
:107AD800807FF9D11369DB03FCD484F3108830BDAF
:107AE80000400058064B5A69002ABFBF054A9A60F1
:107AF80002F188329A60BABF5869C00F00207047F7
:107B08000040005823016745044B5A6942F000427F
:107B18005A615869C043C00F704700BF0040005801
:107B280070B50546FAF7E8FF124E04463369D903E3
:107B380013D43369DA0744BF012232614CF2FA32B6
:107B4800134011D10B4E306910F480200BD0FAF796
:107B5800D3FF001BA842F6D304E0FAF7CDFF001BC1
:107B6800A842E3D3032070BD024A1361024A0120F0
:107B78005360F8E700400058D00E00202DE9F0418E
:107B8800184D98462B78012B06460C46174626D0EA
:107B980001232B704FF47A7000236B60FFF7C0FF4E
:107BA800A0B9012E16D1104A536943F0010353615D
:107BB8002760BFF36F8FC4F804804FF47A70FFF723
:107BC800AFFF094A536923EA0603536100232B7068
:107BD800BDE8F08139462046FFF76CFFEDE702204B
:107BE800F6E700BFD00E002000400058054A536950
:107BF80023F47E7343EAC00040F4803040F0020072
:107C080050617047004000582DE9F041234F3B7800
:107C1800012B054688463FD001233B704FF47A700C
:107C280000237B60FFF77CFF044688B92B68042B90
:107C380013D11B4A536943F4803343F0040353615F
:107C48004FF47A70FFF76CFF0446154B1A681B68EF
:107C580000233B702046BDE8F0814FF0FF33C8F8A1
:107C680000306E68D5E901321344B3420AD9304670
:107C7800FFF7BCFF4FF47A70FFF752FF50B1C8F816
:107C880000600446064A536923F47E7323F0020316
:107C98005361DAE70136E5E70224DBE7D00E00207E
:107CA800004000582DE9F04F524C00234FF00F09C7
:107CB8000A6832FA03F501D1BDE8F08F012505FA0B
:107CC80003F818EA020200F08E804E68032706F0D7
:107CD80003054FEA430E07FA0EFC6F1E012F6FEAE9
:107CE8000C0C32D8876807EA0C0ACF6807FA0EF737
:107CF80047EA0A078760476827EA0808C6F30017B3
:107D08009F4047EA08074760C76807EA0C088F687A
:107D180007FA0EF747EA0807022DC76017D14FEA9E
:107D2800D30800EB880803F0070AD8F820704FEA58
:107D38008A0A09FA0AFB27EA0B0B0F6907FA0AF7FE
:107D480047EA0B07C8F8207001E0032DDCD107686B
:107D580005FA0EF507EA0C073D4316F4403F0560A7
:107D680041D023F0030707F1804707F5803703F078
:107D7800030CBD684FEA8C0C4FF0070E0EFA0CFE90
:107D8800B0F1904F25EA0E0E2FD01B4DA8422ED0F1
:107D980005F58065A8420CBF0225072505FA0CF5F4
:107DA80045EA0E05BD602568D74316F4801F0CBF51
:107DB8003D4015432560656816F4001F0CBF3D4023
:107DC80015436560D4F8805016F4803F0CBF3D40E1
:107DD8001543C4F88050D4F88450B60354BF3D40CE
:107DE8001543C4F88450013362E70025D6E701251E
:107DF800D4E700BF0008005800040048374A2DE9BE
:107E0800F04F00234FF0010A4FF0070B4FF00F0916
:107E180031FA03F401D1BDE8F08F0AFA03FC1CEA39
:107E2800010654D023F0030404F1804404F580349F
:107E380003F00307A568BF000BFA07F8B0F1904FED
:107E480008EA050E45D0264DA84244D005F58065C0
:107E5800A8420CBF02250725BD40754517D1D2F8A9
:107E6800805025EA0605C2F88050D2F8845025EAE9
:107E78000605C2F88450156825EA06051560556898
:107E880025EA06055560A56825EA0805A560056880
:107E980003265C0006FA04F423FA06F6254300EBF1
:107EA8008606056003F00705376AAD0009FA05F58F
:107EB80027EA05073762856825EA0405856045686D
:107EC80025EA0C054560C56825EA0404C460013349
:107ED8009EE70025C0E70125BEE700BF000800585F
:107EE800000400480369194214BF012000207047AC
:107EF8000AB181617047816270470000044AD16805
:107F0800014208B502D0D060FBF70EFB08BD00BFE8
:107F18000008005803689A69910744BF00229A62D2
:107F28009A69D2075EBF9A6942F001029A61704766
:107F380030B5039D04682B4343EA0243064A606850
:107F4800C1F309010B4342EA555223F0004320EAEA
:107F580002000343636030BDFF63FF0303682DE93C
:107F6800F0419C6914F0100405460F4616466FD080
:107F780010220024DA61A0462B689A69900661D421
:107F8800B8F1000F35D044F0040401202E68B3691D
:107F9800D90541BF4FF48072F26144F00104012019
:107FA8005A0541BF4FF4806244F00804F261012091
:107FB8009B054FD54FF4007344F00204F361284643
:107FC800FFF7A8FF736823F0FF7323F48B3323F4C0
:107FD800FF7323F0010373606B6C23436B642023EE
:107FE80085F84130002385F8423085F8403001207B
:107FF80032E07A1CC1D0FAF77FFD801BB84201D865
:10800800002FB9D12B68596895F842209869000467
:10801800D2B20AD5490408D4202A06D05A6842F4B4
:1080280080425A60FAF768FD06462B689B699B06F2
:10803800A2D4FAF761FD801B1928F6D920244FF045
:10804800010899E7B8F1000F9DD12022DA619AE77B
:1080580020469BE70028B2D1BDE8F08170B5044600
:108068000D46164623689B699B0701D5002070BD05
:10807800324629462046FFF771FFA0B96A1CF1D0A5
:10808800FAF73AFD801BA84201D8002DEAD1636CAB
:1080980043F020036364202384F84130002384F8EC
:1080A800423084F840300120E1E770B504460D46BF
:1080B800164623689B695B070ED43246294620463C
:1080C800FFF74CFF38BB23689A69910625D59A6952
:1080D800520703D5228D0AB1002070BD9A6912F0AB
:1080E80010021CBF1022DA614FF0200118BF0422D1
:1080F8006264D9615A6822F0FF7222F48B3222F44A
:10810800FF7222F001025A60002384F8411084F8BB
:10811800423084F840300120DFE7FAF7EDFC801B9D
:10812800A84201D8002DC4D1636C43F020036364D6
:10813800202384F841300023EBE72DE9F041069F26
:108148000446884616461D462268936938EA0303A2
:108158000CBF01230023B34201D0002015E06B1CA3
:10816800F3D0FAF7C9FCC01BA84201D8002DEBD107
:10817800636C43F020036364202384F841300023B8
:1081880084F8423084F840300120BDE8F08170B5B1
:1081980004460D46164623689B699B0601D50020B8
:1081A80070BD324629462046FFF7D8FE90B9FAF747
:1081B800A3FC801BA84201D8002DECD1636C43F0CE
:1081C80020036364202384F84130002384F842307C
:1081D80084F840300120E3E710B5044600284AD06F
:1081E80090F8413003F0FF021BB980F84020FAF7FD
:1081F80085F9242384F8413023681A6822F00102A3
:108208001A60626822F070621A619A6822F4004269
:108218009A60D4E90221012924D142F400429A60EB
:108228005A6842F0007242F400425A60DA6822F456
:108238000042DA60D4E904210A43A16942EA012232
:10824800DA60D4E907210A431A601A6842F0010289
:108258001A6000202023606484F84130206384F889
:10826800420010BD42F4044202299A6004BF4FF450
:1082780000625A60D4E70120F3E700002DE9F347D4
:10828800984690F841300A9F202B04460E469146A6
:1082980040F0868090F84030012B00F081804FF04C
:1082A800010A80F840A0FAF727FC19230546009038
:1082B80052464FF400412046FFF73FFF18B1012016
:1082C80002B0BDE8F087212384F84130102384F8F8
:1082D80042306064A4F82A80638DC4F824909BB26D
:1082E800FF2B60632F4B26D9FF22228500934FF086
:1082F800807331462046FFF71BFE638D9BB22A46EA
:1083080039462046FBB9FFF742FF0028D7D123683A
:108318002021D9615A6822F0FF7222F48B3222F4AC
:10832800FF7222F001025A6084F8411084F840007C
:1083380084F84200C4E7628D009392B222854FF020
:108348000073D2B2D5E7FFF789FE0028B7D1636A78
:10835800226813F8011B91626362638D228D013BD1
:108368009BB26385638D013A92B29BB22285002B42
:10837800C3D0002AC1D100953B4680212046FFF793
:10838800DCFE00289BD1638D9BB2FF2B03D9FF2213
:1083980022850090ABE7628D009092B22285CEE7ED
:1083A80002208DE7002000802DE9F347984690F8D9
:1083B80041300A9F202B04460E46914640F08780A4
:1083C80090F84030012B00F082804FF0010A80F8CD
:1083D80040A0FAF791FB19230546009052464FF446
:1083E80000412046FFF7A9FE18B1012002B0BDE800
:1083F800F087222384F84130102384F842306064E7
:10840800A4F82A80638DC4F824909BB2FF2B606384
:10841800304B26D9FF22228500934FF080733146D6
:108428002046FFF785FD638D9BB22A4639462046D4
:10843800FBB9FFF7ACFE0028D7D123682021D9610A
:108448005A6822F0FF7222F48B3222F4FF7222F073
:1084580001025A6084F8411084F8400084F8420010
:10846800C4E7628D009392B222854FF00073D2B2B6
:10847800D5E7FFF71AFE0028B7D123685A6A636A5E
:108488001A70636A228D01336362638D013B9BB26C
:108498006385638D013A92B29BB22285002BC2D0CC
:1084A800002AC0D100953B4680212046FFF745FEB3
:1084B80000289AD1638D9BB2FF2B03D9FF22228516
:1084C8000090AAE7628D009092B22285CDE7022043
:1084D8008CE700BF0024008010B590F84120202AC6
:1084E8000346D4B21CD190F84020012A18D0242287
:1084F80080F841200268106820F0010010601068C0
:1085080020F4805010601068014311601168002049
:1085180041F00101116083F8414083F8400010BD2B
:108528000220FCE710B590F84120202A0346D4B277
:108538001BD190F84020012A17D0242280F841202E
:108548000268106820F001001060106820F4706064
:1085580040EA012111601168002041F00101116019
:1085680083F8414083F8400010BD0220FCE700007A
:10857800024A136843F4807313607047000400587C
:108588000D4B10B55B690C4628B99A0507D500F064
:1085980027F820B110BD9B0501D400F019F8074A4F
:1085A8001369012C23F00403136101D130BFF1E7F3
:1085B80040BF20BF20BFEDE70004005800ED00E0F9
:1085C800024B186800F4C060704700BF00040058F0
:1085D800024A136843F4804313607047000400584C
:1085E8000C4A136823F4804313600B4B1B68322139
:1085F8004B430A49B3FBF1F35169890500D533B9F7
:10860800536913F4007F14BF032000207047013B17
:10861800F2E700BF000400582808002040420F007D
:108628000B4A136823F0070343F002031360094B56
:108638001A69012842F004021A6105D130BF1A698B
:1086480022F004021A61704740BF20BF20BFF6E73E
:108658000004005800ED00E04FF0B0431868C0F384
:10866800404070474FF0B0431868C0F3400070476F
:108678004FF0B042536823F47F4343EA002353602A
:1086880070474FF0B0431868C0F34060704700006F
:108698007FB54FF0B0432C4AD3F80831C0F303102C
:1086A80003F00F0352F82040284A52F82330B4FB55
:1086B800F3F4FFF785FF264B054693E80700B5F569
:1086C800007F04AB03E9070010D0224B9C4218D36B
:1086D80003F5B70303F67F539C4229D903F57413B6
:1086E80003F510639C4225D802230BE01A4B9C42E9
:1086F80007D91A4B9C421BD903F5370303F5D85306
:10870800F0E7002304AA02EB830353F80C4C144D42
:108718002B6823F0070323432B60FAF7EDF906468D
:108728002B6803F007039C4206D1002004B070BDFB
:108738000123E7E70024EAE7FAF7DEF9801B0228BD
:10874800EED90320F2E700BFF44101089441010883
:1087580030400108C0CF6A00BFEA21013F933402CC
:10876800004000584FF0B04310B59A68D96812F02D
:108778000C0205D00C2A4AD101F00303012B50D179
:108788004FF0B0412B480B6813F0080306D00B6874
:1087980013F0080337D1D1F8941007E00C682407C8
:1087A80056BFD1F894300968C3F3032350F8233037
:1087B800002A0CBF184600204FF0B0418A6802F02A
:1087C8000C020C2A1ED1CA6802F00302022A2ED01B
:1087D800032A06D10B68184A13F4801F174B18BFD9
:1087E80013464FF0B042D068D168D268C0F3062073
:1087F8005843C1F302130133B0FBF3F0530F0133B5
:10880800B0FBF3F010BD0B68C3F30313CEE7042AE3
:108818000AD0082A05D11B6813F4801304D107482D
:10882800CAE700231846C7E703480023C4E7024BFA
:10883800D7E700BFF44101080024F4000048E8012C
:1088480008B5FFF78FFF4FF0B043044A9B68C3F3A6
:10885800031352F82330B0FBF3F008BD944101082C
:108868002DE9F0410446002853D04FF0B0439D68ED
:10887800DE6803689B0605F00C0506F0030668D55C
:10888800026A1DB10C2D46D1012E44D1002A40D0D8
:108898004FF0B043A16A1A68170756BFD3F894304F
:1088A8001B681B0903F0F00399421FD90846FFF71C
:1088B800EFFE00282DD14FF0B042136843F00803B3
:1088C80013601368A16A23F0F0030B431360606A16
:1088D800FFF7CEFEFFF7B4FFAB4B1860AB4B186841
:1088E800FAF708F9002834D0BDE8F0814FF0B0421B
:1088F800136843F008031360136823F0F0030B4375
:108908001360606AFFF7B4FE0846FFF7C1FE00284F
:10891800E0D00120E8E74FF0B043002A54D01A68AD
:1089280042F001021A60FAF7E7F80746FFF79AFEE5
:10893800002842D04FF0B042136843F00803136098
:108948001368A16A23F0F0030B431360606AFFF712
:108958008FFE2368D80748D42368990700F18C80D4
:1089680023681E0740F1FA80A3694FF0B046002B38
:1089780000F0E180D6F89430E16903F010029142EA
:1089880000F0C48003F00302022AC2D0D80740F1E5
:10899800B380D6F8943023F00103C6F89430FAF780
:1089A800ABF80746D6F89430990740F1A580FAF756
:1089B800A3F8C31B112BF5D904E0FAF79DF8C01BE7
:1089C8000228B3D903208FE71A6822F001021A603F
:1089D800FAF792F80746FFF745FE0028B9D0FAF7EC
:1089E8008BF8C01B0228F6D9ECE7082D03D00C2D14
:1089F80005D1032E03D16368002BADD189E74FF071
:108A0800B043A1681A6822F480120A431A606268A7
:108A1800B2F5803F10D11A6842F480321A60FAF732
:108A28006BF80746FFF718FE002895D1FAF764F8A7
:108A3800C01B6428F6D9C5E7B2F5041F04D11A682B
:108A480042F400121A60E6E7196821F480311960CF
:108A5800196821F400111960002AE0D1FAF74CF8DE
:108A68000746FFF7F9FD00283FF476AFFAF744F818
:108A7800C01B6428F5D9A5E7042D236903D00C2D64
:108A88000ED1022E0CD1002B3FF443AF4FF0B04271
:108A98006169536823F0FE4343EA016353605FE76B
:108AA8004FF0B046BBB1336843F480733360FAF7D4
:108AB80023F8074633685A0507D57368626923F0B7
:108AC800FE4343EA026373604AE7FAF715F8C31BEB
:108AD800022BEFD976E7336823F480733360FAF713
:108AE8000BF8074633685B057FF53AAFFAF704F8E9
:108AF800C31B022BF6D965E74FF0B042E169D2F803
:108B0800943023F010030B43C2F894304FF0B04771
:108B1800D7F8943043F00103C7F89430F9F7ECFF25
:108B28000646D7F894309A0718D4F9F7E5FF831B5F
:108B3800112BF6D946E7D6F8943023F00103C6F88E
:108B48009430F9F7D9FF0746D6F894309B0705D536
:108B5800F9F7D2FFC31B112BF6D933E7236858075F
:108B680054D50B4F3B68D90514D4FFF701FDF9F72D
:108B7800C3FF06463B68DA050CD4F9F7BDFF831B33
:108B8800022BF7D91EE700BF280800202C08002078
:108B980000040058E3684FF0B046002B58D023F08B
:108BA8008003052B02BFD6F8903043F00403C6F8C3
:108BB80090304FF0B046F9F79FFFD6F8903043F069
:108BC80001030746C6F8903041F28838D6F890304D
:108BD8009B0705D4F9F790FFC31B4345F6D9F1E687
:108BE800E36823F00403812B1BD1F9F785FFD6F83E
:108BF800903043F08003C6F8903007464FF0B046F7
:108C080041F28838D6F89030180504D5E06A002873
:108C18004AD1002068E6F9F76FFFC01B4045F1D93B
:108C2800D0E6F9F769FFD6F8903023F08003C6F84C
:108C3800903007464FF0B04641F28838D6F8903069
:108C48001905E3D5F9F758FFC01B4045F6D9B9E631
:108C5800F9F752FFD6F8903023F080030746C6F89C
:108C6800903041F28838D6F890301A0516D4F9F7C2
:108C780043FFD6F8903023F00103C6F8903007463A
:108C88004FF0B04841F28836D8F890309B07BDD5F0
:108C9800F9F732FFC31BB342F6D993E6F9F72CFF75
:108CA800C01B4045DFD98DE60C2D4ED04FF0B043A8
:108CB80002281A6822F080721A6033D1F9F71CFF73
:108CC8000546FFF7DEFC38BBD4E90C314FF0B04263
:108CD8000B43D0682D4901400B43E16B0B43216CDA
:108CE8000B43616C0B43A16B43EA0123D360136808
:108CF80043F080731360D36843F08053D360F9F76F
:108D0800FBFE0446FFF7BDFC002882D1F9F7F4FE0C
:108D1800001B0A28F6D955E6F9F7EEFE401B0A288B
:108D2800CFD94FE6F9F7E8FE0446FFF7AAFC30B9B9
:108D38004FF0B042164BD1680B40D360D4E5F9F739
:108D4800DBFE001B0A28F0D93CE601283FF4CCAD35
:108D58004FF0B043226BDB6803F0030191427FF4CC
:108D6800D8AD616B03F070028A427FF4D2ADA16B7B
:108D780003F4FE42B2EB012F7FF4CBAD626C03F03B
:108D8800604393423FF445AFC3E500BF8C80C111F7
:108D9800FCFFFEEE2DE9F0410D46044610B9012016
:108DA800BDE8F081684E336803F007038B4216D3A1
:108DB80023689A0727D54FF0B047A268BB6823F00D
:108DC800F0031343BB60F9F797FE0646BB68DB0365
:108DD80019D4F9F791FE831B022BF7D911E03368F8
:108DE80023F007030B433360F9F786FE0746336821
:108DF80003F00703AB42DBD0F9F77EFEC01B022865
:108E0800F5D90320CCE72368580617D54FF0B047AB
:108E18006269D7F8083123F00F0343EA1213C7F841
:108E28000831F9F769FE0646D7F80831D90305D4A1
:108E3800F9F762FE831B022BF6D9E2E723685A078B
:108E480013D54FF0B047E268BB6823F4E0631343DF
:108E5800BB60F9F751FE0646BB689B0305D4F9F7DA
:108E68004BFE831B022BF7D9CBE72368180714D5D1
:108E78004FF0B0472269BB6823F4605343EAC2034A
:108E8800BB60F9F739FE0646BB68590305D4F9F704
:108E980033FE831B022BF7D9B3E72368DA070FD415
:108EA800294C236803F00703AB4239D8FFF7C8FC05
:108EB800264B1860264BBDE8F0411868F9F71ABE32
:108EC8006268022A1DD1FFF7C7FB00283FF467AF8D
:108ED8004FF0B04641F28838B36823F003031343D8
:108EE800B360F9F709FE0746B368626803F00C033C
:108EF800B3EB820FD4D0F9F7FFFDC01B4045F3D97F
:108F08007FE7032A02D1FFF7BCFBDEE712B9FFF7C0
:108F1800A9FBDAE74FF0B0431B685B05D8D43EE7FE
:108F2800236823F007032B432360F9F7E5FD064682
:108F3800236803F00703AB42B8D0F9F7DDFD801BC7
:108F48000228F5D95DE700BF004000582808002036
:108F58002C08002008B5FFF773FC4FF0B043044A13
:108F68009B68C3F3022352F82330D84008BD00BFE2
:108F7800D441010808B5FFF763FC4FF0B043044A39
:108F88009B68C3F3C22352F82330D84008BD00BF02
:108F9800D44101084FF0B043D3F89000C0F340002B
:108FA80070474FF0B0410209D1F8883002F47F22AF
:108FB800000123EA020300F47F200343C1F888304C
:108FC80070474FF0B041020CD1F88830120423EA00
:108FD800020343EA0040C1F88800704770B506688C
:108FE80016F48036044638D0FFF7C2FAF9F784FD44
:108FF800614E05463368DB0529D54FF0B043616BF8
:10900800D3F8902002F44072914214D0D3F8901013
:10901800D3F8902042F48032C3F89020D3F89020FF
:1090280021F4407022F480328D07C3F89020C3F8F1
:10903800900000F190804FF0B042616BD2F8903010
:1090480023F440730B43C2F89030002605E0F9F78B
:1090580053FD401B0228CDD903262568E8070AD509
:109068004FF0B0416268D1F8883023EA124392B2D7
:109078001343C1F88830A9070AD54FF0B041A26858
:10908800D1F8883023EA124392B21343C1F88830EA
:10909800AA0609D54FF0B0422169D2F8883023F4E6
:1090A80040630B43C2F88830AB0502D5206AFFF74E
:1090B80088FF680502D5606AFFF783FF290502D596
:1090C800A06AFFF77EFF6A0602D56069FFF769FFAD
:1090D8002B0602D5A069FFF764FFE80502D5E06911
:1090E800FFF75FFFE90610D54FF0B042E168D2F80C
:1090F800883023F440730B43C2F88830B1F5807F81
:1091080002BFD36843F08073D3602A040ED54FF0B2
:10911800B042216BD2F8883023F040430B43C2F8A9
:10912800883019B9D36843F08073D3606B0410D5C5
:109138004FF0B042E16AD2F8883023F040530B4335
:10914800B1F1005FC2F8883003D1D36843F48033AB
:10915800D360304670BDF9F7CFFC41F2883605463A
:10916800FFF718FF01283FF466AFF9F7C5FC401B6D
:10917800B042F5D970E700BF0004005830B590F848
:109188002C30012B02464FF0020022D0174B82F8F8
:109198002D00CA24012582F82C505C6253245C629D
:1091A800B1F5807F146B996914D121F488519961C4
:1091B800596C24F0010421F0004159641463DD6501
:1091C8000A4BFF2159620020012382F82D3082F8D2
:1091D8002C0030BD21F408519961D96C24F00204A7
:1091E80021F00041D9641463D865E9E700280040FC
:1091F80070B50B4E036B756D1D40EA07044603D529
:109208000123F365F9F7E9FDAB0704D50223F365FC
:10921800204600F0CBF9012384F82D3070BD00BF43
:109228000028004038B50A4CE36823F02003E360C7
:10923800F9F762FC0546E3689B0601D5002038BDB6
:10924800F9F75AFC401BB0F57A7FF4D90320F6E70A
:10925800002800402DE9F041114DEC6814F040045D
:1092680007461AD1EB6843F08003EB60F9F744FC3A
:109278004FF003080646EB685B0601D4032C02D1C5
:109288002046BDE8F081F9F737FC801BB0F57A7FFE
:1092980084BF87F82D800324EDE70024F0E700BFA2
:1092A8000028004038B50F4CE36823F08003E360E2
:1092B800A3699B06054606D4FFF7B4FF10B1032047
:1092C80085F82D0038BDA36923F02003A361FFF7BB
:1092D800A9FF10B1032085F82D00A36943F02003EE
:1092E800A361EFE70028004038B5044600284BD0BA
:1092F80090F82D3003F0FF021BB980F82C20F9F705
:1093080009FA0223214D84F82D30EB68DB0632D4AC
:10931800CA236B6253236B622046FFF79BFF78BB1F
:10932800AB6923F08E6323F04003AB612169636866
:10933800AA690B431343A2691343AB61D4E902231F
:1093480043EA02432B61D4E90931EA680B4322F46A
:10935800F8521343EB602046FFF7A4FF80B9D4E925
:109368000713AA690B4322F060421343626913434F
:10937800AB61FF236B62012384F82D30002002E0EB
:10938800024BFF225A6238BD0120FCE7002800404A
:109398000023092803D840EA0310C0B270470A38EE
:1093A8000133C0B2F5E700002DE9F04790F82C3002
:1093B800012B05464FF0020069D0012385F82C30B7
:1093C8004E4B85F82D00DE6806F44076B6F5807FB2
:1093D80078D04C69087891F8019091F802A091F83A
:1093E8002470002A55D19B6913F0400308BFCB7045
:1093F800FFF7CEFF80464846FFF7CAFF02465046B1
:10940800FFF7C6FF81463846FFF7C2FF0B6ACF78E1
:10941800234343EA875343EA090343EA084343EAF9
:10942800022343EA0063354ACA205062532050623F
:109438008C6A8869B4F5807F946945D124F488548E
:1094480094610124D465B6F5807F09BFCB691364A4
:109458000343536418BF5064284B4A681A672A6B41
:1094680042F001022A639A6942F488529A61244AB6
:10947800D2F8803043F40033C2F880301F4BFF220B
:109488005A620020012385F82D3085F82C00BDE8AC
:10949800F087B4F1803F07D0B4F5000F04D09B6982
:1094A80013F0400308BFCB700B6ACA781C4344EA28
:1094B8000A0444EA004343EA092343EA825343EA9D
:1094C8000763B0E70023AEE724F40854946102244C
:1094D800D465B6F5807F09BFCB6993640343D36431
:1094E80018BFD064054B4A685A672A6B42F00202DB
:1094F8002A639A6942F40852B8E700BF002800407E
:109508000008005890F82C20012A03464FF002006A
:1095180012D00A4A83F82D00CA21516253215162A0
:10952800916941F020019161FF21516200200122DF
:1095380083F82D2083F82C00704700BF00280040D6
:1095480090F82C20012A03464FF0020019D00D4A4A
:1095580083F82D00CA2151625321516291690A484A
:1095680041F080019161D0F8801041F48021C0F869
:109578008010FF2151620020012283F82D2083F8FA
:109588002C0070470028004000080058064B5A6D10
:10959800520610B5044603D54022DA65F9F720FCD7
:1095A800012384F82D3010BD002800407047890041
:1095B80001F1804101F531410A607047890001F1EC
:1095C800804101F53141086870470000034AD2F82C
:1095D800903043F40043C2F89030704700040058BC
:1095E800034AD2F8903023F40043C2F89030704711
:1095F80000040058074B1A6822F040021A6040F431
:1096080041704FF4B85218605A601A6842F040022C
:109618001A6070470000015837B5054600284ED03B
:10962800837903F0FF046BB1032C0BD0254B4FF467
:1096380000629A612868FFF7DDFF002401232B717F
:10964800AC602FE000236B712846F9F76DF91E4ACC
:10965800D2F8903043F48053C2F89030002CE5D112
:1096680002234FF0B042AB71D2F8943023F4004398
:10967800C2F89430154B1B681C214B43DB0C64214A
:109688004B430193019B93B90124AC60FFF79EFF04
:109698000C4B9A6842F400629A604FF400629A6137
:1096A800002CC7D00123AB71204603B030BD019B0D
:1096B800013B0193D2F894305B04E3D4E6E701243C
:1096C800F2E700BF000400580008005828080020EE
:1096D80037B5174D2B6802461C204343DB0C64202A
:1096E800434314480193019B93B901209060114CA6
:1096F80021732B681C214B43DB0C64214B430193E2
:10970800019B6BB9012090600A4BDB6803B030BD48
:10971800019B013B019383689C07E4D50020E6E7A1
:10972800019B013B0193A368DB07E9D5ECE700BF88
:10973800280800200000015837B5184D2B6802464C
:109748001C204343DB0C6420434315480193019BD1
:10975800A3B901209060124CFF2323732B681C25AA
:109768006B43DB0C64256B430193019B73B90120A8
:1097780090600B4BDB680B7003B030BD019B013B65
:10978800019383689C07E2D50020E4E7019B013B35
:109798000193A368DB07E8D5EBE700BF28080020A2
:1097A800000001580F4B13B51B680F4C1822534388
:1097B8001B0D64225343014601936269019B02F029
:1097C800040223B902238B60012002B010BD019B63
:1097D800013B0193606910F00200F6D0002AECD139
:1097E8001046F2E7280800200004005807B503795E
:1097F800012B0FD10A4B1B68182253431B0C0193F2
:10980800FFF7EEFE019B013B0193019B002BF9D171
:10981800FFF7DCFE03B05DF804EBFFF7C3BF00BF42
:1098280028080020F8B51E468379012B1546044602
:109838000F46DAB22DD14379012B2AD00223427187
:109848008371FFF7D3FF0D212046FFF7C9FEFFF70D
:109858003FFF390A2046FFF73BFFF9B22046FFF7E2
:1098680037FF2E44B5420ED12046FFF7AFFEFFF773
:1098780099FFA06801230038A3714FF0000318BFB7
:1098880001206371F8BD15F8011B2046FFF720FF82
:10989800E8E70220F6E7F8B51E468379012B15465E
:1098A80004460F46DAB22FD14379012B2CD04271EE
:1098B800FFF79CFF1D212046FFF792FEFFF708FFE8
:1098C800390A2046FFF704FFF9B22046FFF700FFE8
:1098D80000212046FFF7FCFE2E44B5420ED120465B
:1098E800FFF774FEFFF75EFFA06801230038A3713D
:1098F8004FF0000318BF01206371F8BD29462046C8
:10990800FFF71AFF0135E8E70220F6E7F8B51F462A
:109918008379012B154604460E46DAB22CD14379D9
:10992800012B29D04271FFF761FF06F0EF03A3F185
:10993800840253425341237131462046FFF750FEBB
:10994800FFF7C6FE2F44AF4210D1FFF73FFE842E2B
:1099580002D02046FFF726FFA06801230038A37134
:109968004FF0000318BF01206371F8BD15F8011B03
:109978002046FFF7ADFEE6E70220F6E7F8B51E46FB
:109988008379012B154604460F46DAB227D143796D
:10999800012B24D04271FFF729FF39462046FFF7F3
:1099A8001FFEFFF795FE00212046FFF791FE2E448B
:1099B800B5420ED12046FFF709FEFFF7F3FEA06877
:1099C80001230038A3714FF0000318BF0120637111
:1099D800F8BD29462046FFF7AFFE0135E8E702202B
:1099E800F6E737B50023ADF8043001AA02231221A7
:1099F8000546FFF7C3FFBDF80440022364BA01AA75
:109A0800A4B219462846FFF781FFE20702D5284687
:109A180009F088FBA30702D5284609F089FB6007EF
:109A280002D5284609F0AEFB210702D5284609F0E1
:109A3800AFFBE20602D5284609F0B0FBA30602D523
:109A4800284609F099FB600602D5284609F076FBFE
:109A5800210606D514F4807118BF0121284609F0A3
:109A680073FBA20502D5284609F07EFB630402D5E4
:109A7800284609F099FB03B030BDF8B51E46837936
:109A8800012B154604460F46DAB227D14379012B3C
:109A980024D04271FFF7AAFE0E212046FFF7A0FD51
:109AA800FFF716FE39462046FFF712FE2E44B54250
:109AB8000ED12046FFF78AFDFFF774FEA068012348
:109AC8000038A3714FF0000318BF01206371F8BD7F
:109AD80015F8011B2046FFF7FBFDE8E70220F6E733
:109AE800F8B51E468379012B154604460F46DAB2AF
:109AF8002BD14379012B28D04271FFF777FE1E2125
:109B08002046FFF76DFDFFF7E3FD39462046FFF7D6
:109B1800DFFD00212046FFF7DBFD2E44B5420ED1C4
:109B28002046FFF753FDFFF73DFEA06801230038EC
:109B3800A3714FF0000318BF01206371F8BD2946D7
:109B48002046FFF7F9FD0135E8E70220F6E702684D
:109B580052E8003F23F0C00342E8003102680029C0
:109B6800F5D102F1080353E8003F23F4000302F1A2
:109B7800080C4CE800310029F3D12023C0F88830C4
:109B88007047000010B5026852E8003F23F4907354
:109B980042E8003102680029F5D10F4C02F10803B0
:109BA80053E8003F234002F1080C4CE8003100293B
:109BB800F4D1C36E012B07D152E8003F23F0100304
:109BC80042E800310029F7D12023C0F88C30002367
:109BD800C366436710BD00BFFEFFFFEFF8B504463C
:109BE8001346D4F88850202D32D1F1B1EAB1E06F94
:109BF800A4F85620A4F8542000262122C4F8906026
:109C08002165C4F88820226888B1124FC762124FB4
:109C18000763124F2832C0E90D76FDF745FE30B1D3
:109C28001023C4F89030C4F8885001200FE023684E
:109C380040221A62226802F1080353E8003F43F009
:109C4800800302F1080141E800300028F3D1F8BD93
:109C58000220FCE7699C0008B19C0008BD9C000834
:109C680008B50346806A1B681B6813F0200317D1E8
:109C7800A0F85630026802F1080353E8003F23F0C9
:109C88008003083242E8003102680029F2D152E824
:109C9800003F43F0400342E800310029F7D108BDF6
:109CA800F9F7D4F9FBE7704708B5806AFFF7FBFFBF
:109CB80008BD7047806A38B50468D0F88830D0F895
:109CC8008C50A268120606D5212B04D10023A0F8D7
:109CD8005630FFF73CFFA3685B0606D5222D04D15A
:109CE8000023A0F85E30FFF74DFFD0F8903043F026
:109CF8001003C0F89030FFF7DCFF38BD08B5806A64
:109D08000023A0F85E30A0F85630FFF7D2FF08BD58
:109D1800704700000368D9691A682DE9F04140F6D8
:109D28000F0631429D68044610D18E0640F1978097
:109D380002F0200605F080573E4300F09080436F04
:109D4800002B00F08580BDE8F0411847AB4EAC48C9
:109D58002E401040304300F08280CF0709D5D0054F
:109D680007D501201862D4F8900040F00100C4F82B
:109D780090008F0709D5E80707D502201862D4F8A4
:109D8800900040F00400C4F890004F0709D5E80798
:109D980007D504201862D4F8900040F00200C4F8F7
:109DA80090000F070BD502F02000304307D00820A1
:109DB8001862D4F8900040F00800C4F890000E052E
:109DC8000AD5500108D54FF400601862D4F89030D5
:109DD80043F02003C4F89030D4F89030002B37D0EB
:109DE8008B0609D502F0200205F080552A4303D0DE
:109DF800636F0BB1204698472668D4F89020B36863
:109E080002F0280203F0400353EA0205204621D05D
:109E1800FFF7B8FEB3685F0617D5226802F108039A
:109E280053E8003F23F04003083242E8003100299C
:109E3800F3D1D4F8800040B1724B8363FDF7ADFDD8
:109E480030B1D4F88000836B7DE72046FFF731FFFF
:109E5800BDE8F081FFF72DFFC4F89050F8E7E06EF9
:109E6800012840F08980CE0640F18680D00640F176
:109E7800838010221A629A6851064BD5D4F8802044
:109E880011684A6892B2002AE2D0B4F85C009042A5
:109E9800DED9A4F85E200A6892062FD453E8002F72
:109EA80022F4807243E800210029F7D103F1080267
:109EB80052E8002F22F0010203F1080040E80021D7
:109EC8000029F3D103F1080252E8002F22F04002E2
:109ED80003F1080040E800210029F3D12022C4F84A
:109EE8008C20E16653E8002F22F0100243E800219D
:109EF8000029F7D1D4F88000FDF71AFD0223236763
:109F0800B4F85E30B4F85C10C91A89B22046FFF77D
:109F1800FFFE9DE7B4F85E20B4F85E00B4F85C106C
:109F280080B292B2002893D0891A89B200298FD0C2
:109F380053E8002F22F4907243E800200028F7D15C
:109F4800314D03F1080252E8002F2A4003F10806B8
:109F580046E800200028F4D12022C4F88C2060674D
:109F6800E06653E8002F22F0100243E800200028A2
:109F7800F7D102232367C9E7CF0209D56E0207D5B7
:109F88004FF4801220461A62BDE8F04100F0A0BDEF
:109F980008060BD502F0800005F40005284305D01B
:109FA800A36F002B3FF454AF2046CCE64F0611D5E3
:109FB80056060FD553E8002F22F0400243E800214F
:109FC8000029F7D12023C4F88830A1672046F9F783
:109FD8003DF83DE70D0206D5500004D52046BDE802
:109FE800F04100F077BDCB017FF532AF002ABFF614
:109FF8002FAF2046BDE8F04100F06BBD0100001016
:10A0080020010004059D0008FEFFFFEFD0F88C201A
:10A01800B0F86010222A08B5036855D15B6A826DD2
:10A028000B401370836D01338365B0F85E30013BDC
:10A038009BB2A0F85E30B0F85E309BB2002B42D1E4
:10A04800026852E8003F23F4907342E80031036845
:10A058000029F5D103F1080252E8002F22F001028D
:10A0680003F1080C4CE800210029F3D12022C0F8A4
:10A078008C20184A41679342016705D1C26E012AB4
:10A088000ED0F8F7F1FF1EE05A681102F6D553E832
:10A09800002F22F0806243E800210029F7D1EDE784
:10A0A8000022C26653E8002F22F0100243E8002184
:10A0B8000029F7D1DA69B0F85C10D20644BF102243
:10A0C8001A62FFF725FE08BD9A6942F008029A61F4
:10A0D800F9E700BF00800040D0F88C20B0F860108D
:10A0E800222A08B5036852D15A6A1140826D22F8B3
:10A0F800021B8265B0F85E20013A92B2A0F85E2099
:10A10800B0F85E2092B2002A40D153E8002F22F422
:10A11800907243E800210029F7D103F1080252E8C0
:10A12800002F22F0010203F1080C4CE8002100295D
:10A13800F3D12022C0F88C20174A41679342016767
:10A1480005D1C26E012A0ED0F8F78EFF1EE05A68BC
:10A158001102F6D553E8002F22F0806243E800216F
:10A168000029F7D1EDE70022C26653E8002F22F05C
:10A17800100243E800210029F7D1DA69B0F85C1031
:10A18800D20644BF10221A62FFF7C2FD08BD9A69C1
:10A1980042F008029A61F9E7008000402DE9F74F84
:10A1A8000368B0F86080DF691A689D68D0F88C1081
:10A1B80001922229044640F0B480B0F86890DFF894
:10A1C8006CA1DFF86CB10026B9F1000F01D0BB0615
:10A1D80021D4B4F85E309BB2D3B1B4F868209A4267
:10A1E80016D9226802F1080353E8003F23F0805390
:10A1F800083242E8003122680029F2D14D4B6367EA
:10A2080052E8003F43F0200342E800310029F7D12B
:10A2180003B0BDE8F08F2368A26D5B6A03EA080308
:10A228001370A36D0133A365B4F85E30013B9BB294
:10A23800A4F85E302368DF6978072CD0F9070AD5BF
:10A24800019AD20507D501211962D4F8901041F07E
:10A258000101C4F89010B80709D5E90707D502210C
:10A268001962D4F8901041F00401C4F890107A07EC
:10A2780009D5E80707D504211962D4F8903043F0CE
:10A288000203C4F89030D4F8903023B12046FFF789
:10A2980010FDC4F89060B4F85E309BB2002B93D1E7
:10A2A800216851E8003F23F4807341E800302368B7
:10A2B8000028F5D103F1080252E8001F01EA0A015B
:10A2C80042E800100028F5D120215B45C4F88C1025
:10A2D800606720670AD05968090207D553E8001F4C
:10A2E80021F0806143E800100028F7D1E16E0129D0
:10A2F80013D1E66653E8001F21F0100143E800106F
:10A308000028F7D1D969CA0644BF1021196220462E
:10A31800B4F85C10FFF7FCFC56E72046F8F7A4FEFB
:10A3280052E79A6942F008029A6171E7FEFFFFEF6F
:10A338000080004015A000082DE9F74F0368B0F829
:10A348006080DF691A689D68D0F88C100192222914
:10A35800044640F0B280B0F86890DFF868A1DFF8F2
:10A3680068B10026B9F1000F01D0BB0621D4B4F8BA
:10A378005E309BB2D3B1B4F868209A4216D92268ED
:10A3880002F1080353E8003F23F08053083242E803
:10A39800003122680029F2D14C4B636752E8003F34
:10A3A80043F0200342E800310029F7D103B0BDE8AB
:10A3B800F08F2368A26D596A08EA010122F8021B8E
:10A3C800A265B4F85E20013A92B2A4F85E20DF6973
:10A3D80078072CD0F9070AD5019AD20507D50121AB
:10A3E8001962D4F8901041F00101C4F89010B80730
:10A3F80009D5E90707D502211962D4F8901041F070
:10A408000401C4F890107A0709D5E80707D5042194
:10A418001962D4F8903043F00203C4F89030D4F8AD
:10A42800903023B12046FFF744FCC4F89060B4F89C
:10A438005E309BB2002B95D1216851E8003F23F490
:10A44800807341E8003023680028F5D103F1080241
:10A4580052E8001F01EA0A0142E800100028F5D17D
:10A4680020215B45C4F88C10606720670AD05968C2
:10A47800090207D553E8001F21F0806143E8001066
:10A488000028F7D1E16E012913D1E66653E8001FD1
:10A4980021F0100143E800100028F7D1D969CA0655
:10A4A80044BF102119622046B4F85C10FFF730FC55
:10A4B80058E72046F8F7D8FD54E79A6942F00802B1
:10A4C8009A6173E7FEFFFFEF00800040E1A00008FB
:10A4D80038B5044603682169A2681D68C0690A4343
:10A4E80061690A437D49024329400A431A605A6850
:10A4F800E16822F440520A435A60794AA1699342BA
:10A508001CBF226A11439A6822F06E4222F430621C
:10A518000A439A60DA6A616A22F00F020A43DA6231
:10A52800704A93421CD14FF0B043D3F8883003F0FF
:10A53800030343F44033A3F54033013B022B00F2FD
:10A54800C780694A9B5CB0F5004F40F08980082BB2
:10A5580024D8DFE803F061C0832380232323650028
:10A56800624A934209D14FF0B043614AD3F8883028
:10A5780003F00C0343F44023E4E7594A93420DD116
:10A588004FF0B043D3F8883003F44063B3F5006F5D
:10A598001AD005D853B1B3F5806F12D0012009E065
:10A5A800B3F5406FFAD14FF400400EE0FEF7D2FC4D
:10A5B80058B900204FF00113A3660023C4E91D33E6
:10A5C80038BDFEF7CFF8F3E74A4865684A4B626A38
:10A5D80005EB450133F81220B0FBF2F39942DDD8C0
:10A5E800B3EB053FDAD800231946F7F78DFA0902CD
:10A5F80041EA10616B080002C0182A464FF00003B8
:10A6080041F10001F7F780FA3C4BA0F540729A42FD
:10A61800C4D82368D860CCE7FEF79CFC0028C8D0D3
:10A628006168354B626A33F81220B0FBF2F24B08CE
:10A6380003EB42034FF6EF72B3FBF1F3A3F1100102
:10A648009142ABD823F00F02216892B2C3F34203C0
:10A658001343CB60ADE7FEF785F8DFE72548DFE772
:10A66800082B9BD801A252F823F000BFBDA6000812
:10A67800C9A60008D5A60008A5A50008CFA6000809
:10A68800A5A50008A5A50008A5A5000899A6000885
:10A698004FF400406368616A174A32F81120B0FB32
:10A6A800F2F000EB5300B0FBF3F04FF6EF73A0F1BC
:10A6B8001002ACE7FEF74EFC00283FF47AAFE9E75A
:10A6C800FEF758FCF8E7FEF74DF8F5E70948E1E72B
:10A6D800B0F5004FF4D1FEF74DFC9FE7F369FFCFCB
:10A6E8000080004000380140344201080044004026
:10A6F8003742F5070024F40044420108FFFC0F002C
:10A70800836ADA0710B506D50168C46A4A6822F474
:10A71800003222434A609C0706D50168046B4A68E8
:10A7280022F4803222434A60590706D50168446BF7
:10A738004A6822F4802222434A601A0706D5016833
:10A74800846B4A6822F4004222434A60DC0606D53C
:10A758000168C46B8A6822F4805222438A60990691
:10A7680006D50168046C8A6822F4005222438A6084
:10A778005A060FD50168446C4A6822F480122243B5
:10A78800B4F5801F4A6005D14A68846C22F4C0027F
:10A7980022434A601B0606D50268C16C536823F43D
:10A7A80000230B43536010BD2DE9F041DDF81880FC
:10A7B80004460E4615461F462268D36936EA030347
:10A7C8000CBF01230023AB4201D0002027E0B8F1E1
:10A7D800FF3FF2D0F8F790F9C01B4045206802D837
:10A7E800B8F1000F1DD150E8003F23F4D07340E8C2
:10A7F8000032002AF7D100F1080353E8003F23F0A4
:10A80800010300F1080141E80032002AF3D12023B6
:10A81800C4F88830C4F88C3084F884200320BDE85C
:10A82800F08103685A07C7D5C3691B05C4D54FF41F
:10A838000063036250E8003F23F4D07340E800321D
:10A84800002AF7D100F1080353E8003F23F0010381
:10A8580000F1080141E80032002AF3D12023C4F8AE
:10A868008830C4F88C30C4F89030D5E773B5044606
:10A878000026C0F89060F8F73FF923681B681A07AC
:10A88800054619D423681B685B070AD56FF07E4319
:10A89800009300222B464FF480012046FFF784FFE7
:10A8A800B0B900202023C4F8883084F88400C4F8A4
:10A8B8008C30E06620670CE06FF07E4300933246F0
:10A8C80003464FF400112046FFF76EFF0028D9D049
:10A8D800032002B070BD10B5044650B3D0F88830DC
:10A8E8001BB980F88430F8F7BDFA22682423C4F82D
:10A8F8008830136823F0010313602046FFF7E8FD52
:10A90800012816D0A36A13B12046FFF7F9FE236881
:10A918005A6822F490425A609A6822F02A029A6091
:10A928001A6842F0010220461A60BDE81040FFF79D
:10A938009DBF012010BD000030B581658168A0F879
:10A948005C200023B1F5805FA0F85E20436735D115
:10A958000369002B40F2FF1318BFFF23A0F86030F3
:10A968000023C0F890302223C0F88C30016801F130
:10A97800080353E8003F43F00103083141E800347D
:10A988000368002CF2D1456E84680169B5F1005F57
:10A9980034D1B0F86850954230D8B4F5805F1DD1F5
:10A9A800254A264C002918BF22464267C1B153E800
:10A9B800002F42F4807243E80021F7E729B90369C0
:10A9C800002B14BF7F23FF23C8E7B1F1805FC5D1F7
:10A9D8000369002B0CBF7F233F23BFE7174AE4E737
:10A9E80003F1080252E8002F42F0805203F10800F8
:10A9F80040E800210029F3D1002030BDB4F5805F84
:10AA08000FD10F4A0F4C002918BF2246426751B197
:10AA180053E8002F42F4907243E800210029F7D14F
:10AA2800EAE7084AF2E753E8002F42F0200243E839
:10AA380000210029F7D1DFE741A30008A5A10008FC
:10AA4800E1A0000815A00008D0F88C30202B30B405
:10AA580015D1B9B1B2B100230468C3660A4B9C4250
:10AA68000AD063681B0207D554E8003F43F08063AF
:10AA780044E80035002DF7D130BCFFF75DBF022058
:10AA880030BC70470120FBE700800040436E30B5C2
:10AA98002BB90123A0F86A30A0F8683030BD0368EC
:10AAA800094D9A689968094C490FC2F342626B5C78
:10AAB800615CDB00B3FBF1F3A0F86A30AB5CA25C2D
:10AAC800DB00B3FBF2F3E7E7644201085C420108EC
:10AAD8007047704770471FB504AB03E9060090F84C
:10AAE8008430012B04463AD0012380F88430242393
:10AAF800C0F8883003681A6822F001021A609A6860
:10AB080022F440120A439A6071B95A68BDF80C00E1
:10AB18009DF80E1022F0100202435A605A6822F083
:10AB28007F4242EA01625A601A6842F001021A60E2
:10AB3800F7F7E2FF6FF07E42034600924FF4800180
:10AB480000222046FFF730FE38B92023C4F88830A9
:10AB5800002384F8843004B010BD0320F8E70220F5
:10AB6800F9E790F88430012B0FD0012380F8843066
:10AB7800016851E8002F42F0020241E80023002B4F
:10AB8800F6D180F88430184670470220704710B517
:10AB980090F88430012B044617D02423C0F888305D
:10ABA80003681A68196821F00101196042F000521F
:10ABB8004FF0005141661A60FFF768FF2023C0F884
:10ABC8008830002084F8840010BD0220FCE770B5AE
:10ABD80090F88430012B044617D005682423C0F868
:10ABE80088302E682B6823F001032B60AB6823F0B4
:10ABF80060431943A960FFF749FF20232E60C0F87E
:10AC08008830002084F8840070BD0220FCE770B50D
:10AC180090F88430012B044617D005682423C0F827
:10AC280088302E682B6823F001032B60AB6823F073
:10AC380060631943A960FFF729FF20232E60C0F83D
:10AC48008830002084F8840070BD0220FCE70000F2
:10AC580038B5084D052455F8043B2BB9013C14F0D0
:10AC6800FF04F8D1204638BDDB6898470028F5D0A6
:10AC7800F9E700BF04100020034BD870034B1B6892
:10AC88001B6C03B1184770471810002000100020F3
:10AC9800034B1874034B1B685B6C03B11847704770
:10ACA8001810002000100020F0B5314D314B95F9F7
:10ACB8000420314E91B00C46012795F905108DF806
:10ACC800047002288DF809208DF80A1010D18DF82B
:10ACD8000800D8711C7202F09FFD337803B114B1DB
:10ACE80001A803F003FA254B059A1A6011B0F0BDCC
:10ACF80059714FF480711A71D9801C7233788DF8AC
:10AD0800087053BB1F2306A88DF81C208DF8183037
:10AD180002F064FF20238DF8183006A82B798DF8EF
:10AD28001C3002F05BFF22238DF8183006A86B79DF
:10AD38008DF81C3002F052FF21238DF8183006A838
:10AD48006B798DF81C3002F049FF29238DF81830F3
:10AD580006A80B4B079302F041FF02F05DFD0123AB
:10AD680006A88DF818308DF81C3002F037FFB4E7CC
:10AD78001810002030080020F40F0020F80F0020E1
:10AD8800000400017FB5092301A88DF8043003F001
:10AD9800ADF90038044B059A1A6018BF01204042EB
:10ADA80007B05DF804FB00BFF80F002070B504463B
:10ADB8000B46134962784A700020A2780A7208701C
:10ADC8001A884A729A788A72DB780B746368CB6047
:10ADD8000C4B1B68DA6A2AB1237803F0FB030A2BB1
:10ADE80000D09047084E052556F8043B1BB15B6A16
:10ADF8000BB120469847013D15F0FF05F4D170BD11
:10AE08003C080020001000200410002070B5044603
:10AE180010480123037063784370A3788372E36852
:10AE2800C360E378037623694376237943720A4B38
:10AE38001B689B6A03B19847084E052556F8043BE2
:10AE48001BB19B690BB120469847013D15F0FF05E2
:10AE5800F4D170BD5008002000100020041000201C
:10AE6800014B1868704700BFF80F002000B58BB081
:10AE7800012368468DF8003002F088FD38B99DF846
:10AE88000400003818BF01200BB05DF804FB002057
:10AE9800FAE7000008B501F073FE48B9FFF7E6FFCE
:10AEA800012806D0054BD879197AFFF7FDFE012055
:10AEB80008BDBDE80840FFF7CBBE00BF3008002042
:10AEC8002DE9F04186B005460E46174601F058FEBA
:10AED80000287FD101F06CFE044640B9FFF7C6FF99
:10AEE800012807D03D4B197AD879FFF7DDFE6FF0BE
:10AEF800020462E0DFF8E88088F80860003E18BFC6
:10AF080001268DF80460374E687833798DF8123051
:10AF1800694602F0D9FC00283ED08DF8044003941D
:10AF2800ADF810406FF0060495E803002E4B83E857
:10AF38000300337988F80A30394601A803F0DAF9B2
:10AF48002A4B059A1A60112841D801A353F820F01A
:10AF5800B7AF0008DDAF0008D7AF0008D7AF0008CB
:10AF6800D7AF0008D7AF0008D7AF0008F7AE000882
:10AF7800D7AF0008D7AF0008D7AF0008D1AF000897
:10AF8800D7AF0008D7AF0008DDAF0008DDAF000875
:10AF9800DDAF0008CBAF00082B788DF808306B7850
:10AFA800ADF810306B6803934FF0FF34BCE7104BDB
:10AFB80000221A70E31D18BF1446204606B0BDE8EB
:10AFC800F0816FF00404F8E76FF00504F5E74FF03F
:10AFD800FF34F2E76FF00104EFE700BF300800200C
:10AFE800500800201810002060080020F80F0020EA
:10AFF800FC0F002037B501F0E5FD144D052455F888
:10B00800043B5BB11B694BB155F8043C9B682BB101
:10B01800984718B155F8043C1B699847013C14F04F
:10B02800FF04ECD1FFF714FE68B9094D2B7853B132
:10B03800084BADF80040D978019422466846FFF7DE
:10B048003FFF00B92C7003B030BD00BF04100020D2
:10B05800FC0F00201810002030B58BB0054601F019
:10B068008FFD0446002839D1FFF700FF012838D1A9
:10B0780068468DF8004002F089FC10B14FF0FF30AF
:10B0880004E09DF80430AB4202D100200BB030BD83
:10B09800012DF3D0022D11D0002DF7D1002BF4D0C3
:10B0A80068468DF8045002F099FD0028E6D10E4B51
:10B0B8001B681B6B002BE8D09847E6E7002BDDD117
:10B0C80068468DF8045002F089FD0028D6D1064B59
:10B0D8001B681B6B002BD8D02846EDE76FF00100EA
:10B0E800D4E76FF00200D1E70010002010B5044645
:10B0F8008AB018B94FF0FF300AB010BD0023684677
:10B108008DF8003002F042FC0028F3D19DF804309D
:10B118002370F1E77FB500220B4620498DF8072000
:10B1280001220A7042784A700446002A33D1027913
:10B138000A721A884A729A788A72DB780B740369E1
:10B14800CB60C378164D8DF80830037B8DF8093035
:10B15800836803932B68DB6A0BB102A898472B68B6
:10B168009B6B13B1227E02B198470E4E052556F807
:10B17800043B1BB1DB690BB120469847013D15F034
:10B18800FF05F4D10DF10700FFF7B0FF637913B1A4
:10B19800054B01221A7004B070BD00BF3C080020A6
:10B1A8000010002004100020FC0F002010B50446F9
:10B1B8008AB018B94FF0FF300AB010BD2023684696
:10B1C8008DF8003002F0E2FB0028F3D1024A9DF925
:10B1D800043023701371EFE71810002000B58BB00E
:10B1E8002323019068468DF8003002F0F7FC003800
:10B1F80018BF012040420BB05DF804FB70B5654CE8
:10B2080001468EB01822204606F0FEF8624B002256
:10B218001A70F8F729FF23784068012202FA03F12F
:10B22800014004D15D4B084608F0E4F8FEE75C49AC
:10B238005C481A4602F032F918B14FF0FF300EB0F0
:10B2480070BD272304A88DF8103002F0C7FC564EB5
:10B25800564D002870D1012333702B68DB690BB180
:10B2680000209847272304A88DF8103002F08EFBA1
:10B27800059B93F84820227093F8182193F81A3107
:10B288006270A370464BD3E9020105F0AFFF054693
:10B298000028D2D1464E062304A88DF8103002F0BB
:10B2A80075FB059B736104A802F098FC022304A8AF
:10B2B8008DF81030059602F069FB0836032304A8C0
:10B2C8008DF81030059602F061FB0F2606F052F853
:10B2D800012304A88DF814308DF8106002F07EFC6C
:10B2E80010230DEB03008DF810308DF8145002F088
:10B2F80075FC04238DF8103004A8A3788DF8143059
:10B3080002F06CFC3A238DF8103004A863690593A9
:10B3180002F064FC02A920788DF8086004F0E8F8CF
:10B32800003818BF0120E0711420FFF757FFE079BB
:10B3380003F0A4F9284682E728238DF810302B68FB
:10B348001B6943B104A802F021FB2B6805981B690F
:10B3580040F2C4519847272304A88DF8103002F012
:10B368003DFC50B9012304A88DF8103002F00EFB03
:10B378009DF81430002B7FF46EAF3378002B7FF4E8
:10B388006CAF052204A88DF81020059302F026FC66
:10B3980078E700BF18100020FC0F00206C4201085D
:10B3A8004010002058100020F40F0020001000204A
:10B3B800DC0F002037B500230D4601930446D0B9B1
:10B3C80000F0A8FB0190019BD3B10F4A42F824304A
:10B3D8000E4A9A620E4A1268916B1963916C59630E
:10B3E80092690C49D9625A6128465B680A49F22277
:10B3F8009847002006E001A900F092FB0028E2D05F
:10B408004FF0FF3003B030BD04100020B1AC00088D
:10B41800001000208DAD0008E80E0020194B07B57C
:10B428001860194B194A1A60194A5A60194A9A60E1
:10B43800194ADA60194B02681A6042685A608268D1
:10B448009A60C268DA60164A1A6182695A61154BB5
:10B45800C26B5A60144A019119609A601946134ADE
:10B46800DA600020FFF7A6FF48B901A800F056FBF4
:10B47800003818BF0120404203B05DF804FB4FF0CC
:10B48800FF30F9E7001000205810002015AE000822
:10B498001DB1000835B50008B5AD00084010002002
:10B4A800A9F400083010002081AC000899AC00080D
:10B4B80051B118B1012804D000207047044B0B602B
:10B4C8007047044B0B60F7E74FF0FF30704700BF41
:10B4D800000400010100010208B503F0EBF80028A0
:10B4E80014BF6FF00100002008BD08B502F0BCF9D8
:10B4F800002814BF6FF00100002008BD10B50446F5
:10B508008AB018B94FF0FF300AB010BD2123684641
:10B518008DF8003002F03AFA0028F3D1024A9DF97A
:10B52800043023705371EFE7181000202DE9F04123
:10B538002E4D2F4F00232B7043786B703B689B6A0E
:10B548008AB004460BB128469847DFF8A88005263C
:10B5580058F8043B1BB11B6A0BB120469847013EC3
:10B5680016F0FF06F4D12378052B2FD00B2B35D0FE
:10B57800012B25D1204C062368468DF8003002F0B7
:10B5880005FA0199E07905F077FE10B91B4B019A8D
:10B598005A611B48FFF70AFE1A48FFF7AFFF6B789E
:10B5A8008BB9A371184B5878FFF756FD3B685B6A57
:10B5B8000BB1114898476B7813B9E07905F0ECFEA8
:10B5C8000AB0BDE8F081FF23A371EFE70F4B01221A
:10B5D8005A74227A9A74627ADA74F1E76378002BE3
:10B5E800EED00AB0BDE8F041FFF7CCBB5008002010
:10B5F800001000200410002030080020DC0F00207C
:10B608003408002035080020181000203C080020CD
:10B6180030B58BB0FFF769FF0446F0B903F048FF77
:10B62800831C1DD0F8B9134D2B685B69DBB1272348
:10B6380068468DF8003002F0A9F92B6801985B691B
:10B648004FF4B961984703F045FF78B92CB9094B15
:10B658001B68DB690BB10120984720460BB030BD51
:10B668006FF00704EFE74FF0FF34ECE74FF0FF34DB
:10B67800F3E700BF00100020014B1878704700BFA7
:10B688006C100020014B5878704700BF6C100020E8
:10B6980070470000044B9A7A0AB101225A70034B92
:10B6A8005B6903B1184770476C1000206C080020D4
:10B6B80073B5224C6378002B33D008F085F966689F
:10B6C8000546FFF7CDFB0644AE4214D2A37A93B1E8
:10B6D800E0228DF800208DF80130217AE36801938B
:10B6E80001226846FFF7ECFB08B1073010D10023B0
:10B6F8006370A372656094F83430EBB1002384F86A
:10B7080034300F4B5B6BBBB102B0BDE870401847DB
:10B7180040F2DC510B4808F023FA0A4808F0E6F931
:10B72800E8E794F83520002AE5D094F8360084F844
:10B738003530FFF791FCDEE702B070BD6C100020D9
:10B748006C080020A410002037B5104D104CC8B16B
:10B75800C1B10123627200222860E16023700D48A4
:10B768000D4B00924FF0FF3108F014F900250B48FB
:10B7780025822022294605F05BFE6570A574A58602
:10B7880003B030BD00232B602370EFE76810002062
:10B798006C100020A41000209DB600088010002026
:10B7A8002DE9F0478E4C23788CB0002B56D0C27808
:10B7B8000AB9837B13B1238A01332382437B002B8D
:10B7C8004CD0E02A4AD10023A372876897F80080FA
:10B7D800B8F1220F27D8B8F1220F30D8DFE818F0D7
:10B7E8004100FB0052005A0061006E0075008E0097
:10B7F8009D00B400C7002F002F002F002F002F003E
:10B808002F002F002F002F002F002F002F002F00B8
:10B818002F002F002F002F002F002F002F002F00A8
:10B82800C900D000D400B8F17E0F00F0CC80B8F188
:10B838007F0F00F0DF80B8F17D0F00F0AB80A57AB4
:10B84800002D00F05B81674C637A3BB94FF47A7145
:10B85800204608F085F9204608F048F90CB0BDE804
:10B86800F087E36801220021A2721970A37AE168C7
:10B878009818A0720620C854A37AE1689818A07294
:10B88800CA54DCE7584B9B6A002BD8D00121022010
:10B898009847D4E77B7884F83630012384F835302C
:10B8A800CDE704238DF804307B78003B18BF0123D3
:10B8B80001A88DF8083002F091F9C0E778780038CF
:10B8C80018BF012002F0DAFEB9E7484E0FCE01ADED
:10B8D8000FC50FCE0FC596E8070085E807007B78EF
:10B8E8000A2BACD8424A12685268002AA7D00CA981
:10B8F80001EB830353F82C0C9047A0E77878431E9C
:10B90800012B9CD83A4B01381B6818BF01202072C4
:10B918009B68002B93D0984791E7E26801230821A0
:10B92800A3721170627A057BA17AAA4228BF2A46BF
:10B93800934284D285685A1CEB5CE56801334E1C3F
:10B94800A6726B54D3B2EDE7E3680122A272092212
:10B958001A70A37AE268218A581CA072D154A27A7C
:10B96800238AE1681B0A501CA0728B5467E7238264
:10B9780065E705238DF8043001A802F0B7FB5EE700
:10B98800194BDB6A98475AE7194B78781B6860753A
:10B99800DB68BEE7037B072B7FF451AF06238DF8E6
:10B9A8000430B7F80130ADF808307B793A791B04D8
:10B9B80043EA0223FA781343642253430393BB797F
:10B9C8008DF81030D8E73B2201A88DF804208DF8B7
:10B9D800083002F003F9012384F834302FE700BF60
:10B9E8006C100020A41000206C0800203C400108C6
:10B9F800681000202A2301A88DF8043001F0C6FF42
:10BA080094F80A90E6689DF808009DF809509DF89A
:10BA18000A709DF80BC09DF80D309DF80E209DF81A
:10BA28000F109DF80CE009F1010A84F80AA006F845
:10BA38000980354E94F80A903668D4F80C8009F1DC
:10BA4800010A84F80AA096F803A008F809A094F857
:10BA58000A90D4F80C8009F1010A84F80AA096F833
:10BA680002A008F809A094F80A90D4F80C8009F10B
:10BA7800010A84F80AA096F801A008F809A094F829
:10BA88000A9009F1010A84F80AA096F80080E6688D
:10BA980006F8098094F80A80E66808F1010984F834
:10BAA8000A9006F808C094F80AC0E6680CF1010884
:10BAB80084F80A8006F80C70A77AE66807F1010C8A
:10BAC80084F80AC0F555A57AE6686F1CA772705508
:10BAD800A07AE568461CA6722954A17AE0684D1C34
:10BAE800A5724254A27AE168501CA0728B54A37AC2
:10BAF800E268591CA17202F803E0A0E6034807F0C7
:10BB0800A7FF6570AAE600BF68100020A4100020F7
:10BB180070470000004870476C08002000207047FC
:10BB28004FF0FF3070470000044B054A93F8183176
:10BB3800022B18BF062382F8903470478016002025
:10BB4800481C0020034BD3F8483313B15B6903B199
:10BB580018477047481C0020034A137843F0040331
:10BB68001370FFF7EFBF00BF441C00201FB50A4B3E
:10BB78008DF8090093F87C208DF80A2093F88C2022
:10BB880093F848000D3202A98DF8082003F0B0FCA4
:10BB9800C0B205B05DF804FB8016002010B5074C54
:10BBA80004F5806007F054FF94F81A3413B10123A8
:10BBB80084F81934BDE81040FFF7C4BF481C0020C2
:10BBC80010B50C4CD4F8403343F08003C4F840332C
:10BBD80094F81A3413B10020FFF7E0FF94F8913479
:10BBE80023F0120343F0120384F89134BDE81040A7
:10BBF800FFF79ABF481C00202DE9F041DFF8AC8020
:10BC080098F81831022B06460D4602D0284BDB6AFD
:10BC1800984702F0E9FD044628B1022002F0DAFD57
:10BC2800002002F0DCFD98F81831012B17D102F042
:10BC3800DDFD074630B1002002F0CDFD002002F006
:10BC4800CFFD3C4602F0D4FD48B1002002F0C4FD0F
:10BC5800002002F0C6FDBDE8F041FFF765BF002CEB
:10BC6800F9D1144C94F8902494F81A34BAB90BB159
:10BC780084F84164304602F065FFD8F82C0007F0DC
:10BC8800ADFED4F8B4339842E5D30B4807F0E0FE94
:10BC980094F8913443F0100384F89134DBE70BB146
:10BCA80084F84154284602F04DFFF1E78016002041
:10BCB800F0490108481C0020E01F002073B5164C0D
:10BCC800164D04F57A76EB6C95F8502095F97810B6
:10BCD80095F84800009603F031FC95F8303184F867
:10BCE800FC3395F8480040F2012304F2244231461F
:10BCF800A4F8FA3303F02EFC58B194F8243484F8ED
:10BD08006A34074B00205B6B984794F8FB3384F840
:10BD1800903402B070BD00BF481C0020801600207F
:10BD2800F0490108074A10B5137843F0020313706D
:10BD3800FFF708FFBDE81040034B01220021022055
:10BD480007F058BB441C0020B5420108074A10B54B
:10BD5800137843F008031370FFF7F4FEBDE81040B2
:10BD6800034B01220021022007F044BB441C0020A1
:10BD7800C54201082DE9F0410F4616461D4680468A
:10BD880007F022FE0B4A0C4C1378278123F011038D
:10BD980043F011031370C4E9000866812573FFF7A7
:10BDA800D1FEBDE8F041054B01220021022007F039
:10BDB80021BB00BF441C0020F4210020D54201080B
:10BDC80013B507F001FE0D4B6C461860204607F0CE
:10BDD8004FFD94E803000A4A0A4B83E803001378EE
:10BDE80043F020031370FFF7ADFE074B012200213B
:10BDF800022002B0BDE8104007F0FCBA042200207F
:10BE0800441C0020801F0020E2420108F8B5334D91
:10BE180095F81841012C06464BD0022C51D064B934
:10BE280038B9D5E91B0105F1740383E803002046FE
:10BE3800F8BD01283DD0022801D00324F7E7284F98
:10BE480085F8180107F5747EBEE80F0007F57A7CBF
:10BE5800ACE80F009EE8030095F8E9308CE8030091
:10BE680087F8FB63E3B195F80031022B18D1D5F8B8
:10BE780004316B67C7F8EC3395F87D3095F80821E5
:10BE880087F8F83395F88C3085F8782087F8F933F7
:10BE980097F81B2487F8E82340F20133A7F8FA3310
:10BEA800002387F81A340F4BDB6A9847FFF706FF21
:10BEB800BDE702F0A4FC04460028B8D185F8186153
:10BEC800B5E70028B9D1064B85F81801062283F892
:10BED8009024044BDB6A98473446A8E78016002074
:10BEE800481C0020F04901082DE9F04192B00646AF
:10BEF80002F07AFC002840F05981AD4D95F81831D0
:10BF0800012B09D02B6BAB4C93B194F80431BBB126
:10BF1800042B6FD0032003E002F068FC18B10F2057
:10BF280012B0BDE8F08102F063FC0028EAD0F6E721
:10BF3800B5F82031D4F81C24013B53432B63E4E7C4
:10BF48009D4803F00CFA002840F02C8194F80C313D
:10BF580023802B6B0C930DF1180895F839308DF868
:10BF68003830404695F81C318DF83A3007F0A6FC79
:10BF7800D5F82831009302AF98E80600D5F82431A7
:10BF8800384607F032FC97E803000FAB83E803005C
:10BF9800EB6A0D9300238DF844302388ADF84630C2
:10BFA80095F8303101228DF839201BB98DF84420DD
:10BFB8008DF83930814B0093814B95F84800A3F1F7
:10BFC80079020CA903F009FBC0B10B28A8D1D4F859
:10BFD800941499B1002EA3D0D4F84033794843F093
:10BFE8002003C4F8403307F0BBFD764807F07EFD18
:10BFF800002095E7704803F0E6F9A4E795F8487043
:10C0080095F9693095F9392095F87D106E4E3846C6
:10C0180003F0F0FA009641B2EB6C95F850203846E0
:10C02800183603F08BFA0096EB6C95F8502095F9CA
:10C03800701095F8480003F081FAD4F8C413AB6D7A
:10C04800D4F8DC230B44C4F8B033EB6D1344C4F8C4
:10C05800B43394F80431042B07D02B6E0B44C4F886
:10C06800B0336B6E1344C4F8B4330023089395F8C7
:10C07800303183B108A802F095FC00284ED195F91B
:10C08800390094F837629DF82070FFF76FFD3E4441
:10C0980080B2B04240D300238DF8133095F8393080
:10C0A8008DF8213095F838308DF82230D5F8803069
:10C0B8000993D5F884300A932388ADF82C3095F885
:10C0C800303194F81B648DF82E3095F848003F4BBA
:10C0D8008DF820600DF1130208A903F043FA01233B
:10C0E80084F8413495F8393084F842349DF8133097
:10C0F80084F84334D4F81C34C4F85064C4F8483481
:10C10800C4F8583402F076FB50B1D4F81C0402F09D
:10C1180083FB28B1102003E7082001E71320FFE67E
:10C1280095F81831012B01D102F078FB02F065FB7C
:10C138000023059394F8043195F9395094F81B6459
:10C148009BB1042B7FF4E6AE05A802F067FE58BB4E
:10C1580094F8183413B1059B013B0593164B0598C9
:10C168003246E9B202F0C0FE02E0134802F090FE47
:10C17800C0B9D4F8403394F80C11218043F002037D
:10C18800C4F8403394F8183411480133DBB284F80A
:10C19800183484F845340F4B00259B6AC4F898542A
:10C1A800984725E71120BBE61220B9E60E20B7E62E
:10C1B80080160020481C0020501D0020B0160020CA
:10C1C800DC200020B01F0020002000206420002078
:10C1D8004A1C0020F0490108F0B5504C504EB4F804
:10C1E800DC202287D4E92D0194F8B12084F8692055
:10C1F80004F16C0282E80300D4E92F0104F174020F
:10C2080082E80300B4F8C420A4F87C2091B0D4F8E4
:10C21800CC20D4F8C810C4F884200025D4F8D02045
:10C22800C4F888200123A4F82031C4F8801084F8C9
:10C238003051A56284F81B5184F83A5084F81D5196
:10C2480084F81E51C4F83451C6F89854A6F8185406
:10C2580086F81A54A4F838518DF8183004F5097383
:10C26800039304F50A7394F84800A4F8465104931C
:10C2780003A92C4B84F84551C4E94F55059303F0A5
:10C2880045F9E36EC6F8D43394F87D3086F8E03388
:10C2980094F88C3086F8E1334FF48073A6F8E233D3
:10C2A80086F8D05394F8303186F8E43306F574777D
:10C2B8000FCF06F57A740FC497E8030040F2012304
:10C2C80084E80300A6F8FA33D6F8483386F81B54F6
:10C2D800CDE901551BB15A685B6901920293124B73
:10C2E8000793A3F148020892A3F1140209920F4A96
:10C2F8000B9229330A93A2F19C030C93A2F19803A1
:10C308000D93131D0E9301A902F14C0307A802F522
:10C3180099620F9302F05DFA11B0F0BD801600200B
:10C32800481C002064210020B02000206417002051
:10C33800F8B50D4F0D4C0E4E0D4607F089FB3B6BC3
:10C34800984796F8480004F22442294603F002F977
:10C3580048B194F8243484F86A34706D7B6B98473C
:10C36800EB7C84F89034F8BDF0490108481C0020A3
:10C37800801600200F4890F81B3480F8B8330E4B15
:10C3880093F8692080F8BB2393F87D2080F8C823B0
:10C3980093F88C2080F8C92393F8303180F8CC3397
:10C3A8000022A0F8CA2300F56E7100F56070FFF74F
:10C3B800BFBF00BF481C002080160020114890F81D
:10C3C8009034EBB190F81B3480F8D0330E4BDA6E12
:10C3D800C0F8D42393F87D2080F8E02393F88C20CC
:10C3E80080F8E12393F8303180F8E4334FF4807219
:10C3F800A0F8E22300F5747100F56670FFF798BFA6
:10C40800704700BF481C00208016002070B5344CCF
:10C418002421204605F00EF8636A984218BF60622E
:10C428004FF01C012F4814BF0125002505F002F824
:10C43800636C984218BF60644FF480712A4818BF33
:10C4480045F0020504F0F6FFD4F84831984218BFC9
:10C45800C4F848014FF0D401244818BF45F004053A
:10C4680004F0E8FFD4F82032984218BFC4F820023C
:10C478004FF000011E4818BF45F0080504F0DAFF28
:10C48800D4F82432984218BFC4F824024FF46071DB
:10C49800184818BF45F0100504F0CCFFD4F8A835AB
:10C4A800984218BFC4F8A8054FF01401124818BFE5
:10C4B80045F0200504F0BEFFD4F8C03598420F4B74
:10C4C80018BFC4F8C005D3F8483318BF45F0400575
:10C4D8002BB11B691BB12846BDE87040184770BDD9
:10C4E80080160020A8160020C8160020CC170020AF
:10C4F800A4180020A81800202C1C0020481C00208C
:10C508002DE9F04F91B04FF00008012B05460F467A
:10C5180002928DF81580ADF8188003D8C84EC14630
:10C52800B94502D311B0BDE8F08F15F8090002F043
:10C5380077FA4844B842F5DC15F8093009F10104E6
:10C54800023BE4B2112BEDD801A252F823F000BF50
:10C55800A1C50008D3C50008D3C60008FDC6000859
:10C5680085C70008ADC700081FC8000851C80008E3
:10C57800CDC800082DC500082DC500082BC9000826
:10C588002DC500082DC50008E9C9000811CA000812
:10C5980055CA000893CA0008052002F0EDFA90B1C8
:10C5A8000521002002F0ACFA2A5DA64B09F103042C
:10C5B80009F102095FFA89F983F85C2415F8092062
:10C5C80083F85D24E4B2A146AAE700238DF816306B
:10C5D8008DF817308DF81C308DF82030B8F1000F29
:10C5E8006CD14FF0050896F87C208DF83920631E31
:10C5F80096F839208DF83B202B4496F838200D9377
:10C608008DF83C2096F81A3196F868208DF83D2070
:10C61800D6F82C218DF83A300C9273B37B1C1B1B77
:10C62800DBB28DF8383008AB019307AB009396F86E
:10C6380048000DF117030DF116020CA902F09EFF38
:10C648008DF8150000F00700072813D196F9392056
:10C658009DF9163086F839309A429DF8173086F8D9
:10C668003830B8BF01229DF81C30B8BF86F81D21AC
:10C6780086F868304FF0000909E00523D1E7012268
:10C688000DF11501032002F0DBF809F101095FFA49
:10C6980089F29DF82030B3FBF8F19142EFD823449A
:10C6A800DCB2631EDBB29F420DD9EA5C032A9AD042
:10C6B800A74288BF1C464FF0010884E709F1050925
:10C6C8005FFA89F4F7E71C46F5E72B5D012203F0D2
:10C6D8000F0309F1020986F81B3102FA03F35FFA26
:10C6E80089F9A6F82031002206A9042002F0A8F84A
:10C6F8004C4668E707238DF815302B5D96F84800FF
:10C70800C3F3021203F00F038DF8303009F103036D
:10C71800DBB28DF83120EA5C09F10403DBB209F1E0
:10C728000504EB5C09F102095FFA89F91B0443EA85
:10C73800022315F809201343642253430CA90D93CF
:10C7480002F02BFF00F00703072BE4B28DF8150069
:10C758000CD19DF8303086F8703086F878300D9B13
:10C76800F36673679DF8313086F869308DF81800E4
:10C77800012206A9052002F063F824E7314BD3F81B
:10C7880048336BB11B685BB19847029B8DF8180062
:10C7980003F03F038DF81930022206A90620EAE7C4
:10C7A800FF20F2E703238DF815302B5D8DF8243038
:10C7B8000CAB089309F10303DBB209F10604EA5C48
:10C7C80096F8480009F10403DBB208A9EB5C1B04E6
:10C7D80043EA022309F10202D2B209F10509AA5C6F
:10C7E8001343642253435FFA89F90C9300230D9392
:10C7F80015F809308DF8383002F0D5FEC3B200289C
:10C80800E4B28DF81530FFF6DEAE8DF8183001224F
:10C8180006A90720AFE72B5D03F00F03012B4FF4A8
:10C828007A7238BF0123534309F10209B3651344EF
:10C838005FFA89F9F365002206A9082056E700BFC8
:10C8480080160020481C00202B5D96F84800C3F392
:10C8580040128DF81D2007A9C3F3001203F00F033F
:10C868008DF81C208DF81E3002F0A3FE09F1020994
:10C8780001305FFA89F93FF43BAFBDF81C30914AAB
:10C88800A6F87C309DF81E309DF81C40D05CF5F76A
:10C89800BDF80223C6F880000CA996F848008DF868
:10C8A80030308DF8324002F023FE96F93930089086
:10C8B80040B29842B8BF184686F83900002206A947
:10C8C800092013E703238DF815302B5D8DF83030E0
:10C8D80009F10303DBB209F10504EA5C96F84800A4
:10C8E80009F10403DBB209F10209EB5C5FFA89F98B
:10C8F8001B0443EA022315F8092013436422534317
:10C908000CA90D9302F05BFEC3B20028E4B28DF8C7
:10C918001530FFF658AE8DF81830012206A90A2006
:10C9280029E7092002F028F9DFF89CA1002854D053
:10C938000921002002F0E4F80023ADF8263009F1BF
:10C948000203DBB24FF47A71EA5C09F10303DBB24C
:10C958000DF1300BEB5C1B0443EA02232A5D134301
:10C9680009F10402D2B209F1060409F10509AA5C29
:10C978005FFA89F943EA026315F8092003934A43E9
:10C9880012125846ADF8242006F072FF039B03F1FB
:10C99800965303F5A91303F5EC530893DAF83C33DF
:10C9A80000930DF1200999E80600DAF838330AA84F
:10C9B80006F01BFF0B9B00939BE806000A9B48466A
:10C9C80006F0F8FE99E8030006F02AFF01F021FFBF
:10C9D8000123E4B28AF83834F5E58AF83804F2E538
:10C9E8000C2002F0C9F800283FF4EDAD0C2100201E
:10C9F80002F086F8344B93F89034043B012B7FF611
:10CA0800E2AD01F002FFDEE509F10203DBB22A5DC7
:10CA1800E95C09F10303DBB209F10504EB5C09F1F8
:10CA280004095FFA89F91B0415F8090043EA012390
:10CA380013436421594300F00F0001F0E7FEE4B20C
:10CA48008DF81800012206A9112094E60D2002F0A5
:10CA580093F800283FF4B7AD0D21002002F050F8FC
:10CA680009F10203DBB2194AE85C2B5D126809F18F
:10CA7800040409F103095FFA89F943EA002015F86B
:10CA88000910E4B201F0C4FE9DE52A5D09F1020334
:10CA980009F1040409F10309DBB25FFA89F9E95CD9
:10CAA80015F809301B0443EA012313436420584353
:10CAB80001F0B0FEE4B28DF81800012206A9132097
:10CAC80059E600BFEF420108481C0020F42100206D
:10CAD8000E4B93F89124920703D593F88F24012ADB
:10CAE80008D90B4991F81A2122B18A6A501C18BF3B
:10CAF80001328A620022A3F8182483F81A24D3F892
:10CB0800402322F00202C3F840237047481C00204B
:10CB18008016002070B5184C184D04F55A7006F0B0
:10CB280097FFD4F84033D4F89804D5F8906023F0F0
:10CB38002003C4F8403338B106F050FF864203D2D0
:10CB4800002385F83A3070BD0120FFF7CDF90028A1
:10CB5800F9D00B28F7D095F8393084F842340920F9
:10CB680094F8183484F8453484F8410401F0EAFF55
:10CB7800BDE87040FFF7ACBF481C002080160020BD
:10CB8800094BD3F84023012A0AD008490978C90774
:10CB980008D43AB993F89204013818BF01207047B5
:10CBA8000020704701207047481C0020441C0020CA
:10CBB800034BD3F84003431E58425841704700BF07
:10CBC800481C00202DE9F04FA9B0EFF3108272B68F
:10CBD800DFF8F4820021D8F80030C8F8001082F39A
:10CBE8001088BA4C002B00F0E480DAB29B0603925E
:10CBF80064D5B74D95F81831022B02D0B54BDB6AD6
:10CC08009847EFF3108972B6B34F06F0DDFE3E6821
:10CC1800D4F8B013361A3144B04806F0A1FFAF4833
:10CC280006F064FFD4F8B413AD48314406F098FF19
:10CC3800AB4806F05BFF89F3108894F81A34002B90
:10CC480000F06D81152312A995F848008DF8483039
:10CC580002F04EFCD4F8B4130F900144A14806F03A
:10CC68007FFFA04806F042FF3B6894F81B24EB6264
:10CC78000DAF38468DF870201D9306F01FFED5F8CD
:10CC88002831009306AE97E80600D5F824313046DF
:10CC980006F0ABFD96E803001FAB83E80300D4F869
:10CCA8001C341E9395F8303195F84800003B18BFA6
:10CCB80001231CA98DF8713002F023FC039BDF06C9
:10CCC8004BD5834DDFF820A2D5F8E420BAF90A3015
:10CCD800059298F800200493002363F300020A9356
:10CCE80088F8002084F84434049AA4F8223484F89C
:10CCF8002534C4F82834A4F82C3484F82E34C4F825
:10CD0800303484F82034C4F8343484F83834C4F81F
:10CD18003C34704B9AF90C90A4F88C2494F8902425
:10CD2800DB6A84F88E9484F88F24DAF80470BAF8F1
:10CD38000860984794F88F3413B9694806F088FE5C
:10CD48003146384601F04EFD8346002800F0EA805F
:10CD5800049BA4F87E3484F88094039B19071AD5A1
:10CD68005B4B93F81831022B02D05A4BDB6A984779
:10CD78000220FEF7D9FE84F8410401F0E3FE94F89E
:10CD88001A3413B1012384F8193494F8913443F018
:10CD9800100384F89134039B5A0703D50621052014
:10CDA800FEF72AFF039B9B0703D504210320FEF708
:10CDB80023FF01F035FD94F89124D7065FD50023B1
:10CDC80084F89234D4F840331E0644BF23F082031B
:10CDD800C4F8403312F0050F00F0FC820B2001F07C
:10CDE800CBFE002800F0F68294F89134DD0700F1BC
:10CDF800F182580740F10883D4F8403323F0020346
:10CE0800C4F84033D4F8402382BB94F8915415F009
:10CE180001011EBF2B4662F3000384F8913494F895
:10CE280091345E0744BF6FF3820384F89134012381
:10CE380084F8923421B1D4F844332C481B689847BD
:10CE48006D070BD52A4801F0A3FE01F0D1FE28B1E9
:10CE580094F8913443F0040384F8913401F0CEFC43
:10CE680094F891346FF3041384F89134012384F80F
:10CE7800923494F8913443F0200384F8913494F870
:10CE8800913418070AD56FF3C3031A4984F891340B
:10CE9800D4F84433A1F12400DB68984794F891341E
:10CEA80099070AD56FF34103124984F89134D4F8ED
:10CEB8004433A1F16C005B68984794F89034022BD6
:10CEC8001AD1FEF7FBFE17E0441C0020481C002086
:10CED80080160020F049010804220020C81F002005
:10CEE800E01F002048200020F42100208820002096
:10CEF8009C200020D420002094F891349A0640F118
:10CF0800C6826FF3451384F89134D4F84033002B6C
:10CF180040F0BD8229B0BDE8F04FFFF777BA84F83A
:10CF28004134A1E695F81821012A0CD101F05EFCE4
:10CF3800804668B1584601F04EFC584601F050FC56
:10CF4800042384F88F347EB9012384F8213450E116
:10CF580001F04EFC0028F6D0404601F03DFC40466A
:10CF680001F03FFC0523ECE73B7804935B09013BA8
:10CF7800062B00F21882DFE813F00700160295006E
:10CF88001602920016020702102EDDD995F83031EC
:10CF98001297F6B28DF84C60002BD5D11CA804F07E
:10CFA8005DF912AA1CA9FF2002F0B2F89DF85830CA
:10CFB800C3F3030307468DF82C3095F8480095F81D
:10CFC8007D308DF82D3007220BA902F0A4FA002F2E
:10CFD8005DD100285BD09DF853309DF852201599FB
:10CFE800C5F8E4101B0443EA02239DF851200220EF
:10CFF8001343C5F8E03004F03FF99DF8583095F830
:10D00800480085F82E71C3F30212C3F3030385F8B1
:10D01800703085F878309DF8593085F86920012BF3
:10D0280038BF01234FF47A725343AB651344EB6561
:10D038000DF15A034FF001081093113E94F81B3478
:10D048008DF83C300FA985F868808DF8446002F0AF
:10D058006AFA0223404685F8303101F08DFD18B197
:10D068004146384601F04CFD94F88F34012B00F20C
:10D07800A88194F81A34002B40F09B8194F89134DD
:10D0880043F0100384F89134FEF74EFD65E6012065
:10D0980001F072FD0028E7D001210720E2E7012313
:10D0A80084F8203495F87D308DF82E3094F82434A7
:10D0B8008DF82D3095F88C3095F848000D330BA974
:10D0C8008DF82C3002F014FAA6F10D031BB209906A
:10D0D80023EAE37300B283423FF736AF0B2E7FF6A5
:10D0E80033AFBB4B25931CA8FF231C978DF87460A6
:10D0F8008DF8983002F0D8F8074600287FF424AF5E
:10D1080095F81831012B13D101F070FB002873D06A
:10D11800384601F060FB384601F062FB04239DF8B5
:10D128007C101E9884F88F34C1F3001101F077FB4E
:10D138009DF87C301E99C4F8341413F00F0203D004
:10D148009DF89000002863D19DF89800002862D0CF
:10D15800002A7FF4F9AE9DF89020002A0CBF4FF00A
:10D1680002084FF0030800220A92D5F8EC209142F9
:10D1780054D195F8E910002950D0D5F80C1195F83C
:10D18800EAB009680A9195F81811022902D1032119
:10D1980084F88F14B8F1030F7FF4D6AE13F0600F44
:10D1A8007FF4D2AE0592012795F82E31BBF1000F1E
:10D1B80037D0BBF1010F38D1012B34D16FF00906FC
:10D1C80046FA08F606F00106C6F10206F6B2BDF800
:10D1D8007E100AAA304601F02DFE40B307280CBF86
:10D1E8000823012384F821340A9BC4F83034C4F896
:10D1F8006C34FEF7E5FCB0E501F0FAFA002897D0A8
:10D20800384601F0E9FA384601F0EBFA052386E7DB
:10D218004FF00008A7E74FF00108A4E74FF0010B13
:10D22800C2E70426D3E70326D1E70123DAE71CABDC
:10D23800009305990A9B3246584601F0BBFE20B17F
:10D2480002280CBF0A230B237FE60A9BC4F830345C
:10D25800C4F86C349DF87C3084F82104C3F340137F
:10D2680084F82E3484F8443494F88F3484F8227483
:10D27800012B9EBF0122A86285F81E21012FC4F848
:10D28800280484F82C0484F8410438D1022284F854
:10D29800202495F83A20002A4AD19DF87C20D60609
:10D2A80046D4012B94F840149DF87C2005D8012918
:10D2B80001D1900601D501F05FFBB8F1020F94F897
:10D2C8008F3443D0B8F1030F0AD09DF87C10B8F121
:10D2D800010F4A4601F00F0120A83BD0FFF710F9D3
:10D2E8009DF8903084F82334259BC4F828349DF8A1
:10D2F800983084F82C34012384F82D3430E0049AD3
:10D3080002F0E002A02A1BD195F82E11012285F81F
:10D318003A2009B927996963012B84F8202407D991
:10D32800D5F89020C4F83C24DAF80020C4F89824F2
:10D3380095F81821002AB4D1012284F82524B0E7F1
:10D34800002285F83A2084F82024A6E79DF8981052
:10D3580025984A46FFF7D4F89DF8903084F823348E
:10D368009DF89020E02A08D195F81F312BB984F850
:10D378002324C4F82834A4F82C3494F8913443F0C6
:10D38800020384F891346FE6114D013EB2B2791C64
:10D39800284604F039F80323A4F82034C4F82854A4
:10D3A80084F82C64E9E7012384F82134FEF708FCAB
:10D3B8005AE694F84434002B3FF460AE0020FEF7A0
:10D3C800EDFB94F88F34022B3FF45EAE56E600BFB7
:10D3D800801E002094F89134590715D5012001F0DA
:10D3E800CBFB60B1012001F09DFB08B984F818045B
:10D3F800D4F8403323F00203C4F8403304E0062095
:10D4080001F0BAFB0028F3D194F89134DA077FF5DC
:10D41800F9AC94F840240AB1032A18D11D4A94F8AB
:10D42800181492F86820914205D29B0723D594F8E6
:10D438008F34012B1FD8184806F00AFBD4F8403364
:10D4480023F02003C4F84033FFF742FBDAE4012A53
:10D4580011D194F81924002A3FF4D4AC0D4A94F859
:10D46800181492F868209142E5D29F0703D594F8E2
:10D478004434002BDFD194F8913400206FF3041367
:10D4880084F8913484F81904FFF744FBBAE429B00E
:10D49800BDE8F08F80160020B01F00202DE9F04F66
:10D4A80089468DB090460746002800F08F810029F4
:10D4B80000F08C810368002B00F088814368002B02
:10D4C80000F084818368002B00F08081C368002B02
:10D4D80000F07C81104602F007F8002800F07881FF
:10D4E800BD4CBE4D384601F0C1FA40F2C45200218D
:10D4F800204603F09DFF40F21C520021284603F00D
:10D5080097FFB74BC4F82C3104F50973089304F559
:10D518000A7300264046099308A9B24B84F848804C
:10D528000A9384F8186184F88C608DF82C6001F0F7
:10D53800EDFF0F2306A994F848008DF8183001F084
:10D54800D7FF801B18BF01204FF00A0B84F81C017D
:10D5580006A994F848008DF818B001F0C9FF4FF0FB
:10D56800060A84F8DC0006A994F848008DF818A08B
:10D5780001F0BEFF102384F8DD0006A994F84800E6
:10D588008DF8183001F0B4FF1123C4F89C0006A9E7
:10D5980094F848008DF8183001F0AAFF1223C4F857
:10D5A800A00006A994F848008DF8183001F0A0FFF3
:10D5B8001323C4F8A40006A994F848008DF818307D
:10D5C80001F096FF1423C4F8A80006A994F84800AF
:10D5D8008DF8183001F08CFF1623C4F8AC0006A9AA
:10D5E80094F848008DF8183001F082FF172384F86A
:10D5F800B10006A994F848008DF8183001F078FFBA
:10D6080018230DEB0301C4F8B400C4F8BC0094F867
:10D6180048008DF8183001F06BFFC0B21D2384F864
:10D62800B80084F8C00006A994F848008DF81830AE
:10D6380001F05EFF1E2384F8C40006A994F8480090
:10D648008DF8183001F054FF1F2384F8C50006A98F
:10D6580094F848008DF8183001F04AFF2023C4F8E8
:10D66800C80006A994F848008DF8183001F040FF6A
:10D678000B23C4F8CC0006A994F848008DF818309C
:10D6880001F036FF0C2306A9A4F8D00094F848004E
:10D698008DF8183001F02CFFD4F89C306365D4F86D
:10D6A800A030A365D4F8A430E365D4F8A830236685
:10D6B8004FF00108D4F8AC300590A4F8D2006366A6
:10D6C80084F8B080C4F894B084F898A0C4F84CB03A
:10D6D80084F850A084F8688084F81F81C5F84893BE
:10D6E800FEF77AFD404B009632464FF0FF3105F5C4
:10D6F8005A70C5F84473C4E90B6684F8198185F833
:10D708009164C5F8408306F045F9384B00963246D7
:10D718004FF0FF3105F5607006F03CF9344B009688
:10D7280032464FF0FF3105F5667006F033F902AF67
:10D73800304B009632464FF0FF3105F5806006F019
:10D7480029F9384606F0BAF897E8030004F5927309
:10D7580083E80300284B294F1E60294BC5F84C333A
:10D76800284BC5F85433284BC5F85C33274BC5F80C
:10D778005033274BC5F8583305F553703B68984725
:10D7880004F5A67003F088FB20B1112630460DB0D1
:10D79800BDE8F08F204601F01DFB0028F5D101F00F
:10D7A80041F8B8B91B4801F067FB06460028ECD1E0
:10D7B8007B69984703F006FEBB6D94F819019847FA
:10D7C800FB6A9847012385F89234DFE70326DDE7F3
:10D7D8000926DBE71326D9E780160020481C00201D
:10D7E80000040001642100201DCB00087DC300084F
:10D7F800C5C30008A5BB0008441C0020F049010867
:10D80800C9BD00087DBD000861BB000855BD000802
:10D818002DBD00086817002008B5034B0020C3F889
:10D828004003FEF781F908BD481C002010B5FFF73A
:10D83800A7F90A4C60B90A4B93F81831022B02D1A8
:10D84800084BDB6A98470123C4F84033002010BD19
:10D85800D4F84003013818BF0120F8E7481C00201D
:10D8680080160020F049010838B5134C04F55A70A9
:10D8780006F0EEF804F5607006F0EAF804F5667054
:10D8880006F0E6F804F5806006F0E2F800F0B5FF6F
:10D898000A4B0025DB6A9847C4F84053FEF7B6FDEB
:10D8A8000749084840F2C45203F0AEFD0123C4F80A
:10D8B8004033284638BD00BF481C0020F049010805
:10D8C80080160020BC10002070B52E4B8AB005468B
:10D8D80093F8DD008DF8090093F8DC008DF80A0054
:10D8E80029489A6A90F81804039200268DF80B00CC
:10D8F80004960C46002940D00692D3F88820079257
:10D908001A8F93F81A118DF8151052BAADF8202015
:10D9180093F87C2093F848308DF8243003AB8DF8C9
:10D9280022008DF8232000930DF10A020DF10B035C
:10D938000DF1090105A88DF8146000F0DDFE9DF9D0
:10D948000900FEF713F9607004A801F02BF8B0B9CC
:10D95800049A0F2A0DD863789A420AD81544AB4224
:10D96800A3EB02012CBF002001202170C0000AB0E7
:10D9780070BD002323700820F9E70320F7E7132080
:10D98800F5E700BF80160020481C00201FB504469C
:10D99800002800F012810078412800F20881DFE8B1
:10D9A80010F0420048004D00520056005A005F0037
:10D9B8000601060106010601060106010601060127
:10D9C80066006A006E0079008000830086008B0084
:10D9D80089008D009100940097009A009D00A00096
:10D9E800AF00B300BB00B700BF00C200C600CF0045
:10D9F800CB00CD000601D300060106010601060191
:10DA080006010601060106010601060106010601D6
:10DA1800060106010601DB00DF00E300E800EC0078
:10DA2800F000F400FD00674B93F81831237104B03F
:10DA380010BD644B93F83031237102E0606803F045
:10DA4800C7FB0020F3E7606803F008FCF9E75D4BCB
:10DA580093F81A31F0E75B4BD3F8E0306360F0E7F6
:10DA6800584B211D93F8300103F010FCE9E7554BA2
:10DA780093F81931E0E7534B93F88C30DCE71C231B
:10DA88008DF808304F4B02A993F8480001F030FD9B
:10DA98006060D6E74C4B043493E8030084E8030045
:10DAA800CFE74A4B0434F7E7494B0434F4E7494BD2
:10DAB8000434F1E71A23E3E71923E1E7414B93F82C
:10DAC8006830B9E73F4B5B6DC8E73E4B9B6DC5E7D8
:10DAD8003C4BDB6DC2E73B4B1B6EBFE7394B5B6EC4
:10DAE800BCE702238DF80830364B02A993F87C2056
:10DAF80093F848008DF80A2001F0FAFC2071A0E79D
:10DB0800304B93F8DD3097E72E4B93F8393093E795
:10DB18002C4B93F8DC308FE72A4B93F838308BE79F
:10DB2800284BDB6C9AE7274B93F8503084E7254B5A
:10DB3800D3F88430636084E7224B8FE7264B8DE768
:10DB4800204BD3F8CC30F5E71E4BD3F82C3163606B
:10DB580001F05CFDA06074E71A4BD3F890307DE7C4
:10DB6800184B93F81F3167E7164BB3F88830A3803A
:10DB780067E7144BB3F88A30F9E7124BB3F8D030A3
:10DB8800F5E7104BB3F8D230F1E70E4B93F8482085
:10DB98000AB1062A13D1B3F8A035E8E7094B93F880
:10DBA80048200AB1062A0AD1D3F8A43556E72046F8
:10DBB80004B0BDE8104000F024BE032037E7182069
:10DBC80035E700BF80160020EC160020341700202F
:10DBD800F41600203C170020BC1000207FB5044636
:10DBE80010B9032004B070BDA44DD5F840339A078E
:10DBF80000F171820278412A00F26A82DFE812F0AD
:10DC08004200480056005C00600065006A0077002A
:10DC1800820088008E0094009A00A000A600AC0044
:10DC2800B6006802BB00DD00F000170139012A01C7
:10DC380044014D015101550159015D01680261011D
:10DC480073019B018901AD01B301BA01BF01C40190
:10DC580068022A02680268026802680268026802AA
:10DC6800680268026802680268026802680268025C
:10DC78006802680236023B02400245024A024F022D
:10DC880054025E020079FEF7C1F80028AAD105E027
:10DC98000379022BA5D07A4A82F8303195F891346D
:10DCA80043F0200385F8913400209BE7406803F097
:10DCB80081FA0028F2D094E7406803F0BFFAF8E749
:10DCC8006F4B027983F81A21E8E76D4B4268C3F875
:10DCD800E020E3E76A4E416896F8300103F0CCFA99
:10DCE80000287FF47EAF6368C6F8E430D6E7416861
:10DCF80000293FF476AF002001F0EEF90028CDD0DE
:10DD080011206FE7416800293FF46BAF0120F3E76A
:10DD1800416800293FF465AF0820EDE74168002914
:10DD28003FF45FAF0920E7E7416800293FF459AFA6
:10DD38000C20E1E7416800293FF453AF0D20DBE7F1
:10DD4800416800293FF44DAF0E20D5E7416800290E
:10DD58003FF447AF0F20CFE74A4C494B007983F88F
:10DD68001901A36D9847E36A984797E7444B0279EE
:10DD780083F88C2092E7424E037A8DF8043096F8A7
:10DD8800480096F87D308DF80530072201A901F08A
:10DD9800C2FB00283FF425AF636896F8480001935A
:10DDA800002201A901F0B7FB00283FF41AAF6C3636
:10DDB800D4E9010186E8030070E7314E037A8DF853
:10DDC800043096F8480096F87D308DF80530072223
:10DDD80001A901F0A0FB00283FF403AFB436E7E740
:10DDE800274E037A8DF8043096F8480096F87D306F
:10DDF8008DF80530072201A901F08DFB00283FF4BA
:10DE0800F0AED4E9010106F1740383E8030096F843
:10DE18001831022B7FF442AF96F83031002B3FF4D3
:10DE28003DAF184BDB6A9847FDF748FF36E7144EBD
:10DE3800037A8DF8043096F8480096F87D308DF80E
:10DE48000530072201A901F066FB00283FF4C9AE9E
:10DE5800BC36ADE74368029301238DF80C30084BBC
:10DE680002A993F8480001F063FB00287FF416AF7D
:10DE7800B7E6436802930023EFE700BF481C002081
:10DE880080160020F049010803795A1E0E2A3FF631
:10DE9800A8AE934A82F8683000E7914B42685A6509
:10DEA800FCE68F4B42689A65F8E68D4B4268DA6566
:10DEB800F4E68B4B42681A66F0E6894B42685A666C
:10DEC800ECE6874C037994F848008DF80430062274
:10DED80001A901F020FB00283FF483AE9DF804302F
:10DEE80084F8DD30DAE67E4C03798DF8043094F856
:10DEF800480094F87C308DF80630052201A901F01D
:10DF08000AFB00283FF46DAE9DF8043084F83930E0
:10DF1800C4E6734C037994F848008DF804300A225B
:10DF280001A901F0F8FA00283FF45BAE9DF804302F
:10DF380084F8DC30B2E66A4C037994F848008DF82E
:10DF48000430092201A901F0E6FA00283FF449AE9D
:10DF58009DF8043084F83830A0E6614B4268C3F875
:10DF68009420DA649AE65E4B027983F8982083F865
:10DF7800502093E65A4B4268C3F884208EE6584BEB
:10DF88004268C3F8CC2089E6012B40F0A480554CA8
:10DF98002421204603F04EFA636A984201D01720E4
:10DFA80020E61C2104F1280003F044FA636C98422F
:10DFB800F5D14FF4807104F1480003F03BFAD4F82E
:10DFC80048319842EBD1D42104F5A67003F032FA17
:10DFD800D4F820329842E2D1002104F5097003F008
:10DFE80029FAD4F824329842D9D14FF4607104F553
:10DFF8000A7003F01FFAD4F8A8359842CFD114213B
:10E0080004F2AC5003F016FAD4F8C0359842C6D1E1
:10E01800334E2146304640F2C45203F0F5F920460B
:10E0280040F2C452002103F003FA95F81B3485F836
:10E03800E833736FC5F8EC3396F87D3085F8F8331C
:10E0480040F20123A5F8FA33274B96F819019B6D86
:10E05800984723E68379012B3FF6C3AD204B4268EE
:10E068004068C3F82C2100F0D1FE47E61C4B4268FB
:10E07800C3F8902012E61A4B027983F81F210DE6A7
:10E08800174B8288A3F8882008E6154B8288A3F8E6
:10E098008A2003E6124B8288A3F8D020FEE5104BB5
:10E0A8008288A3F8D220F9E50D4B93F848200AB1ED
:10E0B800062A12D1A288A3F8A025EFE5084B93F809
:10E0C80048200AB1062A08D16268C3F8A425E5E504
:10E0D80000F099FBD9E5012084E5182082E500BF0E
:10E0E80080160020BC100020F04901082DE9F043FB
:10E0F80087B00023ADF800300646002800F0ED8018
:10E108000361FEF73DFD20B10124204607B0BDE8BC
:10E11800F08300F073FD0028F6D100F069FD014698
:10E1280018B96F48142203F083F96E4D95F89134AD
:10E13800012243F0040385F8552485F89134337897
:10E148008DF804300021013B8DF80520ADF806104C
:10E158000C2B00F2BA80DFE803F007B8B8B8788172
:10E16800B8B88FB8AC99A800D5F8407317F0200755
:10E17800CAD196F80480B8F1020F45D1DFF868815A
:10E188005A4CFEF729F896F9051098F848003A46CF
:10E1980001F01BFA88F83900B37988F83830384626
:10E1A80007238DF80530FDF731FEFF2304F586704F
:10E1B800A5F80C31C5F8084185F8047103F04EF84C
:10E1C80004F58A7003F004F83846FDF78DFE04461E
:10E1D80040B196F9051098F84800012201F0F5F9C8
:10E1E80088F83900D5F894343361002C71D000F0E8
:10E1F800FFFC002889D195F8913485F81A0460F35A
:10E20800820385F8913480E7B8F1010F4FF00204DA
:10E21800E8D1DFF8D4908DF8144099F8480089F8CF
:10E228001D7102A901F072F9337989F830318DF83E
:10E2380005708DF80680FDF785FC95F8913443F05C
:10E24800100385F891340024CCE7002269460220A7
:10E2580000F0F6FA0028F6D01324C3E7244BB2885E
:10E26800DB6B96F90C10B0689847D5F8403343F04B
:10E278000203C5F84033E6E702A90D2000F060FB71
:10E288000028E0D0002269460D20E1E7164B93F8FC
:10E298001831D3B9347904F0070000F0ADFA8DF8DD
:10E2A8000040012269461020D2E700226946122068
:10E2B800CEE78DF8072000F090FA044638B900F050
:10E2C80089FA204600F08BFA8CE702248AE70124B9
:10E2D80088E701A800F0DEFB17E7032415E700BF75
:10E2E8009C200020481C0020801600204A1C00208A
:10E2F800F04901082DE9F04F99B08046059118B909
:10E30800032019B0BDE8F08F00230361FEF738FC45
:10E318000646002840F0AB8045460FCD0EAC0FC432
:10E328005A4C98F800A0B8F80C7098F90EB014225E
:10E3380004F58860314603F07BF8012284F8412413
:10E34800534C94F83021022A35460BD194F8182101
:10E35800022A07D194F81E2122B9BAF1010F38BF59
:10E368004FF0010ABAF1010F2DD0BAF1030F2CD0EA
:10E37800BAF1000F35D102229DF83C30DDF840900B
:10E38800029362F34715012694F87C108DF8321039
:10E3980002220CA994F848008DF8302001F0A8F862
:10E3A80094F81A3194F830C194F81D1140B2022241
:10E3B800002B6FD0BCF1010F65D1002963D1002E6D
:10E3C8006DD1104627E00422D6E70023DDF83C9003
:10E3D800BDF840709DF942B0029365F01F05012613
:10E3E800D2E74FF0000BD946CDF808B0CCE74FF094
:10E3F800010084F81A04DDE005F29A420BA900F046
:10E40800DDFA002800F020811320049B33871F4B7E
:10E41800002283F81A241D4BD3F89434C8F810301E
:10E428006FE705F29A452A460BA900F0C7FA0028BB
:10E43800EAD10B9B84F82801C4F82C5184F83031B8
:10E4480002E1B9F1000F00F0FF80002A00F0FC8023
:10E458004946E01C02F0D8FF94F837320133238094
:10E46800F2E01220D1E70220CFE70720CFE7012012
:10E4780047E7064B93F8912483F840A442F0010241
:10E4880083F89124C7E7EEB90220C4E7481C0020AE
:10E4980080160020002E94D05845B8BF584694F8EE
:10E4A8007C308DF82000052294F848008DF8223041
:10E4B80008A901F030F800283FF422AF9DF8203079
:10E4C80084F83930694A6A4BD2F89804D3F89040F6
:10E4D80038B105F083FA664B84423CBF002283F8CA
:10E4E8003A20198F1A8F93F830010491996A09918B
:10E4F80052BA0028B9D093F81B0100B9186393F8F1
:10E508001801ADF85820013893F87C2093F81A4187
:10E518001491D0F1000BD3F888108DF85B204BEBE9
:10E52800000B93F8482093F83A0093F868308DF878
:10E538005A3009AB00934F4B03904FF001008DF810
:10E548004C0015918DF85C20A3F12F01A3F1300246
:10E5580013A88DF84D4000F0CFF8039B4FEA0B1B32
:10E568004BEA431B00264BEA801B4BEAC413B14518
:10E578003E4C039308BF37463A46494604F59C701B
:10E58800CDE90A669B46268084F81A6402F03CFFAF
:10E59800E9B2A570C5F34215FAB2042D344E039BB7
:10E5A80084F837223FF423AF072D3FF44AAF022DFA
:10E5B8007FF459AF304D84F80D110420029984F886
:10E5C8000401FF2084F80C0184F8281184F8143120
:10E5D800D6F8E410C4F8085105F59B730AA8C4F8E6
:10E5E800101184F83021C4F82C3100F017FC0028F1
:10E5F8007FF437AF0A9BA4F844040BA8A4F816319B
:10E60800C4F84C3400F0CEF900287FF4FDAE0B9B23
:10E61800D3B196F93900FDF7A9FA94F83732002BEF
:10E628003FF4FFAE0B9B0F2B3FF6E6AE05F58B7262
:10E638000BA90F2000F0C2F900287FF4E5AE0B9B70
:10E6480063F3030B84F814B10598FDF74DFC00281B
:10E658007FF4DBAE099B86F83A00B36200F07EF9DE
:10E6680000283FF406AF1320D1E600BF481C002065
:10E6780080160020E81600204A1C002037B50B4DF4
:10E688008DF8040004460F2295F8480001A900F00F
:10E6980042FF40B1064A85F81C4192F8913443F094
:10E6A800200382F8913403B030BD00BF80160020EB
:10E6B800481C002010B5FFF7B9F8044688B90A4885
:10E6C80005F0C6F9094805F0C3F9094805F0C0F98D
:10E6D80000F093F8FDF780FD064BDB6A984720466B
:10E6E80010BD0124FBE700BFB01F0020C81F002099
:10E6F800E01F0020F04901082DE9F04F8BB0477862
:10E708000093149B90F90C8090F90D6090F80E908E
:10E718008B464168196004469246002F57D0022361
:10E728008DF8103004A9C37B007C8DF8123000F0FE
:10E73800DFFEB4F808C0618943B260689845454671
:10E748006144B8BF1D46604534BF00270127884291
:10E7580009D30A218DF81010207C019304A900F038
:10E76800C7FE019B46B2B4F808C0608961680CEB2B
:10E77800400E714520D3A1EB0C01B1FBF0FC00FB6E
:10E788001C11C9B998450ADC237833B10223207CCF
:10E798008DF8243006A900F0B9FE4FF001092123B5
:10E7A8008DF81030207CE37B8DF8115004A98DF88A
:10E7B800123000F09DFE45B2009B8BF800503846A1
:10E7C8008AF8006083F800900BB0BDE8F08F4546EA
:10E7D800F2E77047704770477047002070477047EE
:10E7E800704770470020704700207047002070472E
:10E7F800002070470020704770477047704702201C
:10E808007047022070470220704770470020704709
:10E818007047704700207047002070477047704766
:10E828007047000010B5054C4FF4037220460021D4
:10E8380002F0FEFD0020C4E9000010BD08220020FF
:10E848002DE9F8438146174600293FD0244B00257F
:10E8580003F1010C1A462801103312F8018FB8F1A0
:10E86800000F36D19A42F8D11E4E33680BB9C6F85C
:10E8780000C073680BB1C3F800C033180024013519
:10E888009C6083F80C900D302B01BAB206EB05158D
:10E898003044F750C6F804C002F0B6FDB9F1110FC4
:10E8A8004FF0000398BF104C6B71D6F8083298BF30
:10E8B80024FA09F403F1010398BF04F001043B446E
:10E8C8002C71C6F808324046BDE8F8834FF00108BD
:10E8D800F9E70135202DBBD14FF00208F3E700BF5F
:10E8E8000F220020082200202007020010B510B3D4
:10E8F800124A1368984204D103681360002304E0A5
:10E908000B4613B119688842FAD15168884208BF8A
:10E9180053600BB101681960D2F808328168013B75
:10E9280000245B1A04602146C2F80832102202F063
:10E938007FFD204610BD0120FCE700BF0822002013
:10E94800054B1B6813B11A798242FAD1002B0B6070
:10E958000CBF0320002070470822002010B5054B8B
:10E96800186800B910BD037B04680BB9FFF7BEFF38
:10E978002046F6E70822002038B5084B084C1868EE
:10E9880000B938BD03790568112B05D824FA03F3BB
:10E99800DB0701D5FFF7AAFF2846F1E70822002088
:10E9A8002007020028B1044BD3F808320360002086
:10E9B80070470120704700BF082200202DE9F04170
:10E9C80007460E4615463AB331B3144B1C6800236C
:10E9D8002CB93046FFF7E6FF0020BDE8F081A268B9
:10E9E800F91A0132914210D32279EA54581C22892B
:10E9F8005FFA80F8611D55FA80F002F005FDA36802
:10EA0800246898445FFA88F3E2E720462468FFF711
:10EA18006DFF002CF9D1DCE70120DEE70822002099
:10EA28000238C0B211289ABF014B185C0020704709
:10EA3800FF42010830B50B4B93F8202004460846E6
:10EA480072B100211C330578A54208D001319842E3
:10EA5800CDB20CBF04480430AA42F4D8002030BD1F
:10EA68001046FCE7142400202024002010B5084C90
:10EA780000232060142204F10C00FF2184F82030C8
:10EA8800C4E9010002F0D4FC012384F8213010BD50
:10EA98001424002010B50E4A92F82010042915D825
:10EAA800936804781C7044785C70C4788078987097
:10EAB8000131DC7082F8201002F11C018B4214BF76
:10EAC800043302F10C039360012010BD0020FCE721
:10EAD80014240020094B93F8200068B15A6803F108
:10EAE8001C018A4200F1FF3014BF043203F10C020A
:10EAF80083F820005A600120704700BF14240020CA
:10EB080010B5074B93F820200446084632B15968DF
:10EB1800FFF790FF10B101234470837010BD00BF50
:10EB28001424002008B5064B93F820202AB1596810
:10EB3800FFF780FF08B1407808BD0120FCE700BF5F
:10EB48001424002030B50A4A92F82010536882F83D
:10EB5800210061B1916801241C32DD78587005B933
:10EB68009C7093420CBF034B04339942F5D130BDDE
:10EB7800142400202024002008B5044B5968FFF70E
:10EB880059FF003818BF012008BD00BF1424002019
:10EB98002DE9F3410422154E044600210DEB020035
:10EBA80096F8208002F044FC0025EBB2984502D884
:10EBB80002B0BDE8F0817368197821705A786270E4
:10EBC8009F785FB1336820469B689847FFF782FFBC
:10EBD80017B901A8FFF75EFF0135E6E7DB788DF886
:10EBE80004108DF805208DF80730EFE71424002075
:10EBF800014B93F82000704714240020034B93F82E
:10EC08002000042894BF002001207047142400200D
:10EC18001FB50024CDE90244C41F8DF800408DF8CB
:10EC280001100C0AADF80420090C120C8DF8031021
:10EC38008DF806208DF8073002461B0A0121684628
:10EC48008DF802408DF8083002F04FFA002818BFFE
:10EC58000E2004B010BD2DE9F04188B017460D46CE
:10EC68000F9A064600284DD000240121CDE904441E
:10EC78008DF810109DF838108DF81510ADF8163075
:10EC8800190CCDE900441B0ECDE902448DF819306A
:10EC9800ADF81A20130C120E07948DF818108DF881
:10ECA8001C308DF81D20E3B24FEA0318002D5FFADF
:10ECB80088F803DC002008B0BDE8F081013310219A
:10ECC8008DF81F303A466B460DEB010002F0A3F9B0
:10ECD8000346C8B9102DAC46A8BF4FF0100CDAB2E5
:10ECE800624503F1010303DB103D2DB20134DAE77D
:10ECF80008EB020020326A44315C12F8202C4A40AA
:10ED08003254ECE70920D6E70E20D4E7013803286F
:10ED180015D8DFE800F002080C100A4B1B681B69C5
:10ED28000B6000207047074B1B685B69F8E7054BD1
:10ED38001B689B69F4E7034B1B68DB69F0E7052058
:10ED4800704700BF382400202DE9F041C4B00C46BC
:10ED58004A9E17461D468046B8B3B1F5807F36D81F
:10ED68004FF488720021684602F062FB4923009341
:10ED78004FF48073ADF804302B0C8DF80830330C49
:10ED8800ADF80650ADF80A608DF80C302246002325
:10ED9800414604A82D0E360E8DF80E308DF8095018
:10EDA8008DF80D608DF80F4002F02EFB04F1100174
:10EDB8004B9A3B4689B2684602F017F910B1012810
:10EDC80018BF0E2044B0BDE8F0810920FAE70D20F5
:10EDD800F8E7000010B590B10A4C28220021206005
:10EDE80002F026FB2368084A1A6000204FF0FF3221
:10EDF800C3E90302C3E90522C3E9072210BD0820BD
:10EE0800FCE700BF3824002000010101024B1B6809
:10EE180018600020704700BF3824002030B1044B30
:10EE28001B68DB68013303600020704709207047C6
:10EE38003824002013B500230C460193D2B101A950
:10EE4800FFF764FF18B9019B591C02D1146002B086
:10EE580010BD99B2611A002902DD0B441360F6E770
:10EE680002D113600720F2E71B0C1B0403F5803363
:10EE78002344F3E70920EAE728B1044B1B681C3355
:10EE88004362002070470920704700BF38240020E3
:10EE98001FB5044600B3002303A8039302F07CF9CE
:10EEA800104ABDF80C30126820469380E38200F0C7
:10EEB80056FA98B904F11803009321680123132224
:10EEC80002F08AF860B9204600F049FA003818BF05
:10EED8000120000104B010BD0920FBE71020F9E76C
:10EEE8000E20F7E738240020F0B5054687B01C4609
:10EEF8003BB32F4E3368DB68834257D894F8202001
:10EF0800002A14BF09220822834205D3204600F0B4
:10EF18005AFA70B110200AE0002301900093A36808
:10EF280094F82810606AFFF796FE0028EED007B024
:10EF3800F0BD23792168B4F808C0A768043B9AB2E9
:10EF480009B90920F3E7B2F5807F2DD8ADF80EC0D6
:10EF58008DF817304FEA174C04F12C033F0E8DF84B
:10EF6800117000932F0C08234FF0490EADF80C00D8
:10EF78008DF814708DF816002F0E0DEB0300CDF8E8
:10EF880008E08DF810C0ADF812508DF8157002F039
:10EF980023F808B10E20CAE7204600F014FA00282A
:10EFA800B8D13368DD60C2E70D20C0E70620BEE7B0
:10EFB800382400202DE9FF410A9D80460F46164659
:10EFC8001C46002D5AD0002303A910460393FFF7CF
:10EFD8009DFE18B1062004B0BDE8F081039B9C4259
:10EFE80001D80133F6D1284600F05EF9002847D150
:10EFF800264B1A78424503D01A79424542D101205E
:10F00800AA68BA4240D103EB8002EB6A92F8018009
:10F018002979CDE900430439927828683B4689B2BA
:10F02800FFF792FE0028D6D195F820300194002BE6
:10F038004FF00103009314BF4246082295F82810A8
:10F04800686A3B46FFF707FE0028C4D1013E032E3D
:10F05800C1D8DFE806F002070B0F0D4B1B681C61D7
:10F068001C62B8E70A4B1B685C61F9E7084B1B6830
:10F078009C61F5E7064B1B68DC61ACE70920AAE751
:10F088000F20A8E70B20A6E70220A4E7A408002089
:10F09800382400201FB50A460B2A4FF00001CDE99D
:10F0A8000011CDE9021107D00C2A13D00A2A0FD07B
:10F0B8000A2005B05DF804FB012802D120238DF851
:10F0C8000030684602F011F8002818BF0E20F0E75B
:10F0D8003023F4E70B21F4E738B5054602F000F8D1
:10F0E800044678B97DB9094B1B680B219878FFF75E
:10F0F800D1FF38B90C21FFF7CDFF18B90A21FFF766
:10F10800C9FF00B10E24204638BD00BF38240020B6
:10F118002DE9F04380468FB00C461746002A6BD085
:10F12800002969D0002529461D2206A8059504F066
:10F13800A1FE8DF81350344D2B680DF114099E88EB
:10F14800CDF804900DF1130302933B7900933B68CB
:10F1580032462146404601F0E4FF00284ED1386887
:10F168003A79494602F050F9384600F04FF800283D
:10F1780046D13C7AFA79BB79240444EA02241C4338
:10F188002B689A6894423DD99C609DF813000B2126
:10F19800FFF780FF034658BB0C21FFF77BFF0346B0
:10F1A80030BB0A21FFF776FF034608BB7B7ABA7AA1
:10F1B800FF7A3F0447EA02271F433A46334621466F
:10F1C8000920FFF725FD034690B933463A46214604
:10F1D8000820FFF71DFD034650B92A689DF8131053
:10F1E80091700021D1604FF0FF31C2E904119161A3
:10F1F80018460FB0BDE8F0830923F9E70E23F7E7B7
:10F208000F23F5E70323F3E73824002010B504465D
:10F21800002845D00168002942D011F8013B43710C
:10F228000322063002F0F0F82046032250F8091BAA
:10F23800043102F0E9F82168CB79E3600A7A43EAFD
:10F248000223E3604A7A43EA0243E3608A7A43EAA4
:10F258000263E360CB7A23740B7B63742379212BDD
:10F268001AD110220D3104F1120002F0CDF81D223E
:10F278002168501C8B5C6362085C43EA0023901C85
:10F288006362085C033243EA004363628A5C43EAD0
:10F2980002636362002010BD112B03DC0D22E7E737
:10F2A8000220F8E70120F6E710B50446002854D0FC
:10F2B8000168002951D00B7843714B7883608A78B4
:10F2C80043EA02238360CA7843EA024383600A79E7
:10F2D80043EA026383604B7903738B79C381CA79EC
:10F2E80043EA0223027BC38102F00F020831103087
:10F2F80002F08AF8237B002203F00F0384F8202011
:10F3080084F82820227903F10800111A04290DDD58
:10F3180021680933043AD21A085C84F82000D2B272
:10F32800606A84F82820194402F06EF8237922686C
:10F338001A44002012F8043CE36212F8031C43EA62
:10F348000123E36212F8021C43EA0143E36212F864
:10F35800012C43EA0263E36210BD0220FCE710B50A
:10F36800044660B3036853B30279162A29D942794F
:10F378001A700146082251F8060B013002F04EF8C7
:10F388002146082251F80E0B093002F047F823688D
:10F39800E28A5A74E38A22681B0A93742368A26972
:10F3A800DA74A36922681B0A13752368628B5A757D
:10F3B8002368E27E9A7517232371002010BD01206F
:10F3C800FCE70220FAE738B50446002863D0016854
:10F3D800002960D0037B90F8282003F00F03002A4F
:10F3E80057D10833207904321344984255D36379AE
:10F3F8000B702368A2685A70A36822681B0A93706E
:10F4080023686289DA702368E27A1A712368227B9A
:10F418005A712368E2899A71E38922681B0A214696
:10F42800D371227B51F8100B02F00F02083001F063
:10F43800EBFF237B94F8282003F00F0303F1080562
:10F448002AB1226894F82010515503F10905206863
:10F4580094F82820616A284401F0D6FF94F82830EF
:10F468002268E16A2B44D1545A1CE16A206892B29E
:10F47800090A81549A1C2168E08D92B28854DA1CDA
:10F48800216894F82F0092B2043388542371002025
:10F4980038BD0933A6E70120FAE70220F8E70000A3
:10F4A800024B1A8810431880704700BF3C24002084
:10F4B80008B5074B1B883BB1FEF7B8F900280CBF0D
:10F4C80000206FF0020008BD6FF00100FBE700BFED
:10F4D8003C24002010B5034B00241C80FEF79CF947
:10F4E800204610BD3C240020B0FA80F04009704747
:10F4F80082B018B9084602B000F0CAB8002002B0BD
:10F50800704710B9084600F077B9704710B9084637
:10F5180000F08EB970470346084611460BB900F053
:10F52800E5B90020704710B9084600F071BD704772
:10F5380010B9084600F006BA0020704710B4044617
:10F54800084611461A46019B14B910BC00F018BAB7
:10F5580010BC70470346084611460BB900F042BA82
:10F568000020704710B40446084611461A4614B9DC
:10F5780010BC00F0AFBA002010BC704730B405468C
:10F58800084611461A46DDE902341DB9029430BC1A
:10F5980000F02EBB002030BC704710B9084600F0C0
:10F5A800DFBB0020704710B9084600F06FBD00208F
:10F5B800704710B9084600F0EEBB0020704710B93C
:10F5C800084600F0EBBB002070470346084611468A
:10F5D8000BB900F005BC0020704710B4044608467B
:10F5E80011461A46019B14B910BC00F0FBBB092058
:10F5F80010BC704710B40446084611461A4614B9A0
:10F6080010BC00F063BDC8B210BC7047004870471A
:10F6180001000102064B10B51B6A0446984730B139
:10F628000448054B204498428CBF0020012010BD9F
:10F63800F049010840C220C980B92A00F0B5114B31
:10F6480085B00C4610491F56054601F049F80F4B86
:10F65800E4B25E6A072D4FF00103CDE9024301468B
:10F668000AD105220023CDE900234FF47A727A43A8
:10F678001846B04705B0F0BD08220020CDE90020AB
:10F688003A46F5E73B43010814430108F0490108ED
:10F698001FB5002300930378013B372B21D8DFE8FF
:10F6A80003F01C242020201E202020204143454E0A
:10F6B8002055585B5E6164206C1E6E73787A20203A
:10F6C8007D8126202020202020202020202020206E
:10F6D80083858A2020838A208C90C3780BB10223EB
:10F6E8000093009805B05DF804FB8378F6E743784B
:10F6F8008DF8043005238DF805308378003B18BF5A
:10F7080001235B008DF8063010238DF80730304B4D
:10F718001B6801A803F55872CDE9022300F0C0FF69
:10F728000090DEE74023DBE72023D9E7827890F9D1
:10F73800013012B9274AD35CD2E7274AFBE782781F
:10F7480090F90130002AF8D1244AF4E740F6B8339A
:10F75800C6E74FF47A73C3E74FF4FA63C0E741F2A0
:10F768008833BDE741F27073BAE71D484FF47A71E8
:10F7780001F02EFE00F5FA60D2E71A4BB0E7144B01
:10F788001B6803F55873ABE7114B1B6803F55B73F4
:10F79800A6E71023A4E70E4B1B68A1E74FF08343AD
:10F7A80000939EE7104BFBE7104B99E740F21113CB
:10F7B800ADF8003095E7032392E790F901300C4A41
:10F7C800B9E70C4990F9010000F08AFFA8E700BFEB
:10F7D80044240020C3430108CB430108D343010854
:10F7E80018FCFFFF00EA06379A99094040F70937E5
:10F7F8003B4301081443010837B50B4B02781B68DB
:10F808000C2101FB02335B7A03EB4304074B1D68B1
:10F8180003690093C3684278816805EBC40000F06F
:10F82800DFFC03B030BD00BF44240020402400208A
:10F8380070B586B0027B6423ADF80030012A4FF022
:10F848000003CDE90133CDE903338DF802308DF89B
:10F85800143030D0022A39D05ABB03684BB34368FE
:10F868003BB31F4D80682B601E4B182269461860F9
:10F8780001F0CAFD1C4B2C6893E807000C3384E8A0
:10F88800070093E8070004F10C06032386E8070045
:10F89800A4F86C33012204F55B7104F5587000F08C
:10F8A80090FC2B684FF6B072A3F878230522C3F8B2
:10F8B8007C2306B070BD0A4908684360036100F5FF
:10F8C8005B7100F5587000F07CFCF2E7044B1B6894
:10F8D800B3F86023B3F86C130A43A3F86023E8E78E
:10F8E80044240020402400206840010808B503464D
:10F8F8000A2924D8DFE801F006232323230B161B4B
:10F9080023212100BDE808400068FFF783BE90F975
:10F9180000009978052271B900F013FC003818BF6F
:10F92800012008BD052293F900000021F4E790F9B1
:10F9380000005978EEE70221EEE70722F3E70020FE
:10F94800EFE7000010B504791CB1012C0BD00020A2
:10F9580010BD0A4B01681B68012203F5587000F0BE
:10F9680030FC0120F4E7054B01681B68224603F5CB
:10F978005B7000F026FC2046EAE700BF4424002024
:10F98800F7B50528144D1C46A8BF052058700E462B
:10F998002946174600F0A4FE94F90130A070072B01
:10F9A80013D1322000F09CFD0C4BDB6D05469847C7
:10F9B80004F10C0208340346019200943A46314699
:10F9C800284600F092FD03B0F0BD054A55F8231013
:10F9D800D05C00F07DFDE7E714430108F049010819
:10F9E8003B4301082DE9F04F344F90F901607B68E3
:10F9F800D0F804908BB004468846984705460028FE
:10FA080059D1E37C73B92E4A2378126803EB430378
:10FA1800990002EB8303D3F80490B9F1000F01D1E8
:10FA280052F80190274B484613F906B0FB689847EF
:10FA3800A37CD7F818A022890993072E28D1002380
:10FA48000121CDE90223204A0693CDE90431CDE90D
:10FA580007330521CDE900214FF47A7202FB0BF23E
:10FA68004CF250311846D047637C13B3174B995D5D
:10FA78007B6D0D31C9B228469847E07C324649462D
:10FA880000F040FE88F8006001200BB0BDE8F08F60
:10FA9800002101250823CDE90013CDE90715CDE99B
:10FAA8000511CDE903110292A1782B465A46284642
:10FAB800D9E7074BDBE70020E7E700BFF04901087B
:10FAC800442400203B43010885450100D343010835
:10FAD800C34301082DE9F04F8DB090F90130DFF8EC
:10FAE800FCA0DFF8FC90CDE90A123E4A12F903B0F7
:10FAF8000278DAF800300C2505FB02333A4A5B7AC3
:10FB0800126803EB430302EBC303044693F90210A4
:10FB180090F9020000F0DFFD3449064694F901002F
:10FB280000F0DEFDA26861688046304600F005FD01
:10FB38002178DAF80020D9F80C3069430746505884
:10FB48009847D9F81C309C4694F901300025072BBA
:10FB58004FF47A63CDE90753CDE905552DD101233B
:10FB6800CDE903530523CDE901534FF47A7303FB21
:10FB78000BF300933946434646F2A81228466746D7
:10FB8800B8472378DAF800200C214B4394F9011088
:10FB9800D05800F0D9FDA18994F90100FFF74EFD76
:10FBA8000B9B217B1860D9F85430284698470A9B4C
:10FBB80001201E700DB0BDE8F08F01200823CDE9AB
:10FBC8000350CDE901032A46CDF800B06546434607
:10FBD8003946A84701200546D3E700BF4424002042
:10FBE800F04901083B430108402400201443010860
:10FBF8002DE9F04F8FB0002405468A469146984675
:10FC08000494ADF81440ADF8024007264FF0010BFC
:10FC18002B7AA34206D9686804A9204400F0F2FBB5
:10FC280000285ED102238DF8083002A86B7A8DF87F
:10FC38000A30FFF72DFDAB7A8DF81D309DF8113095
:10FC48008DF81E309DF812308DF81F309DF8103059
:10FC58008DF82030EB7A8DF821302B7B8DF822300F
:10FC68006B7B8DF8233010238DF81C608DF82430C1
:10FC78003A4E8DF82C000DF102030A9305238DF8F6
:10FC88002D3033680C930723ADF834302B68069376
:10FC98000DF1120204AB0DF1110106A800F0CCFB26
:10FCA800072805460BD130680C22002100F5587052
:10FCB80001F0BEFB3368BDF80220A3F860239DF86D
:10FCC80011308AF800309DF8123089F800309DF81C
:10FCD800103088F80030189B28461C700FB0BDE81B
:10FCE800F08F9DF81330BDF81470ADF80270204401
:10FCF800C4B2F3B917B3194A00201168072602469F
:10FD08004FF00C0C062B1BD10CFB00FE51F80EE03B
:10FD1800BEF1000F04D00BFA00F23A4397B2012269
:10FD280001301028EED1002A3FF472AFADF802700E
:10FD38006EE75A1E042A01D9062BDCD0062667E78F
:10FD480047FA00FE1EF0010FEAD00CFB00FE51F846
:10FD58000EE0BEF1000F08BF0626E1E744240020AC
:10FD680038B505464068FFF755FC0522841D00217B
:10FD780095F90000E4B200F0E4F908B904F0FD04D4
:10FD880095F901000722002100F0DBF908B904F019
:10FD9800FB04204638BD00207047000010B50378EA
:10FDA8000F2B044618D84068FFF734FC22780B491B
:10FDB80002EB42020968831C01EB820051F8222001
:10FDC800DBB21AB903F0FD0358B210BD032B06BF0E
:10FDD800626842600223F7E70020F6E74424002027
:10FDE800022070472DE9F04FDFF838810446D8F833
:10FDF800000099B08946174600211E4601220323B8
:10FE080000F55870CDE90611CDE908118DF81410E8
:10FE18008DF81510ADF8163000F0B5F938B9D8F8E6
:10FE28000020B2F8603343F00303A2F86033D8F837
:10FE38000020637A8DF8283002F55871CDE90B124D
:10FE4800394A94F9083012680D920DF116020F9292
:10FE58002268109262681192D4E90301A27A8DF89F
:10FE6800482001228DF8492013AA82E803001025B2
:10FE7800227DE18A8DF8293018468DF85420ADF896
:10FE88003850FFF7DBFB0AAB17930DF115031690FB
:10FE980000933146019705AB06AA10A800F0BCFBF9
:10FEA800064698BB9DF81410204F013901F090FACE
:10FEB8001F4B1B690393C4B24FF00C0B04F1600392
:10FEC8006B44D8F8000013F848AC9DF814300BFBCD
:10FED8000AFC01343946B4FBF3F203FB1244D0F8B0
:10FEE8007C33B0F9782350F80C00DDF80CC0E4B28C
:10FEF800E04728B189F800A0304619B0BDE8F08F76
:10FF0800013D15F0FF05D9D10D26F5E70C2801BFF5
:10FF1800D8F80020B2F8603343F00303A2F8603346
:10FF2800EAE700BF4424002040240020400D0300DD
:10FF3800F0490108F8B50679012E054601D80620D2
:10FF4800F8BD0F2E2BD80368187A40F3030005225A
:10FF5800002140B200F0F5F82B680446187A40F307
:10FF680003100522002140B200F0EBF8A8B1B4FA62
:10FF780084F4640929680B7A086843F3030243F39D
:10FF8800031352B25BB29A42C8BF0124FFF742FB87
:10FF980048B9002CD3D10420D2E70124EAE7032092
:10FFA800CEE70520CCE7002CFBD10C4F29683B6835
:10FFB80006EB460003EB80000C2201F025FA3A68B4
:10FFC8000C2303FB062320465C72B2F8601301235E
:10FFD800B3400B43A2F86033B2E700BF44240020CB
:10FFE80010B4017801290ED9084B18680C234B432B
:08FFF800C4180022C250C4E944
:020000040801F1
:10000000012200F5587010BC102200F0A7B80020A3
:1000100010BC7047442400202DE9F04186B05023E5
:100020008DF81430037A102B074630D14368DD7BFE
:100030006DBB0224A8466426062C14D87A68535D4A
:1000400003932A44517843EA01230393927843EAC5
:1000500002437343CDE9033863B968468DF8004025
:10006000FFF7C2FF0DE0CDF80C808DF81480CDF8BD
:100070001080F2E703AB01A801938DF80840FFF769
:100080005DFF0134E4B2102C05F10305D4D106B0B4
:10009000BDE8F0811FB502680379116851B901A864
:1000A0008DF80430FFF7A0FF78B9002040B205B00A
:1000B0005DF804FB02A802928DF80C30FFF73EFFBA
:1000C0000628F2D8024B185CF0E70320EEE700BFE9
:1000D00034430108C90020B9034B0B449856C0B201
:1000E0007047024BF9E700BF43430108834301080F
:1000F000F0B59A42069D03DB9DF914309A4220DD4B
:100100000020F0BD03EB430331F814C005EB83037B
:1001100000264CFA06F7FF0707D51F7A07F00F0EE7
:10012000724502DBB2EB171F0DDD0136102E03F115
:100130000C03EED10134E4B22301DBB29842E1D8E2
:10014000DEE70024F8E70120DBE7884204DB904289
:10015000CCBF0020012070470020704710B5140963
:10016000B4EB111F03464FEA11100ED391420CD28B
:1001700002B201F00F0133F81240012000FA01F140
:1001800024EA010123F8121010BD0020FCE7F0B5AD
:1001900028B100EB410501270020914200D3F0BDBA
:1001A000002435F802CB234607FA04F636EA0C069B
:1001B00008BF013304F1010408BFDBB2102CF3D1F6
:1001C00018440131C0B2C9B2E7E710B500B149B96E
:1001D00010BD31F8134020F813400133DCB2A242C5
:1001E000F7D8F5E70023F9E782B030B50488049327
:1001F0006AB9B3F5616F18D349F6AF2542F21072B0
:10020000AB4298BF4FF47A72944238BF1446012C27
:1002100038BF01246143BDE83040C3688B428CBFC6
:100220005B1A0023C36002B070476422ECE7000051
:100230002DE9F04F91B01546DDF86C8004939DF8E0
:10024000683009930C46064603F0C2FB684ADFF8A3
:10025000A4B10590A8F5F633303BB3FBF2F353435A
:1002600003F5F63203F5A83303F5C073039318239F
:1002700013FB054330320692089300254FF0FF3AF6
:10028000089BA34207D1002D14BF50464FF0FF300A
:1002900011B0BDE8F08FBDF97030ADF82C300B997E
:1002A000CDF86C804046CDF8288003F021FBB4F8EF
:1002B00000906EB9B8F5616F5BD349F6AF2242F298
:1002C0001073904598BF4FF47A73994538BF99469B
:1002D0004B46012B38BF01230793002E52D1B9F1B1
:1002E000640F48D1A0605F46A1680EA803F022FB0E
:1002F0000F9B0093DDE90A120E9B0CA803F079FA1C
:10030000049B0C9A0BB9099B2BB12369BB4202D108
:10031000394B9A420DD9394BE760984509D90023EA
:10032000ADF83430069B0D990C93184603F0E0FAB3
:10033000A060606800B9E760276126B103F052FB56
:10034000E3680344E360D4E903329342059B1D99BB
:100350006360079B88BFE2604B43E168994202D229
:100360000498A8B9A6B101231D442375EDB2183431
:1003700086E76423A9E7B9F57A7F0ABF204F214FAA
:10038000A060B1E7049B0BB9C4F80CB05F46D0E79E
:1003900000209342207506D85B1A9A4505F10105A5
:1003A00028BF9A46EDB2002EE1D1B9F1640F164A8A
:1003B000ADF8346019D049F6B023B9F57A7F18BF8B
:1003C0001346904584BF039A9B180C931C9B009383
:1003D0000CAF97E806001B9B384603F00AFA97E833
:1003E000030003F085FA8246C1E74FF46163E8E752
:1003F0008051010040771B007F5101002FEC01006C
:1004000080A81201002E930230EC01000378032B28
:1004100014D1437803F00F021B098A704B70837864
:100420008B80C27843EA02238B800379C3F30212E4
:1004300003F00F03CA700B7005207047002070474F
:100440002DE9F34798464379057990F9076091467D
:10045000044690F906208A4683B190F9087075B376
:100460000F2A12D194F909200F2E1ED194F90A6097
:10047000072D24D1002F08BF012720E090F90B7031
:1004800090F9092090F90A60E9E7A369019394F9CA
:1004900015300093216994F91430207BFFF728FE72
:1004A0000028E1D105F0FD05DEE794F91D30B342E7
:1004B0000FDC94F91C30B342DADA05F0FB0528466C
:1004C0008AF8002089F8006088F8007002B0BDE862
:1004D000F0871E46CCE70000024B03FA00F0B0FBA9
:1004E000F1F0704740420F004FF4FA53B3FBF0F0C5
:1004F000704730B54FF47A750C1F6A4300FB042235
:1005000052001EBF00F1FF341219B2FBF0F291420B
:1005100038BF1146039A1160820048431CBF013066
:1005200040084FF47A71121A01FB1323002BCABF43
:1005300003F2E73393FBF1F1B3FBF1F1049B196094
:1005400030BD38B5400014460D46F1F763FA014658
:100550002846F1F7ADF92146F1F7AAF9F1F79CF831
:1005600003F0DAFCF1F778F940B238BD2DE9F74F26
:10057000019300231F469C461C01058A5FFA84FEF6
:1005800004F0F004A54206D8019B82F800C01F7059
:1005900003B0BDE8F08F0EEB4E054FEA4309AD0006
:1005A0000024466836F809602641F60727D5866894
:1005B00006EB050A765916B3067836B9466926B1B0
:1005C00036F809602641F60719D59AF8086090F9BF
:1005D00001B046F303084FFA88F8D8450FDC46F31C
:1005E000031676B25E450ADB9AF8096006EB460808
:1005F000C66806EBC806367D4EB90137FFB2013436
:10060000102C05F10C05CCD10133DBB2B4E70CF1B1
:1006100001060EEB040801F80C805FFA86FCEEE799
:100620002DE9FF4704464068DDE90C671D468A4610
:10063000914603F0D7F923681B1A3B604FF000087E
:100640000123337085F80080636813B12368834207
:1006500024D8CAF80080D4F81CC0A3699CF800E034
:100660000393D4E9030101AB83E80300237D0093E6
:10067000DCF80C10237A627A7046FFF7D9FD334616
:1006800038602A46E0694946FFF770FF2B782BB1A6
:10069000C7F80080002004B0BDE8F0873378002B55
:1006A00014BF0B200C20F6E737B590F9002090F925
:1006B0000250954204460FD0013A52B295420BD0F7
:1006C000A368019394F9013000936168E0782B46A8
:1006D000FFF70EFD0028EFD0104603B030BD884272
:1006E000B8BF08467047000051F82000054B9842FB
:1006F00005D0054BC31A58425841400070470120AD
:10070000704700BF90D0030020A1070005281FB547
:100710000ED80C4B53F820300093CDE901120A4B50
:1007200001220021022002F069FE05B05DF804FB01
:10073000CDE90012054B01220021022002F05EFEED
:10074000F3E700BF48440108DB430108FA4301080E
:1007500007B5054BCDE9000101220021022002F07E
:100760004DFE03B05DF804FB1644010810B51022DD
:1007700004460021F13000F05FFE0021C4F814119E
:100780002046F022BDE8104000F056BE0246084662
:10079000102100F0A5B92DE9F0430446D0F814016A
:1007A00085B00E46154604F2011988B3C0F1100851
:1007B0009045474628BF1746BAB2484400F028FE85
:1007C000D4F814313B440F2BC4F814312DD9A8456B
:1007D0002BD204F1F00304F5807113F8012F187C7B
:1007E0008B4282EA00021A70F7D104F1F10810225C
:1007F0004146684600F00CFE22466946684600F015
:10080000E9F910226946404600F002FE3E44ED1B25
:1008100004F5807804F1F107102D09D8AAB2314609
:10082000484600F0F5FDC4F8145105B0BDE8F0836A
:1008300004F1F003711E13F8012F11F8010F434565
:1008400082EA00021A70F6D110223946684600F09A
:10085000DFFD22466946684600F0BCF91022694671
:10086000384600F0D5FD1036103DD5E7F0B589B01B
:100870000C46102200210546684600F0DDFD2246A8
:100880006946684600F0A6F99DF90030002B6A46DB
:100890004FF0000143DA137812F8010F01315B00C9
:1008A00043EAD0130F2902F8013CF4D19DF80F3030
:1008B0005B0083F08703D4F81401DBB210288DF8B5
:1008C0000F303BD104F58073694604F5887013F846
:1008D000016F11F8012B984282EA06021A70F6D1D4
:1008E00004F1F00304F5807113F8012F187C8B429A
:1008F00082EA00021A70F7D110220DEB020004F117
:10090000F10100F085FD2246294604A800F062F9B5
:1009100010220021684600F08FFD09B0F0BD137869
:1009200012F8010F01315B0043EAD0130F2902F8DE
:10093000013CF4D19DF80F305B00BCE79DF900301D
:10094000002B6A464FF0000137DA137812F8016F76
:1009500001315B0043EAD6130F2902F8013CF4D1C0
:100960009DF80F305B0083F08703471CDBB28DF8E6
:100970000F30102F04EB0003C0F10F064FF0800280
:1009800088BF002600F5817083F8012100213246DE
:1009900020443E4403F072FAC4F8146104F58073F5
:1009A000694604F5887013F8016F11F8012B98421D
:1009B00082EA06021A70F6D192E7137812F8016FF4
:1009C00001315B0043EAD6130F2902F8013CF4D150
:1009D0009DF80F305B00C8E70A7803785340037036
:1009E0004A784378534043708A78837853408370C1
:1009F000CA78C3785340C3700A79037953400371AE
:100A00004A794379534043718A798379534083719A
:100A1000CA79C3795340C3710A7A037A5340037287
:100A20004A7A437A534043728A7A837A5340837274
:100A3000CA7AC37A5340C3720A7B037B5340037361
:100A40004A7B437B534043738A7B837B534083734E
:100A5000CA7BC37B5340C373704710B50B781478BF
:100A60006340037054784B786340437094788B787C
:100A700063408370D478CB786340C37014790B796A
:100A80006340037154794B796340437194798B7956
:100A900063408371D479CB796340C371147A0B7A44
:100AA00063400372547A4B7A634043728B7A947A30
:100AB00063408372D47ACB7A6340C372147B0B7B1E
:100AC00063400373547B4B7B63404373947B8B7B0A
:100AD00063408373CB7BD27B5340C37310BD000054
:100AE000A1F11003DBB2102B2DE9F04704D8374CED
:100AF00024FA03F3DB0705D4002382F8F030FF204B
:100B0000BDE8F087531E4418A0424ED101F11C03EA
:100B10009B005FFA83F9C3F30313013B2C4D82F86A
:100B2000F03001240B46D618B3FBF1F001FB103076
:100B300010F0FF0016F804AC16F803EC16F802CC1F
:100B400016F8017C36D115F80E8015F80CE015F872
:100B500007C015F80A70E00900EB400084EA0808B5
:100B600000EBC0006400C0B2E4B24440C246581A70
:100B7000C0B212F800808AEA080A02F803A0104402
:100B8000043390F801808EEA080E86F801E090F8B0
:100B900002E08CEA0E0C86F802C0C078DBB2474057
:100BA0009945F770BFD80020AAE710F8015B03F859
:100BB000015FA9E71829DAD9102801BF15F80AA0A2
:100BC00015F80EE015F80CC0EF5DD0E7010101004B
:100BD000604601082DE9F04FA3B092F8F0301D9166
:100BE0001B920193002B00F0538101461EA8FFF7D2
:100BF00034FF1B9BA74CA84DA84E10330293002333
:100C000003939DF87C0004909DF886000590205C7D
:100C100006909DF87B000790205C089004989DF852
:100C200081C0205C099014F80C000A909DF88000A7
:100C30000B909DF885009DF878809DF87DE09DF8EB
:100C400082A09DF887900C909DF87A00029B1C93DF
:100C500014F80A2014F8093014F8081014F80E706B
:100C60000D90205C0E909DF87F000F90205C1090FE
:100C70000B98205C11900C98205C12909DF88400D9
:100C800013909DF8790014909DF87E001590205CDB
:100C900016909DF883001790205C18901398205CA4
:100CA00019901498205C1A900398013003900298D0
:100CB000DDF804B0103002909DF80C00834536D862
:100CC0008DF878108DF87A2009990E9A8DF87C109D
:100CD0008DF882201199069A8DF880108DF87E206B
:100CE0001999169A8DF884108DF886200A99189A09
:100CF0008DF87D108DF887201299109A8DF87B3031
:100D00001B9B8DF881108DF883201A99089A1D98E5
:100D10008DF885108DF87F201EA903EB0B128DF83E
:100D20007970FFF79AFE002023B0BDE8F08F15F828
:100D300008B082EA03008BEA000016F80EB080EAE1
:100D40000B008DF8780015F80E004B40434016F864
:100D50000A0043408DF8793081EA070315F80A103C
:100D6000594016F80930594016F808308DF87A10B5
:100D70007A40534015F8092053408DF87B30089A8B
:100D8000069B5340049AAA5C534016F80C2053402B
:100D90008DF87C30DDE908325A4015F80C305340AC
:100DA000059AB25C53408DF87D30DDE909325A4036
:100DB000059BEB5C5340079AB25C53408DF87E3044
:100DC000069B0A9A5340049AB25C5A40079BEB5C1C
:100DD0005A408DF87F200E9B109A53400B9AAA5CC4
:100DE00053400C9AB25C53408DF88030DDE91032EC
:100DF0005A400C9BEB5C53400D9AB25C53408DF80B
:100E00008130DDE911325A400D9BEB5C53400F9A63
:100E1000B25C53408DF88230129A0E9B53400B9A6D
:100E2000B25C5A400F9BEB5C1C995A408DF88320B2
:100E3000169B189A5340139AAA5C5340149AB25CBA
:100E400053408DF88430DDE918325A40149BEB5C36
:100E50005340159AB25C53408DF88530DDE9193264
:100E60005A40159BEB5C5340179AB25C53408DF887
:100E700086301A9A169B5340139AB25C5340179AC5
:100E8000AA5C1EA853408DF88730FFF7A5FDB8E691
:100E9000FF2049E7604601086044010860450108F9
:100EA00008B538B1044A05491060D82200F0B0FAFC
:100EB000002008BD0220FCE748240020904B0108D8
:100EC0000A4B1A6870B5002302F1180503EB0314EE
:100ED0002E5D864204D1183422440A60002070BD81
:100EE00001330B2BF2D10320F9E700BF4824002087
:100EF0002DE9F041CCB00646DDF8488117461C4686
:100F00000D4631B3B8F1000F23D006A8FFF72EFC31
:100F1000204601A9FFF7D4FF0446B0B9019906A8FD
:100F20000131FFF733FC26B11022314606A8FFF746
:100F300032FC3A46294606A8FFF72DFC06A902A86E
:100F4000FFF794FC029BC8F8003020464CB0BDE887
:100F5000F0810224F9E7000030B595B013A90446EA
:100F6000FFF7AEFF002830D11B490C2303FB00F232
:100F7000555CA5422BD1139B187C1090D87B0F9009
:100F8000987B0E90587B0D90187B0C90D87A0B9024
:100F9000987A0A90587A0990187A0890D879079028
:100FA000987906905879059018790490D87803902C
:100FB000987802900A445B7801939368009300222A
:100FC000064B1146022002F019FA15B030BD01306F
:100FD0000B28CBD1F9E700BFD848010860470108CA
:100FE0000B2B10B402D810BCFFF782BF032010BC3B
:100FF000704730B50D4685B01446014668B103AA66
:10100000002000922A460390FFF772FF18B9039858
:10101000001B18BF012005B030BD0220FBE72DE901
:10102000F0430D46BFB014469946804620B31BB32B
:1010300011F00F0122D1F02201A800F0FDF92046A5
:101040006946FFF73DFF044648B9009801AA102100
:101050000130FFF745FD2E46AF1BFFB21EB92046FB
:101060003FB0BDE8F08301AA09EB070108EB0700D8
:10107000FFF7B0FD103EEFE70224F0E70524EEE7AE
:10108000F0B5184E3468024685B00846002304F1D6
:10109000180103EB03154F5D97421ED10D2A05F190
:1010A000190513D10023CDE90033CDE902330C2219
:1010B00010216B46FFF7B3FF0446306810226946E3
:1010C000284400F0A5F9204605B0F0BD01461022E5
:1010D000601900F09DF90024F5E701330B2BD8D1FE
:1010E0000324F0E74824002009B1FFF7C9BF02201C
:1010F00070471FB51446A0B10C2A01D10B2912D19B
:101100000023CDE90033CDE902330A466B461021B6
:10111000FFF785FF18B969462046FFF7B1FF04B015
:1011200010BD0220FBE70320F9E7F8B51E46DDE914
:1011300007479DF818505BB354B34FB3212D29D8FE
:1011400019462A46204600F063F90122631C691EF5
:10115000B018FFF764FFF8B9E37ADB093B70EBB92D
:101160006319204613F8012C13F8021C120642EAF8
:10117000014213F8041C0A4313F8031C012342EA3A
:101180000122291FFFF735FF003818BF0120F8BDE5
:101190000220FCE70520FAE70720F8E70420F6E73D
:1011A00010B5044628B1044B5B69984720600020C5
:1011B00010BD0220FCE700BFF049010808B5014658
:1011C00030B1044B0822186800F022F9002008BD55
:1011D0000220FCE74824002008B530B1044B082267
:1011E000196800F015F9002008BD0220FCE700BFD7
:1011F000482400207FB5124E0023044602A8019324
:101200000D46FFF7E9FF33685B6901936CB102AAF1
:10121000082312F8011B41B9013B13F0FF03F8D179
:1012200002A8A04702A8FFF7C9FF35B1019B23B967
:1012300001A8A8473368019A5A61002004B070BD24
:101240004824002008B5014638B1054B186808222B
:10125000104400F0DDF8002008BD0220FCE700BFCC
:101260004824002008B538B1044B196808221144FD
:1012700000F0CEF8002008BD0220FCE74824002042
:10128000034B1B6802280CBF19615961002070478D
:101290004824002041B1054B1B6802280CBF1B6984
:1012A0005B690B60002070470220704748240020D3
:1012B00030B58FB0002405460CA80994FFF78CFFC9
:1012C0009DF8373007939DF8363006939DF83530FA
:1012D00005939DF8343004939DF8333003939DF8C3
:1012E000323002939DF8313001939DF830300093F5
:1012F000224621461E4B022002F080F80AA8FFF782
:10130000B1FF9DF82F3007939DF82E3006939DF87E
:101310002D3005939DF82C3004939DF82B300393CA
:101320009DF82A3002939DF8293001939DF82830CA
:10133000009322460F4B2146022002F05FF809A9D4
:101340002846FFF7A7FF9DF8243003939DF825302A
:1013500002939DF8263001939DF827300093224692
:10136000054B2146022002F049F80FB030BD00BF06
:10137000BC470108FA4701083848010808B50020B1
:10138000FFF7EAFD0120FFF7E7FD0920FFF7E4FD85
:101390000820FFF7E1FD0020FFF78AFF002008BDCD
:1013A00010B504460B20FFF7D7FD0C20FFF7D4FD46
:1013B0000920FFF7D1FD0820FFF7CEFD0A20FFF737
:1013C000CBFD2046FFF774FF002010BD014B1860D5
:1013D000704700BFAC0800200B4A30B514680B4DB5
:1013E00043F2390305FB04331360091A6FF000421E
:1013F000B3FBF2F2C2EBC27201319B1A93FBF1F222
:1014000001FB1233184430BDAC0800206D4EC641BC
:1014100001380A44914200D1704711F8013B00F8AD
:10142000013FF7E710440A44914200D1704711F898
:10143000013B00F8013DF7E702F020BD30B530B1C7
:101440000A4D01444FF0FF33814201D1D84330BDF2
:1014500010F8012B5340082243F30004013A2C40BA
:1014600092B284EA5303002AF6D1EDE72083B8ED67
:1014700001207047054B4FF400529A62044B1B68E1
:1014800013B15B6803B11847704700BF0004004800
:101490004C250020054B4FF480529A62044B1B6888
:1014A00013B1DB6803B11847704700BF0004004860
:1014B0004C250020012070470120704701F048B9F9
:1014C00001F036B910B501F019FE0E21044640F6C0
:1014D0001F1001F02DF92046012101F0F9FDBDE8B2
:1014E000104001F0D7BA000070B50C4E01EB40037C
:1014F0000D46B3654FF6FF71002304461A460846B1
:1015000001F05EFB96F85600002101F0E1FD29464E
:101510002046BDE8704001F095BA00BF6825002064
:1015200010B5044601F0AAFE01281CD101F0AEFE60
:1015300034B11248214602F017FB104802F0DAFAE3
:101540000F4C104B00214FF48052A1659A6194F822
:10155000560001F0BDFD63786BB16FF07F40BDE8D0
:10156000104001F053BA002340F262211A460846A7
:1015700001F026FBDCE7A0688001F0E750250020A1
:101580006825002000040048002001F0BFB90000D9
:1015900008B501F0C7F80438C0B2032896BF024B63
:1015A0000020185C08BD00BFEC49010808B501F037
:1015B000BAFD033008BD01F049B901F009B908B519
:1015C00001F000FD00B208BD38B50D46144601F02B
:1015D0005DFB284601F092FD0E21054640F61F10E6
:1015E00001F0A6F828460121074D01F071FD01F038
:1015F00051FA4FF47A716143284602F0B5FA284651
:10160000BDE8384002F076BAC425002001F03EBBA8
:1016100008B5084B002193F8560001F059FD00234E
:101620004FF4C0711A46084601F0CAFABDE80840F6
:1016300001F024BA6825002010B5044601F01EFE12
:1016400001281CD101F022FE34B11248214602F0DB
:101650008BFA104802F04EFA0F4C104B00214FF459
:101660008052A1659A6194F8560001F031FD6378CB
:101670006BB16FF07F40BDE8104001F07DB90023F1
:1016800040F262211A46084601F09AFADCE7A068A7
:101690008001F0E750250020682500200004004864
:1016A00008B54FF0040001F017F9BDE8084002202A
:1016B000F1F72EBA08B500231A461946184601F06C
:1016C0007FFABDE8084001F06DB900001D4B73B50D
:1016D0001D4D186000241D486C70C5E90144AC65BF
:1016E00001F098FAAC8101F003FA2146204601F09E
:1016F0004BFC21460422012001F0FCFA144E154D4A
:101700004FF6FF7123462246084601F059FAFFF7CB
:10171000C7FF2246104B00944FF0FF31304602F0D5
:101720003DF90E4B009422464FF0FF31284602F05F
:1017300035F9304602F090F9284602B0BDE8704015
:1017400002F08AB94C2500206825002015270108E1
:10175000C4250020502500207514010895140108A7
:101760000128084805D1084BC17719700E3001F0E7
:10177000A7BB437D012B03D1034B81751970F5E79E
:10178000704700BF68250020B00800200D4B10B541
:10179000044618735873012000F016F85CB1342128
:1017A0004FF4E86000F0C4FF4421BDE8104040F26F
:1017B000417000F0BDBF14214FF4E86000F0B8FFA5
:1017C0002421F2E76825002038B5114C0546207029
:1017D00001F061FD052D04D8DFE805F0090B0317C2
:1017E0001709032001F070FA0023637338BD00204D
:1017F000F8E7012001F068FA207B637B8342F5D093
:101800006073BDE83840FFF7C1BF0220EAE700BFC0
:10181000682500202DE9F0431E4687B000230546C9
:10182000CDE901330C46174601F027FD032D61D8A1
:10183000DFE815F07B00C3000E010400A27C082A3B
:1018400004D94FF0FF3007B0BDE8F083A16801A8CC
:1018500001F0DCFE21680029F3D042F210729142BF
:10186000E37C864D51D80322AA7385F83820E963BA
:1018700085F844304FF002086368A17DDB002B82BD
:101880000423AB74A37CDB00EB7402294FF000034C
:101890002B75637D02D0227D022A42D103F10F0213
:1018A000D2B2012A01D9012BCBD1754B754A1968E7
:1018B00003944FF0010903A88DF8149001F0DAFCAD
:1018C0000028BED1287685F817906875FFF75CFE72
:1018D0004046FFF779FF6C4801F086FA6B4801F04B
:1018E000EFFA01A800F084FF208A00F055FFA089DC
:1018F00000F09AFF384601F001FC604C84F8560075
:1019000001F0C0FC666000209DE74FF00008E9632D
:10191000890885F80E8085F8388085F84430296478
:10192000AAE7EB7529766A75D0E72368002B88D083
:10193000A27C082A85D8514DA16801A801F066FE55
:10194000002385F838302268EA63E27C85F8442079
:10195000A269AB732A646268A17DD2002A82042244
:10196000AA74A27C2B75D2000229637DEA7402D08E
:10197000227D022A1DD103F10F02D2B2012A02D91F
:10198000012B7FF45EAF3E4B3E4A196803944FF043
:10199000010803A88DF8148001F06CFC00287FF486
:1019A00050AF287685F817806875FFF7EDFD0020A9
:1019B0008FE7EB7529766A75F7E7304D012185F8D9
:1019C0003810227885F85020637885F85130A37854
:1019D00085F85230E3788B4202D0022B03D03BB91A
:1019E00085F8533004E00B3A012A29D885F85310C2
:1019F0004FF0010885F80E80A388AB83A379AB77FD
:101A0000E37985F82030237A85F82130FFF7BCFD93
:101A10004046FFF7D9FE1C4801F0E6F91B4801F0EB
:101A20004FFA95F85130062B40F689000AD100F0A4
:101A30008FFE00F0FB0140F6890000F079FE59E7C7
:101A40000023CDE700F084FE40F00401C9B2F2E7C4
:101A50002368013BB3F57A7FBFF4F3AE0320FFF7B1
:101A6000B3FE0648022380F83830236883641623C7
:101A700080F84C30383001F0B7F93BE7682500209A
:101A80004C250020C4250020A0250020762500201C
:101A90002DE9F041002686B01F461446CDE90166C7
:101AA00080460D4601F0E9FBB442764C16BF012397
:101AB000334637466370B8F1000F06D0B8F1010F16
:101AC0007CD0002006B0BDE8F081AB68002B00F0B0
:101AD000D680EB68002B00F0D280AA7F082A00F2A3
:101AE000CE80296901A801F091FD2868003818BF4F
:101AF000012000F0D9FF84F83880AB68E36395F8E3
:101B0000203084F84430686801F05AFB84F80E8075
:101B100084F84500EB68DB002382EB7FA374AB7F86
:101B2000DB00E37495F82130237595F82230002B03
:101B30003ED12A7D95F82410A275022995F823201C
:101B400001D0022B36D102F10F03DBB2012B02D9F7
:101B5000012A40F0948000238DF814304A4B4B4A00
:101B60001968049503A801F085FB002840F08780E0
:101B700001232076E3756075FFF706FD0020FFF76F
:101B800023FE434801F030F9424801F099F901A8D9
:101B900000F02EFEA88B00F0FFFD288B00F044FE25
:101BA0004FF4FA53AA687B43B3FBF2F3A36088E7D0
:101BB000FF22BFE7E27521766375DDE72B8E002BF0
:101BC0005DD095F83230A86A012B0CBF95F81480CF
:101BD0004FF0FF08003818BF012000F065FFF8B291
:101BE00000F06EFF012184F8381095F82C2084F85D
:101BF000502095F82D3084F8513095F82E3084F827
